:020000040000FA
:0400000039EF0AF0DA
:0800080058EF0AF0186A1C6AA7
:100010001B6E010E086E1C50185C02E11B50175C31
:10002000040ED8B0010ED8B4020E0814D8A4010EE4
:100030001200800E016EFE0EADEC02F0010EADEC72
:1000400002F0750E186E300E26EF03F0016A018E75
:10005000266EFE0EADEC02F02650ADEF02F0056A02
:10006000800E326E00D01F6A206A216A226A089AC6
:10007000B3EC02F0D8A01200D30FD8B4088A2D0F29
:10008000C60FF6E20A0FF4E31B6E1A6A196A186AC1
:100090000A0E176EA4EC03F01B5017241F6E1850A5
:1000A000206E000ED8B0010E20261950216E000ED1
:1000B000D8B0010E21261A50226E000ED8B0010EC3
:1000C0002226050608E0B3EC02F0D8A01200C60F05
:1000D00002E20A0FD9E208AA0BD01F1E201E211E21
:1000E000221E1F2AD8B4202AD8B4212AD8B4222A02
:1000F0001F50D8801200056A1F6E206A00960550B6
:10010000D8B40086050E046E270E1C6E100E0CD897
:10011000030E1C6EE80E08D81C6A640E05D81C6A13
:100120000A0E02D81F5008D01B6E2050186E1F50A8
:10013000176E8DEC03F01750176E044E00960550A5
:1001400003E0045CD8B008D01750D8A4009600B6DD
:1001500003D0300FADEF02F012002E6E0CC039F05C
:10016000D880E86A0E220D220C2202E32CD90B2A39
:1001700036900CBE03D07F0E0B6008D00CAE05D0BD
:10018000800E0C5C7F0E0B5801E2368039AE0C9E5F
:10019000106A126A116A306A0CAE01D02E8C0C8E75
:1001A0000B506DE07F0E0B5C43E30B6E316A040E67
:1001B000346E01D9342EFDD7040E0B5C06E2030E1B
:1001C0000B5C57E10A0E305C54E3030E0B5E312AE0
:1001D000E9D8F1D8D2D8020E346EF3D8342EFDD738
:1001E000E1D8040E346ED8900F3210321132123230
:1001F000342EF9D7C2D8D6D811C012F010C011F0E1
:100200000FC010F00F6AB9D8CDD810C012F00FC0CF
:1002100011F00F6A106AB1D830B6CED70B5205E193
:100220000E2A0D2A0C2A302A24D0C5D80B06C4D792
:100230000B1E0B2A7F0E0B26316A040E346EBBD8C0
:10024000342EFDD7040E0B26050E0B5C1AE3AAD83C
:10025000B2D8B1D892D8AFD8312A030E346EB1D803
:10026000342EFDD7030E0B5E30A8EED7AAD80B06AE
:10027000EBD70B1E0B2A030E0B26010E03D0020E2A
:1002800001D0000E356E2D0E2EBC67D92E9E2E9CF1
:1002900035A007D031C035F031C039F02E283926CD
:1002A00027D035A202D02E28316E2E52D8B412009B
:1002B000300E36B052D92E0E50D931C02DF02D0649
:1002C0002E502D5C02E32EC02DF02D5204E0300E96
:1002D00044D92D2EFCD731C034F02E28345ED8B04E
:1002E00012000B062E28396E3150395E39C035F0B8
:1002F00030C037F00B5005E02C6ED89037322C2EE2
:10030000FCD73950D8B41200300E372426D93550D6
:1003100008E12E52D8B41200300E36B01ED92E0E7F
:100320001CD93506394E12000B5005E02C6ED890C2
:1003300037362C2EFCD73750305E30C00FF00CC053
:1003400010F00DC011F00EC012F035D834D8125094
:100350000E2605E30D2A03E10C2A01E1302A115093
:100360000D2603E30C2A01E1302A10500C26D8B0E8
:10037000302A0F5030261FD8BBD712500E2605E367
:100380000D2A03E10C2A01E1302A11500D2603E366
:100390000C2A01E1302A10500C26D8B0302A0F5018
:1003A0003026120030C00FF00CC010F00DC011F05C
:1003B0000EC012F01200D8900E360D360C363036C4
:1003C0001200D89030320C320D320E32120027D883
:1003D0000096055003E100860A0E056E2DC01AF046
:1003E0002CC019F02BC018F02AC017F0046A226A3A
:1003F000216A206A0A0E1F6E33D9042A0450055C54
:10040000D8A4F5D71F50D8A4009600A602D0052C7A
:1004100003D01F50300FA1D8052EE0D712002DAE0B
:1004200012002A1E2B1E2C1E2D1E2A2AD8B42B2A5F
:10043000D8B42C2AD8B42D2A2D0E8FD0246E8A94AD
:1004400000008A96939493960F0E9316245000B250
:100450001ED03A0E186E980EF9D8330E236E29D896
:10046000130E186E880EF2D824D8640EEED821D858
:10047000640EEBD8220E236E1CD8280E07D80C0E63
:1004800005D8060E03D80082245001D00080236EC8
:1004900000A00AD08A9603080BE30AD8070E186E4C
:1004A000D00ED4D8D88012000080FE0814E08A86CE
:1004B00000A000908A840F0E81162350F00B811249
:1004C000000000D08A94233A000000D000B0F1D799
:1004D000FF0EBBD8D88024501200086E1B6E92907D
:1004E000090E1C6ED89007D81B321C2EFCD7D88062
:1004F00002D80850120003E20000808002D08090F1
:1005000000D0660EA2D0ABB2AB98AB8803C017F098
:1005100006C018F01B6A1C6A000000D000009EBADA
:1005200014D0E8681B261C2217221822D8A012001B
:100530001B481C3CF1D7E80E1B6E010E1C6EEED75B
:10054000ABB2AB98AB889EAAFED7AE50D880120053
:100550009EA8FED7AD6ED880120001BE6FD701BC39
:10056000BCD701B4F5D73252CEE03204E9E0D880EE
:1005700032BEEE5012001F6E0F0EEA6E0350120FC5
:10058000E96E0650EF1203C0E9FFEF1428A0061829
:1005900010E01F6607D02650FF0F0CE3C80E48D8A6
:1005A000265008D01F28FF0E04E01F2C02D0275031
:1005B00001D0291E29321200AA6AA96EA66AA68055
:1005C000A850A94AAA2A1200AA6AA86EA66AA684F6
:1005D000550EA76EAA0EA76EA682A6B2FED7A69447
:1005E000A94AAA2A1200A96EAA6A026AA66AA68065
:1005F000A8CF04F0A94AAA2A0450D8B41200ADDF4B
:10060000023EF4D71200E836E8363C0B0109C2126C
:10061000C009C216C050F80B0309C06EC80E15D829
:10062000C282C2B2FED7C4CF2BF0C3502A6E1200D2
:100630001C6A1B6EFF0E1B261C2200D0D8A01200C5
:10064000030E186EE70E02D8F5D7186AFD0F176E65
:1006500001D01706000000D0E86A185AFAE212002A
:100660001A502218800BF46E1AAE06D0D880000EF5
:100670001756185619561A5622AE06D0D880000EB4
:100680001F562056215622561B6A1C6A1D6A1E6A76
:100690002E6A2F6A306A316A2250211020101F10F2
:1006A00023E0200EF36ED8901736183619361A3616
:1006B0002E362F36303631361F502E5C20502F58B4
:1006C000215030582250315809E31F502E5E2050DF
:1006D0002F5A2150305A2250315AD8801B361C369E
:1006E0001D361E36F32EDFD7F4AE06D0D880000EAE
:1006F0001B561C561D561E561BC017F01CC018F06A
:100700001DC019F01EC01AF02EC01FF02FC020F01F
:1007100030C021F031C022F01200206A1F6A100E92
:10072000F36E18341F3620361B501F5C1C502058A7
:1007300005E31B501F5E1C50205AD8801736183610
:10074000F32EEFD7175012001AC031F019C030F055
:1007500018C02FF017C02EF030501F02F3CF19F041
:10076000F4CF1AF02F502002F3501926F4501A2219
:100770002E502102F3501926F4501A2231501F0234
:10078000F3501A2630502002F3501A262F5021021F
:10079000F3501A262E502202F3501A262E501F0212
:1007A000F3CF17F0F4CF18F02F501F02F350182694
:1007B000F4501922000E1A222E502002F35018264F
:1007C000F4501922000E1A221200F34E02D0E65203
:1007D000FCD7E6CFEEFFE82EFCD712000CD8F80EBF
:1007E000126E0F0E116EC90E106E7F0E0F6E50EC52
:1007F00008F00C9E12000E50126E166E0D50116E07
:10080000156E0C50106E146E0B500F6E136E4AEC7A
:1008100009F00EC012F00DC011F00CC010F00BC0AA
:100820000FF00E6A0D6A0C6A7F0E0B6E4EEC08F02C
:10083000F4EC06F00EC012F00DC011F00CC010F078
:100840000BC00FF016C00EF015C00DF014C00CF068
:1008500013C00BF0E2EC08F0316A0EC01AF00DC0C4
:1008600019F00CC018F00B50176E05E00CAE03D059
:100870003180800E181A18BE21D0010E1A5C000EAD
:100880001958000E18587F0E175818E30E6A0D6A93
:100890000C6A7F0E0B6E1AC012F019C011F018C04E
:1008A00010F017C00FF0E2EC08F00EC01AF00DC007
:1008B00019F00CC018F00BC017F031820A0E0E6E42
:1008C000890E0D6E340E0C6E7C0E0B6E1AC012F07B
:1008D00019C011F018C010F017C00FF04AEC09F061
:1008E0001AC012F019C011F018C010F017C00FF0A4
:1008F0004AEC09F07C0E126E790E116E350E106EF8
:10090000810E0F6E50EC08F01AC012F019C011F0F1
:1009100018C010F017C00FF04AEC09F01AC012F01E
:1009200019C011F018C010F017C00FF04AEC09F010
:100930003F0E126E020E116E330E106E830E0F6E8E
:1009400050EC08F01AC012F019C011F018C010F0E5
:1009500017C00FF04AEC09F01AC012F019C011F0DC
:1009600018C010F017C00FF04AEC09F0330E126EE9
:100970008C0E116E1E0E106E830E0F6E50EC08F072
:100980000EC01EF00DC01DF00CC01CF00BC01BF003
:100990001A500E6E19500D6E18500C6E17500B6ECB
:1009A0001AC012F019C011F018C010F017C00FF0E3
:1009B0004AEC09F01B0E126EE40E116E350E106E2D
:1009C000820E0F6E50EC08F01AC012F019C011F030
:1009D00018C010F017C00FF04AEC09F01AC012F05E
:1009E00019C011F018C010F017C00FF04AEC09F050
:1009F000A40E126EDB0E116E670E106E830E0F6E5C
:100A000050EC08F01AC012F019C011F018C010F024
:100A100017C00FF04AEC09F01AC012F019C011F01B
:100A200018C010F017C00FF04AEC09F0330E126E28
:100A30008C0E116E1E0E106E830E0F6E50EC08F0B1
:100A40000EC022F00DC021F00CC020F00BC01FF032
:100A50001AC00EF019C00DF018C00CF017C00BF042
:100A60001EC012F01DC011F01CC010F01BC00FF012
:100A70004AEC09F022C012F021C011F020C010F0A1
:100A80001FC00FF0E2EC08F00EC012F00DC011F024
:100A90000CC010F00BC00FF031A20AD0DB0E0E6EAE
:100AA0000F0E0D6E490E0C6E7F0E0B6E4EEC08F0A5
:100AB00031A002D0800E0C1A0E5012000EC02BF086
:100AC0000DC02CF00CC02DF00BC02AF01BD80EC0AE
:100AD00014F00DC015F00CC016F00BC013F02BC0B5
:100AE0000EF02CC00DF02DC00CF02AC00BF00CD86D
:100AF00014C012F015C011F016C010F013C00FF0A2
:100B0000E2EF08F0010E01D0000E1F6E36C021F09A
:100B1000368C226A1F6602D00CBE228E0C9E880E76
:100B20000B60368A0EC017F00DC018F00CC019F01B
:100B30000BC01AF0830E126EF90E116E220E106E9B
:100B40007F0E0F6E4AEC09F0369C9AEC09F0368C59
:100B50000EA004D00E2A000E0D220C22070E0E1439
:100B6000206E030E206404D0800E221A040E205E34
:100B70000B6AF6EC09F00B501E6E6DE00EC01BF018
:100B80000DC01CF00CC01DF0126A0F0E116EC90EC4
:100B9000106E7E0E0F6E4AEC09F017C012F018C0EE
:100BA00011F019C010F01AC00FF050EC08F00EC090
:100BB00017F00DC018F00CC019F00BC01AF01BC0D4
:100BC0000EF01CC00DF01DC00CF01EC00BF0126A20
:100BD000A20E116EDA0E106E6E0E0F6E4AEC09F058
:100BE00017C012F018C011F019C010F01AC00FF0A1
:100BF00050EC08F00EC017F00DC018F00CC019F042
:100C00000BC01AF01BC00EF01CC00DF01DC00CF084
:100C10001EC00BF0200E126EA20E116E850E106E0D
:100C20005C0E0F6E4AEC09F017C012F018C011F0FC
:100C300019C010F01AC00FF050EC08F00B501A6EEB
:100C40000F6E0C50196E106E0D50186E116E0E5006
:100C5000176E126E0CD01A500B6E0F6E19500C6E70
:100C6000106E18500D6E116E17500E6E126E4AEC0B
:100C700009F00EC01BF00DC01CF00CC01DF00BC025
:100C80001EF020302018010B1F184DE0CE0E126E02
:100C9000F50E116E4C0E106E6F0E0F6E4AEC09F0D1
:100CA0001A0E126E060E116EB60E106E750E0F6EC7
:100CB000F7D91BC012F01CC011F01DC010F01EC0EF
:100CC0000FF04AEC09F0A50E126EAA0E116E2A0E54
:100CD000106E7A0E0F6EE4D91BC012F01CC011F01A
:100CE0001DC010F01EC00FF04AEC09F01BC012F03E
:100CF0001CC011F01DC010F01EC00FF04AEC09F02E
:100D00001BC012F01CC011F01DC010F01EC00FF06F
:100D10000F660F06C3D9369C126A116A106A7F0EDD
:100D20000F6EBED956D0F90E126E680E116E360EC9
:100D3000106E6C0E0F6E4AEC09F0C00E126E070EAC
:100D4000116ED00E106E720E0F6EAAD91BC012F06B
:100D50001CC011F01DC010F01EC00FF04AEC09F0CD
:100D6000840E126E880E116E080E106E780E0F6EC5
:100D700097D91BC012F01CC011F01DC010F01EC08E
:100D80000FF04AEC09F0AB0E126EAA0E116E106E47
:100D90007C0E0F6E85D91BC012F01CC011F01DC057
:100DA00010F01EC00FF04AEC09F017C012F018C086
:100DB00011F019C010F01AC00FF04AEC09F0369C7F
:100DC00017C012F018C011F019C010F01AC00FF0BF
:100DD00067D9800E1F5202E020B2221A22BE0C1ADE
:100DE00021BC368C0E5012000CBEA5D00B52D8B4CC
:100DF000A3D00BC020F036C021F0368C7F0E0B6ED6
:100E0000126A116A106A0F6E49D90EC017F00DC030
:100E100018F00CC019F00BC01AF0130E126ECB0EA6
:100E2000116E030E106E840E0F6E3AD917C012F0B9
:100E300018C011F019C010F01AC00FF04AEC09F0F8
:100E4000BC0E126E5A0E116E050E106E860E0F6ECF
:100E500027D917C012F018C011F019C010F01AC02D
:100E60000FF04AEC09F0830E126E300E116E720E06
:100E7000106E850E0F6E14D90EC01BF00DC01CF045
:100E80000CC01DF00BC01EF017C00EF018C00DF006
:100E900019C00CF01AC00BF08E0E126ED70E116E28
:100EA0006B0E106E810E0F6EF5D9B50E126E290EF7
:100EB000116E4E0E106E840E0F6EF2D817C012F027
:100EC00018C011F019C010F01AC00FF0E3D9800E4D
:100ED000126E300E116E720E106E840E0F6EE0D810
:100EE0001BC012F01CC011F01DC010F01EC00FF08E
:100EF00069D917C012F018C011F019C010F01AC04B
:100F00000FF0C8D9126A116A106A7F0E0F6EC8D826
:100F100020B009D0F30E126E040E116E350E106E55
:100F20007F0E0F6EB7D97F0E202620300B6E21BCAE
:100F300003D0369C01D0368A0E50120010500C1887
:100F4000386E38BE30D010BE17D00F500B5CD8A012
:100F5000000CD8A4010C10500C5CD8A0000CD8A434
:100F6000010C11500D5CD8A0000CD8A4010C12503B
:100F70000E5CD8A0000C010C0B500F5CD8A0000C2C
:100F8000D8A4010C0C50105CD8A0000CD8A4010C03
:100F90000D50115CD8A0000CD8A4010C0E50125CAE
:100FA000D8A0000C010C0CAE010C000C10500C1859
:100FB000386E38BE34D010BE19D00F500B5CD8A09C
:100FC000000CD8A4010C10500C5CD8A0000CD8A4C4
:100FD000010C11500D5CD8A0000CD8A4010C1250CB
:100FE0000E5CD8A0000CD8A4010C000C0B500F5CB8
:100FF000D8A0000CD8A4010C0C50105CD8A0000C98
:10100000D8A4010C0D50115CD8A0000CD8A4010C80
:101010000E50125CD8A0000CD8A4010C000C0CAE31
:10102000010C000C0C501018386E38BE34D00CBEB9
:1010300019D00B500F5CD8A0000CD8A4010C0C5098
:10104000105CD8A0000CD8A4010C0D50115CD8A0E5
:10105000000CD8A4010C0E50125CD8A0000CD8A42F
:10106000010C000C0F500B5CD8A0000CD8A4010C94
:1010700010500C5CD8A0000CD8A4010C11500D5CD1
:10108000D8A0000CD8A4010C12500E5CD8A0000C03
:10109000D8A4010C000C10AE010C000C800E101A2C
:1010A0000F500B5C356E11E2356C0B500FC00BF01E
:1010B0000F6E0C5010C00CF0106E0D5011C00DF0E2
:1010C000116E0E5012C00EF0126E1A0E356078D0EE
:1010D0000F5276E0346A0C50376E1018396E0C8E51
:1010E000108E080E355E08E312C034F011C012F005
:1010F00010C011F0106AF5D7352607E0D8901032ED
:10110000113212323432352EF9D739AE35D0125071
:101110000E5E11500D5A10500C5A07E2D880000E86
:101120000E560D560C56800E371A346C04E00E061F
:10113000000E0D5A0C5A040E356E0C660DD00DC003
:101140000CF00EC00DF034C00EF0346A080E0B5EC9
:101150002DE3352EF2D72AD00CBE08D0D8903436E5
:101160000E360D360C360B2EF7D720D036AC26D0E7
:1011700034AE24D0346A11D012500E2611500D22F4
:1011800010500C2206E30C320D320E3234320B4A70
:101190000FD036AC13D034AE11D00E3E0FD00D3E72
:1011A0000DD00C3E0BD0D8800E90EDD70B6A02D03C
:1011B00036820B680E6A0D6A800E0C6E37AE0C9E7E
:1011C0000E5012000C50306E1018396E0F5053E054
:1011D0000B5254E00B5E7F0E03E20B2603E24DD070
:1011E0000B264EE20EC02EF00DC02FF0308E108E6A
:1011F000180E376E0E6A0D6A0C6A0BD012502E5CF8
:1012000011502F5811E32F6E306A12502E5E0BD002
:1012100004E21050305CF2E007E312502E5E1150F1
:101220002F5A1050305AD8800E360D360C362E36C6
:101230002F363036372EECD70CBE07D00B521DE0C0
:1012400039320B06372A3936E3D736AC1FD007E2DE
:1012500012502E5E11502F5A1050305A17E30E3E86
:1012600015D00D3E13D00C3E11D00C320D320E3283
:101270000B3E0CD005D0368604D036840B6A02D0E3
:1012800036820B680E6A0D6A800E0C6E39AE0C9EAB
:101290000E5012000C50306E1018396E0B50D8A43E
:1012A0000F503CE00B267E0E03E30B5E03E338D0C9
:1012B0000B5E33E30EC02EF00DC02FF0308E108E7B
:1012C0000E6A0D6A0C6A180E376E30322F322E32CB
:1012D00006E312500E2611500D2210500C220C3233
:1012E0000D320E32372EF1D70CBE07D00E360D362A
:1012F0000C360B5212E00B06303436AC17D016E326
:101300000E3E14D00D3E12D00C3E10D0D8800C32C0
:101310000D320E320B3E0AD003D036840B6A02D057
:1013200036820B680E6A0D6A800E0C6E39AE0C9E0A
:101330000E5012000CC039F07F0E0B5C376E3FE38D
:101340000C8E0B6A2E6A1708376E0BE2080E3726D2
:1013500038E30CC00BF00DC00CF00EC00DF00E6A9F
:101360000CD0080E375E08E30EC02EF00DC00EF054
:101370000CC00DF00C6AF5D73726375208E0D8902C
:101380000B320C320D320E322E32372EF8D70BBE06
:1013900018D036AC0BD02EAE09D00E3E07D00D3E85
:1013A00005D00C3E03D00C2A0BBE0BD039AE10D0AA
:1013B000D880000E0E560D560C560B5609D0000E56
:1013C00002D03682FF0E0B6E0C6E0D6E0E6E0B9EF3
:1013D0000E5012000B6E0C6A0D6A0E6A0B500EC096
:1013E0000BF00E6E0D500CC00DF00C6E960E376E9D
:1013F000396A0BAE07D0D880000E0E560D560C562B
:101400000B56398E0B5218E036AC0DD00EAE0BD009
:101410000D3E09D00C3E07D00B3E05D0D8800B32D4
:101420000C320D32372A080E37260DC00EF00CC0D4
:101430000DF00BC00CF015D00C6613D0080E375E03
:101440000D5005E1080E375E0E5011E00E6A0C6E6D
:101450000EC00DF00E6A05D0D8900E360D360C3643
:1014600037060CAEF9D737C00BF039AE0C9E0E50D4
:101470001200F86A400E366E006A330EAF6E200E10
:10148000AC6E900EAB6E0001070EB46E0F0EC16E07
:10149000CD0EC16E870EC06E1B0E926E020E936E45
:1014A000A70E946EF00E956E040E966E3FEF8AF0C6
:1014B000CF8E3E2A45843C0E3E5C0DE33F2A3E6AB9
:1014C0003C0E3F5C08E3402A3F6A180E405C03E391
:1014D000412A406A458203015053000102E00301A2
:1014E000500703015153000102E0030151070301BA
:1014F0007453000104E003017407000103D0010EDE
:101500000301756F00019E901100F29ED09ECD8662
:101510009E90CD9ACD98CD82CD80CD94CD9EF28CEB
:101520009D80F28E1200030E4214DB6FDB5302E14A
:10153000458001D0459012001D0E415C0FE145A091
:1015400006D0010E0301766F0001120006D0030ED3
:10155000446E010E0301DE6F416E00011E0E415C00
:1015600006E1030E446E010E0301DE6F416E0001C1
:1015700012001F0E415C05E1442A010E0301DE6FDB
:10158000416E00011200200E415C06E1030E446E24
:10159000010E0301DE6F416E000112001D0E415C61
:1015A00028E30301766B0001BEDF020E445C02E11A
:1015B000C3DF0FD0090E445C09E0040E445C06E072
:1015C000060E445C03E00B0E445C02E1D2DF01D066
:1015D000DADF010E0301765D00010BE00D0E445CC5
:1015E00007E1010E446E0301DE6F416E424A432A59
:1015F00000014592120003C10EF002C10DF001C1BD
:101600000CF000C10BF0EBC312F0EAC311F0E9C318
:1016100010F0E8C30FF04EEC08F00EC0E3F30DC07D
:10162000E2F30CC0E1F30BC0E0F3FFC00EF0FEC02C
:101630000DF0FDC00CF0FCC00BF0EFC312F0EEC3D8
:1016400011F0EDC310F0ECC30FF04EEC08F00EC03B
:10165000E7F30DC0E6F30CC0E5F30BC0E4F3DB6B7E
:10166000800E016E26EC00F0030EAA6E2F0EA96EFE
:10167000F5EC02F0480EF3EC02F080B605D0640EF3
:1016800018EC03F0DB2BF9D71F0EDB5D1BE3030126
:10169000E76BE66BE56BE46BE36BE26BE16BE06BD6
:1016A000800E016E26EC00F0030EAA6E3A0EA96EB3
:1016B000F5EC02F0480EF3EC02F0030E1C6EE80E9F
:1016C00019EC03F00001AA6A350EA96E0301E0517E
:1016D000E5EC02F0E151E5EC02F0E251E5EC02F05C
:1016E000E351E5EC02F0AA6A390EA96EE451E5EC8B
:1016F00002F0E551E5EC02F0E651E5EC02F0E751CD
:10170000E5EC02F0640E18EC03F000011200D8962C
:10171000010114A9D8860001D8B69AD003017A53E2
:10172000000107E0070E03017A5D000102E271D0BB
:1017300070D0070E03017A5D00010FE30A0E03016A
:101740007A5D00010AE22DC3AAFF2CC3A9FF0101A3
:101750001351E5EC02F000015CD00A0E03017A5D42
:10176000000118E30C0E03017A5D000113E22DC3A2
:10177000AAFF2CC3A9FF01015951E5EC02F05A510F
:10178000E5EC02F05B51E5EC02F05C51E5EC02F0B7
:1017900000013FD00C0E03017A5D00010FE3130E30
:1017A00003017A5D00010AE22DC3AAFF2CC3A9FF41
:1017B00001011351E5EC02F000012BD0130E0301DF
:1017C0007A5D000118E3190E03017A5D000113E24E
:1017D0002DC3AAFF2CC3A9FF01015951E5EC02F06A
:1017E0005A51E5EC02F05B51E5EC02F05C51E5EC9E
:1017F00002F000010ED01B0E03017A5D000108E12A
:101800002DC3AAFF2CC3A9FF01011351E5EC02F07F
:101810000001010E03017A5D000102E183C33EF085
:10182000020E03017A5D000102E183C33FF0010172
:101830001499800E016E26EC00F0AA0EF3EC02F073
:10184000480EF3EC02F0020E1C6E580E19EC03F079
:101850000001120003018531E832000105E30301B4
:10186000834B842B010114890001D896030185A5BF
:10187000D886000106E403018307000E845B0101A2
:1018800014890001800E016E26EC00F08FC3AAFFC0
:101890008EC3A9FFF5EC02F0056A84C320F083C370
:1018A0001FF07EEC00F0480EF3EC02F01200D2DFE5
:1018B0000301845304E1835100017E5D03E20301CF
:1018C000846B836B00011200D896010114B9D8868D
:1018D000000104E40301846B3EC083F303018F6BBA
:1018E0008C0E8E6F3B0E00017E6FE1DF1200D896EA
:1018F000010114B9D886000104E40301846B3FC0E0
:1019000083F303018F6B910E8E6F3B0E00017E6F90
:10191000CEDF1200D896010114B9D886000104E484
:101920000301846B40C083F303018F6B960E8E6FAF
:10193000170E00017E6FBBDF83C340F0120003016E
:10194000846B41C083F38F6B9C0E8E6F000182DF2E
:1019500083C341F012000301846B44C083F38F6B97
:10196000A10E8E6F000176DF83C344F0120043C0E6
:1019700084F342C083F303018F6BA60E8E6F0001C8
:1019800069DF84C343F083C342F01200090E0301F0
:101990007A5D000106E103018F6B8E692D6B020EEB
:1019A0002C6F00010C0E03017A5D000108E1010EAD
:1019B00003018F6F870E8E6F2D6B0B0E2C6F000146
:1019C0000D0E03017A5D000108E1010E03018F6F26
:1019D000920E8E6F2D6B0C0E2C6F00010E0E0301FC
:1019E0007A5D000108E1010E03018F6F9D0E8E6F7D
:1019F0002D6B0D0E2C6F00010F0E03017A5D00019F
:101A000008E1010E03018F6FA60E8E6F2D6B0E0E77
:101A10002C6F0001100E03017A5D000108E1020E37
:101A200003018F6F8D0E8E6F2D6B0F0E2C6F0001CB
:101A3000110E03017A5D000108E1020E03018F6FB0
:101A4000810E8E6F2D6B100E2C6F0001120E030194
:101A50007A5D000108E1020E03018F6FA60E8E6F02
:101A60002D6B110E2C6F00011B0E03017A5D00011E
:101A700008E1030E03018F6FB50E8E6F2D6B3F0EC5
:101A80002C6F0001D896010114B9D88600010CE42E
:101A90002DC3AAFF2CC3A9FFDEEC02F00101136FD6
:101AA0000301846B13C183F30001D4DE83C313F1FC
:101AB00012000A0E03017A5D000108E103012D6B9B
:101AC000030E2C6F010E8F6F710E8E6F00010B0EC7
:101AD00003017A5D000108E103012D6B070E2C6FF5
:101AE000010E8F6F7C0E8E6F0001130E03017A5D65
:101AF000000108E103012D6B120E2C6F020E8F6F97
:101B00009A0E8E6F0001140E03017A5D000107E149
:101B100003012D6B160E2C6F8F6B670E8E6F0001FD
:101B2000150E03017A5D000107E103012D6B1A0E0A
:101B30002C6F8F6B6F0E8E6F0001160E03017A5D96
:101B4000000107E103012D6B1E0E2C6F8F6B750ECC
:101B50008E6F0001170E03017A5D000107E103019A
:101B60002D6B220E2C6F8F6B7A0E8E6F0001180E6C
:101B700003017A5D000107E103012D6B260E2C6F36
:101B80008F6B830E8E6F0001D896010114B9D88631
:101B9000000111E42DC3AAFF2CC3A9FFDEEC02F063
:101BA0000101596FDEEC02F05A6FDEEC02F05B6F60
:101BB000DEEC02F05C6F03018531E832000135E3B1
:101BC0000E6A0D6A0C6A7F0E0B6E5CC112F05BC16F
:101BD00011F05AC110F059C10FF050EC08F00EC0CE
:101BE0005CF10DC05BF10CC05AF10BC059F180A63D
:101BF0001AD0A40E126E700E116E7D0E106E7E0E37
:101C00000F6E5CC10EF05BC10DF05AC10CF059C1F2
:101C10000BF04EEC08F00EC05CF10DC05BF10CC097
:101C20005AF10BC059F1010114890001D896030142
:101C300085A5D886000135E4126A116A106A7F0E04
:101C40000F6E5CC10EF05BC10DF05AC10CF059C1B2
:101C50000BF04EEC08F00EC05CF10DC05BF10CC057
:101C60005AF10BC059F180A61AD0A40E0E6E700E58
:101C70000D6E7D0E0C6E7E0E0B6E5CC112F05BC1A4
:101C800011F05AC110F059C10FF050EC08F00EC01D
:101C90005CF10DC05BF10CC05AF10BC059F10101B0
:101CA00014890001800E016E26EC00F08FC3AAFF9C
:101CB0008EC3A9FFF5EC02F05CC10EF05BC10DF024
:101CC0005AC10CF059C10BF0020EADEC00F0480EF9
:101CD000F3EC02F01200800E016E26EC00F08FC3D0
:101CE000AAFF8EC3A9FFF5EC02F0480EF3EC02F058
:101CF000C80E18EC03F003018531E83200010AE355
:101D00000301762B7651F15D000102E20301766B4F
:101D1000000112D0D896030185A5D88600010BE4F6
:101D200003017653000103E1F1C376F302D003010E
:101D30007607000101D012002DC3AAFF2CC3A9FF12
:101D400003017651E5EC02F0800E016E26EC00F006
:101D5000AA0EF3EC02F0480EF3EC02F0020E1C6E39
:101D6000580E19EC03F000011200030E0301F16F8D
:101D7000F2C376F37653000104E103018F6BC30EC7
:101D80008E6F0001010E0301765D000104E1030185
:101D90008F6BD20E8E6F0001020E0301765D000183
:101DA00004E103018F6BE10E8E6F0001030E03014E
:101DB000765D000104E103018F6BF00E8E6F03016D
:101DC0002D6B2C6B000187DF76C3F2F312000F0E30
:101DD0000301F16F72C376F37653000107E1010E40
:101DE00003018F6F060E8E6F000166D0010E030196
:101DF000765D000107E1010E03018F6F0E0E8E6FFD
:101E000000015AD0020E0301765D000107E1010EC8
:101E100003018F6F1A0E8E6F00014ED0030E030167
:101E2000765D000107E1010E03018F6F260E8E6FB4
:101E3000000142D0050E0301765D000107E1010EAD
:101E400003018F6F310E8E6F000136D0070E030134
:101E5000765D000107E1010E03018F6F3D0E8E6F6D
:101E600000012AD00A0E0301765D000107E1010E90
:101E700003018F6F480E8E6F00011ED00B0E030101
:101E8000765D000107E1010E03018F6F540E8E6F26
:101E9000000112D00F0E0301765D000107E1010E73
:101EA00003018F6F5F0E8E6F000105D0010E0301DD
:101EB0008F6F6A0E8E6F000103012D6B010E2C6F68
:101EC000000109DF76C372F31200030E0301F16F04
:101ED000AFC376F37653000105E1010E03018F6F66
:101EE000EF0E8E6F0001010E0301765D000105E12A
:101EF000010E03018F6FF90E8E6F0001020E0301B8
:101F0000765D000105E1020E03018F6F030E8E6FF7
:101F10000001030E0301765D000105E1020E0301DD
:101F20008F6F0D0E8E6F03012D6B2A0E2C6F00012B
:101F3000D2DE76C3AFF31200040E0301F16FB0C31B
:101F400076F37653000105E1020E03018F6F170E41
:101F50008E6F0001010E0301765D000105E1020EA6
:101F600003018F6F210E8E6F0001020E0301765D5B
:101F7000000105E1020E03018F6F2B0E8E6F000131
:101F8000030E0301765D000105E1020E03018F6F70
:101F9000350E8E6F0001040E0301765D000105E130
:101FA000020E03018F6F3F0E8E6F03012D6B2B0E00
:101FB0002C6F000190DE76C3B0F31200070E030110
:101FC000F16F08C476F37653000105E1030E0301B7
:101FD0008F6F5A0E8E6F0001010E0301765D0001B6
:101FE00005E1030E03018F6F660E8E6F0001020E76
:101FF0000301765D000105E1030E03018F6F6E0E94
:102000008E6F0001030E0301765D000105E1030EF2
:1020100003018F6F760E8E6F0001040E0301765D53
:10202000000105E1030E03018F6F7F0E8E6F00012B
:10203000050E0301765D000105E1030E03018F6FBC
:10204000880E8E6F0001060E0301765D000105E12A
:10205000030E03018F6F910E8E6F0001070E0301B7
:10206000765D000105E1030E03018F6F9A0E8E6FFE
:1020700003012D6B3D0E2C6F00012DDE76C308F49D
:102080001200AEC376F303017653000107E1010E9F
:1020900003018F6FE00E8E6F000105D0010E03016A
:1020A0008F6FE80E8E6F03012D6B2C0E2C6F0001CD
:1020B00012DE76C3AEF31200B9C376F30301765392
:1020C000000107E1020E03018F6F490E8E6F0001C0
:1020D00005D0020E03018F6F570E8E6F03012D6B1B
:1020E0002D0E2C6F00016BEC0EF076C3B9F31200CD
:1020F000BAC376F303017653000107E1020E030130
:102100008F6F650E8E6F000105D0020E03018F6F79
:10211000730E8E6F03012D6B2E0E2C6F00016BEC76
:102120000EF076C3BAF31200D5C376F303017653EB
:10213000000107E1020E03018F6FC30E8E6F0001D5
:1021400005D0020E03018F6FBC0E8E6F03012D6B45
:102150002F0E2C6F00016BEC0EF076C3D5F312003E
:10216000D6C376F303017653000107E1020E0301A3
:102170008F6FD30E8E6F000105D0020E03018F6F9B
:10218000CB0E8E6F03012D6B300E2C6F00016BECAC
:102190000EF076C3D6F31200D7C376F3030176535D
:1021A000000107E1020E03018F6FDF0E8E6F000149
:1021B00005D0020E03018F6FE70E8E6F03012D6BAA
:1021C000310E2C6F00016BEC0EF076C3D7F31200CA
:1021D000DCC376F303017653000107E1020E03012D
:1021E0008F6FFB0E8E6F000105D0020E03018F6F03
:1021F000F10E8E6F03012D6B320E2C6F00016BEC14
:102200000EF076C3DCF31200DDC376F303017653E0
:10221000000107E1030E03018F6F0C0E8E6F0001AA
:1022200005D0030E03018F6F020E8E6F03012D6B1D
:10223000330E2C6F00016BEC0EF076C3DDF3120051
:10224000DFC376F303017653000107E1030E0301B8
:102250008F6F170E8E6F000105D0030E03018F6F75
:10226000230E8E6F03012D6B340E2C6F00016BEC6F
:102270000EF076C3DFF31200F3C376F30301765357
:10228000000107E1030E03018F6FAC0E8E6F00019A
:1022900005D0030E03018F6FA40E8E6F03012D6B0B
:1022A0003E0E2C6F00016BEC0EF076C3F3F31200C0
:1022B000010E03017A6F0101149919EC00F0010E6F
:1022C0001C6EF40E19EC03F0800E016EC00E26ECAD
:1022D00000F0010EAA6EBA0EA96EF5EC02F0030131
:1022E000866B876B886B896B000182B44CD1830E3F
:1022F000036E800E066E286A2668FE0E276E010E9B
:10230000296E03018651BBEC02F0866F0001D8B044
:102310004ED1830E036E400E066E286A2668FE0EAE
:10232000276E010E296E03018751BBEC02F0876F07
:102330000001D8B042D1830E036E100E066E286ADB
:10234000640E266E1E0E276E010E296E0301885143
:10235000BBEC02F0886F0001D8B035D1830E036E5C
:10236000200E066E286A640E266E1E0E276E010E63
:10237000296E03018951BBEC02F0896F0001D8B0CE
:1023800026D1D896030185A7D886000102E403016F
:102390007A2B0001D896030185A9D886000102E4B2
:1023A00003017A0703017A53000103E1260E0301BA
:1023B0007A6F0001270E03017A5D000103E3010E2D
:1023C00003017A6F0001010E0301F16F010E7A5DC6
:1023D000000103E164EC0CF0CED0020E03017A5D43
:1023E000000103E177EC0CF0C6D0030E03017A5D27
:1023F000000103E18AEC0CF0BED0040E03017A5D0B
:10240000000103E19FEC0CF0B6D0050E03017A5DEC
:10241000000103E1ABEC0CF0AED0060E03017A5DD7
:10242000000103E1B7EC0CF0A6D0070E03017A5DC2
:10243000000103E1B5EC0EF09ED0080E03017A5DB9
:10244000000103E1E7EC0EF096D0090E03017A5D7E
:10245000000103E1C6EC0CF08ED00A0E03017A5D98
:10246000000108E30C0E03017A5D000103E259EC60
:102470000DF081D00C0E03017A5D000108E3130E0C
:1024800003017A5D000103E2C6EC0CF074D0130E78
:1024900003017A5D000108E3190E03017A5D000172
:1024A00003E259EC0DF067D0190E03017A5D0001CB
:1024B00003E165EC0FF05FD01A0E03017A5D0001B5
:1024C00003E19CEC0FF057D01B0E03017A5D000175
:1024D00003E1C6EC0CF04FD01C0E03017A5D000145
:1024E00003E141EC10F047D01D0E03017A5D0001BD
:1024F00003E15CEC10F03FD01E0E03017A5D000199
:1025000002E1F6DD38D01F0E03017A5D000102E121
:102510000BDE31D0200E03017A5D000102E120DEE6
:102520002AD0210E03017A5D000102E135DE23D0BD
:10253000220E03017A5D000102E14ADE1CD0230E67
:1025400003017A5D000102E15FDE15D0240E030174
:102550007A5D000102E174DE0ED0250E03017A5D82
:10256000000103E1DEEC0FF006D0260E03017A5DD8
:102570000001D8B481DE03018599859785938595FF
:102580000001B2D6B2D619EC00F0800E016E26EC36
:1025900000F0010EAA6EAF0EA96EF5EC02F0030E6C
:1025A0001C6EE80E19EC03F019EC00F012000301A8
:1025B0008589000187EC0BF0E4D6030185870001D3
:1025C00087EC0BF0DED6030185830001DAD6030128
:1025D00085850001D6D69A0E0201B36F920EB26FB6
:1025E0005A0EB16F830EB06F3C0EB76FA10EB66F6F
:1025F000360EB56F870EB46FB80EBB6F6F0EBA6F25
:102600005C0EB96F830EB86FA50EBF6F3E0EBE6F26
:102610006C0EBD6F830EBC6FA10EC36FB20EC26F86
:10262000590EC16F830EC06FE80EC76F720EC66F72
:10263000540EC56F8B0EC46F70C10EF06FC10DF0DC
:102640006EC10CF06DC10BF0B3C212F0B2C211F04A
:10265000B1C210F0B0C20FF0E2EC08F00EC0B3F25D
:102660000DC0B2F20CC0B1F20BC0B0F270C10EF0EE
:102670006FC10DF06EC10CF06DC10BF0B7C212F05E
:10268000B6C211F0B5C210F0B4C20FF0E2EC08F01F
:102690000EC0B7F20DC0B6F20CC0B5F20BC0B4F26A
:1026A00070C10EF06FC10DF06EC10CF06DC10BF07A
:1026B000BBC212F0BAC211F0B9C210F0B8C20FF02A
:1026C000E2EC08F00EC0BBF20DC0BAF20CC0B9F2D9
:1026D0000BC0B8F270C10EF06FC10DF06EC10CF0FE
:1026E0006DC10BF0BFC212F0BEC211F0BDC210F03E
:1026F000BCC20FF0E2EC08F00EC0BFF20DC0BEF29B
:102700000CC0BDF20BC0BCF270C10EF06FC10DF079
:102710006EC10CF06DC10BF0C3C212F0C2C211F059
:10272000C1C210F0C0C20FF0E2EC08F00EC0C3F25C
:102730000DC0C2F20CC0C1F20BC0C0F270C10EF0ED
:102740006FC10DF06EC10CF06DC10BF0C7C212F07D
:10275000C6C211F0C5C210F0C4C20FF0E2EC08F01E
:102760000EC0C7F20DC0C6F20CC0C5F20BC0C4F259
:10277000366AB3C20EF0B2C20DF0B1C20CF0B0C2F4
:102780000BF09AEC09F00BC058F10CC057F10DC0DA
:1027900056F10101556F58C10EF057C10DF056C1E9
:1027A0000CF055C10BF0EEEC09F00EC012F00DC0AC
:1027B00011F00CC010F00BC00FF0B3C20EF0B2C29B
:1027C0000DF0B1C20CF0B0C20BF04EEC08F00EC030
:1027D000B3F20DC0B2F20CC0B1F20BC0B0F20E6A8F
:1027E0000D6A340E0C6E870E0B6EB3C212F0B2C2BD
:1027F00011F0B1C210F0B0C20FF04AEC09F00EC0F7
:10280000B3F20DC0B2F20CC0B1F20BC0B0F2B7C25D
:102810000EF0B6C20DF0B5C20CF0B4C20BF09AECDB
:1028200009F00BC058F10CC057F10DC056F1556FAF
:1028300058C10EF057C10DF056C10CF055C10BF048
:10284000EEEC09F00EC012F00DC011F00CC010F04B
:102850000BC00FF0B7C20EF0B6C20DF0B5C20CF04F
:10286000B4C20BF04EEC08F00EC0B7F20DC0B6F2D9
:102870000CC0B5F20BC0B4F20E6A0D6A340E0C6EC9
:10288000870E0B6EB7C212F0B6C211F0B5C210F0CF
:10289000B4C20FF04AEC09F00EC0B7F20DC0B6F2A8
:1028A0000CC0B5F20BC0B4F2BBC20EF0BAC20DF050
:1028B000B9C20CF0B8C20BF09AEC09F00BC058F199
:1028C0000CC057F10DC056F1556F58C10EF057C1ED
:1028D0000DF056C10CF055C10BF0EEEC09F00EC036
:1028E00012F00DC011F00CC010F00BC00FF0BBC205
:1028F0000EF0BAC20DF0B9C20CF0B8C20BF04EEC3B
:1029000008F00EC0BBF20DC0BAF20CC0B9F20BC099
:10291000B8F20E6A0D6A340E0C6E870E0B6EBBC2D7
:1029200012F0BAC211F0B9C210F0B8C20FF04AECFE
:1029300009F00EC0BBF20DC0BAF20CC0B9F20BC068
:10294000B8F2BFC20EF0BEC20DF0BDC20CF0BCC2E8
:102950000BF09AEC09F00BC058F10CC057F10DC008
:1029600056F1556F58C10EF057C10DF056C10CF01D
:1029700055C10BF0EEEC09F00EC012F00DC011F0D5
:102980000CC010F00BC00FF0BFC20EF0BEC20DF0B5
:10299000BDC20CF0BCC20BF04EEC08F00EC0BFF292
:1029A0000DC0BEF20CC0BDF20BC0BCF20E6A0D6AC7
:1029B000340E0C6E870E0B6EBFC212F0BEC211F049
:1029C000BDC210F0BCC20FF04AEC09F00EC0BFF25D
:1029D0000DC0BEF20CC0BDF20BC0BCF2C3C20EF003
:1029E000C2C20DF0C1C20CF0C0C20BF09AEC09F0EB
:1029F0000BC058F10CC057F10DC056F1556F58C1BE
:102A00000EF057C10DF056C10CF055C10BF0EEECB5
:102A100009F00EC012F00DC011F00CC010F00BC088
:102A20000FF0C3C20EF0C2C20DF0C1C20CF0C0C2A2
:102A30000BF04EEC08F00EC0C3F20DC0C2F20CC099
:102A4000C1F20BC0C0F20E6A0D6A340E0C6E870E16
:102A50000B6EC3C212F0C2C211F0C1C210F0C0C2EC
:102A60000FF04AEC09F00EC0C3F20DC0C2F20CC068
:102A7000C1F20BC0C0F2C7C20EF0C6C20DF0C5C293
:102A80000CF0C4C20BF09AEC09F00BC058F10CC06A
:102A900057F10DC056F1556F58C10EF057C10DF0EA
:102AA00056C10CF055C10BF0EEEC09F00EC012F05F
:102AB0000DC011F00CC010F00BC00FF0C7C20EF02B
:102AC000C6C20DF0C5C20CF0C4C20BF04EEC08F04B
:102AD0000EC0C7F20DC0C6F20CC0C5F20BC0C4F2E6
:102AE0000E6A0D6A340E0C6E870E0B6EC7C212F0A2
:102AF000C6C211F0C5C210F0C4C20FF04AEC09F012
:102B00000EC0C7F20DC0C6F20CC0C5F20BC0C4F2B5
:102B1000400E366E810E0E6E030E0D6E7F0E0C6E25
:102B20006B0E0B6E7CC112F07BC111F07AC110F0FC
:102B300079C10FF04AEC09F00EC075F00DC074F0C9
:102B40000CC073F00BC072F02C0E0E6E810E0D6E69
:102B5000140E0C6E750E0B6E75C012F074C011F071
:102B600073C010F072C00FF04EEC08F00EC075F09C
:102B70000DC074F00CC073F00BC072F075C00EF095
:102B800074C00DF073C00CF072C00BF06DC012F089
:102B90006CC011F06BC010F06AC00FF04AEC09F085
:102BA0000EC075F00DC074F00CC073F00BC072F065
:102BB000930E0E6E370E0D6E070E0C6E870E0B6E9B
:102BC000B3C212F0B2C211F0B1C210F0B0C20FF035
:102BD00050EC08F00EC079F00DC078F00CC077F022
:102BE0000BC076F079C00EF078C00DF077C00CF015
:102BF00076C00BF075C012F074C011F073C010F005
:102C000072C00FF04EEC08F00EC087F20DC086F2D5
:102C10000CC085F20BC084F2910E0E6E750E0D6E17
:102C20005D0E0C6E6C0E0B6E7CC112F07BC111F050
:102C30007AC110F079C10FF04AEC09F00EC075F0BE
:102C40000DC074F00CC073F00BC072F0520E0E6E1B
:102C5000490E0D6E1D0E0C6E720E0B6E75C012F0CD
:102C600074C011F073C010F072C00FF050EC08F097
:102C70000EC075F00DC074F00CC073F00BC072F094
:102C800075C00EF074C00DF073C00CF072C00BF084
:102C90006DC012F06CC011F06BC010F06AC00FF084
:102CA0004AEC09F00EC075F00DC074F00CC073F062
:102CB0000BC072F0E80E0E6E3C0E0D6E330E0C6EF5
:102CC000870E0B6EB7C212F0B6C211F0B5C210F08B
:102CD000B4C20FF050EC08F00EC079F00DC078F0DF
:102CE0000CC077F00BC076F079C00EF078C00DF014
:102CF00077C00CF076C00BF075C012F074C011F004
:102D000073C010F072C00FF04EEC08F00EC023F24A
:102D10000DC022F20CC021F20BC020F2870E0E6E05
:102D2000970E0D6E710E0C6E6E0E0B6E7CC112F056
:102D30007BC111F07AC110F079C10FF04AEC09F0B3
:102D40000EC075F00DC074F00CC073F00BC072F0C3
:102D50000B0E0E6E9A0E0D6E160E0C6E780E0B6E1E
:102D600075C012F074C011F073C010F072C00FF093
:102D700050EC08F00EC075F00DC074F00CC073F08C
:102D80000BC072F075C00EF074C00DF073C00CF083
:102D900072C00BF06DC012F06CC011F06BC010F07F
:102DA0006AC00FF04AEC09F00EC075F00DC074F067
:102DB0000CC073F00BC072F0640E0E6E0D0E0D6E33
:102DC000140E0C6E870E0B6EBBC212F0BAC211F05D
:102DD000B9C210F0B8C20FF050EC08F00EC079F094
:102DE0000DC078F00CC077F00BC076F079C00EF013
:102DF00078C00DF077C00CF076C00BF075C012F003
:102E000074C011F073C010F072C00FF050EC08F0F5
:102E10000EC08BF20DC08AF20CC089F20BC088F292
:102E2000810E0E6E030E0D6E7F0E0C6E6B0E0B6E12
:102E30007CC112F07BC111F07AC110F079C10FF0A2
:102E40004AEC09F00EC075F00DC074F00CC073F0C0
:102E50000BC072F02A0E0E6E380E0D6E3C0E0C6E0C
:102E6000750E0B6E75C012F074C011F073C010F0C7
:102E700072C00FF04EEC08F00EC075F00DC074F08B
:102E80000CC073F00BC072F075C00EF074C00DF082
:102E900073C00CF072C00BF06DC012F06CC011F07A
:102EA0006BC010F06AC00FF04AEC09F00EC075F06C
:102EB0000DC074F00CC073F00BC072F0660E0E6E95
:102EC0005E0E0D6E2F0E0C6E870E0B6EBFC212F0D3
:102ED000BEC211F0BDC210F0BCC20FF050EC08F041
:102EE0000EC079F00DC078F00CC077F00BC076F012
:102EF00079C00EF078C00DF077C00CF076C00BF002
:102F000075C012F074C011F073C010F072C00FF0F1
:102F10004EEC08F00EC0CBF20DC0CAF20CC0C9F2E4
:102F20000BC0C8F2B00E0E6E0F0E0D6E210E0C6EA1
:102F3000690E0B6E7CC112F07BC111F07AC110F0EA
:102F400079C10FF04AEC09F00EC075F00DC074F0B5
:102F50000CC073F00BC072F0A40E0E6E6F0E0D6EEF
:102F6000520E0C6E760E0B6E75C012F074C011F01E
:102F700073C010F072C00FF050EC08F00EC075F086
:102F80000DC074F00CC073F00BC072F075C00EF081
:102F900074C00DF073C00CF072C00BF06DC012F075
:102FA0006CC011F06BC010F06AC00FF04AEC09F071
:102FB0000EC075F00DC074F00CC073F00BC072F051
:102FC000A40E0E6E030E0D6E340E0C6E820E0B6E82
:102FD000C3C212F0C2C211F0C1C210F0C0C20FF0E1
:102FE00050EC08F00EC079F00DC078F00CC077F00E
:102FF0000BC076F079C00EF078C00DF077C00CF001
:1030000076C00BF075C012F074C011F073C010F0F0
:1030100072C00FF04EEC08F00EC0CFF20DC0CEF231
:103020000CC0CDF20BC0CCF2A40E0E6E8C0E0D6E49
:10303000380E0C6E6F0E0B6E7CC112F07BC111F05E
:103040007AC110F079C10FF04AEC09F00EC075F0AA
:103050000DC074F00CC073F00BC072F00E0E0E6E4B
:103060002F0E0D6E080E0C6E760E0B6E75C012F0E4
:1030700074C011F073C010F072C00FF050EC08F083
:103080000EC075F00DC074F00CC073F00BC072F080
:1030900075C00EF074C00DF073C00CF072C00BF070
:1030A0006DC012F06CC011F06BC010F06AC00FF070
:1030B0004AEC09F00EC075F00DC074F00CC073F04E
:1030C0000BC072F0760E0E6E970E0D6E010E0C6E2A
:1030D000870E0B6EC7C212F0C6C211F0C5C210F047
:1030E000C4C20FF04EEC08F00EC079F00DC078F0BD
:1030F0000CC077F00BC076F079C00EF078C00DF000
:1031000077C00CF076C00BF075C012F074C011F0EF
:1031100073C010F072C00FF050EC08F00EC0D3F284
:103120000DC0D2F20CC0D1F20BC0D0F29A0E0E6ECE
:10313000990E0D6E210E0C6E830E0B6E7CC112F07B
:103140007BC111F07AC110F079C10FF04AEC09F09F
:103150000EC075F00DC074F00CC073F00BC072F0AF
:10316000CD0E0E6ECC0E0D6E4C0E0C6E840E0B6ED4
:1031700075C012F074C011F073C010F072C00FF07F
:1031800050EC08F00EC075F00DC074F00CC073F078
:103190000BC072F0340E0E6EFA0E0D6E0E0E0C6E2B
:1031A000790E0B6E75C012F074C011F073C010F080
:1031B00072C00FF04AEC09F084EC05F00EC0D7F2B3
:1031C0000DC0D6F20CC0D5F20BC0D4F2340E0E6E88
:1031D000FA0E0D6E0E0E0C6E790E0B6ED3C212F03F
:1031E000D2C211F0D1C210F0D0C20FF04AEC09F0F7
:1031F00084EC05F00EC088F10DC087F10CC086F19B
:103200000BC085F1C50E0E6E4A0E0D6E160E0C6EBD
:10321000780E0B6E7CC112F07BC111F07AC110F0F8
:1032200079C10FF04AEC09F00EC075F00DC074F0D2
:103230000CC073F00BC072F0B80E0E6EDE0E0D6E89
:10324000040E0C6E860E0B6E75C012F074C011F079
:1032500073C010F072C00FF04EEC08F00EC075F0A5
:103260000DC074F00CC073F00BC072F075C00EF09E
:1032700074C00DF073C00CF072C00BF07CC112F082
:103280007BC111F07AC110F079C10FF04AEC09F05E
:103290000EC075F00DC074F00CC073F00BC072F06E
:1032A000AE0E0E6E470E0D6E2D0E0C6E870E0B6E53
:1032B00075C012F074C011F073C010F072C00FF03E
:1032C00050EC08F00EC047F10DC046F10CC045F1BE
:1032D0000BC044F1340E0E6EFA0E0D6E0E0E0C6E17
:1032E000790E0B6E47C112F046C111F045C110F0C6
:1032F00044C10FF04AEC09F084EC05F00EC075F003
:103300000DC074F00CC073F00BC072F0710E0E6E35
:10331000E40E0D6E010E0C6E770E0B6E75C012F082
:1033200074C011F073C010F072C00FF04AEC09F0D5
:103330000EC0DBF20DC0DAF20CC0D9F20BC0D8F22D
:10334000330E0E6E0D6E130E0C6E800E0B6E7CC166
:1033500012F07BC111F07AC110F079C10FF04AEC84
:1033600009F00EC075F00DC074F00CC073F00BC006
:1033700072F0660E0E6E860E0D6E090E0C6E870EC6
:103380000B6ED3C212F0D2C211F0D1C210F0D0C273
:103390000FF050EC08F00EC02DF00DC02CF00CC05A
:1033A0002BF00BC02AF02DC00EF02CC00DF02BC05E
:1033B0000CF02AC00BF075C012F074C011F073C08D
:1033C00010F072C00FF04EEC08F00EC075F00DC09A
:1033D00074F00CC073F00BC072F0340E0E6EFA0E67
:1033E0000D6E0E0E0C6E790E0B6E75C012F074C061
:1033F00011F073C010F072C00FF04AEC09F00EC06B
:103400004BF10DC04AF10CC049F10BC048F14BC162
:103410000EF04AC10DF049C10CF048C10BF084EC2C
:1034200005F00EC0DFF20DC0DEF20CC0DDF20BC005
:10343000DCF2760E0E6E510E0D6E740E0C6E720E68
:103440000B6ED7C212F0D6C211F0D5C210F0D4C2A2
:103450000FF04AEC09F00EC075F00DC074F00CC00E
:1034600073F00BC072F0740E0E6EB60E0D6E0C6A19
:10347000760E0B6E88C112F087C111F086C110F074
:1034800085C10FF04AEC09F00EC079F00DC078F05C
:103490000CC077F00BC076F087C20EF086C20DF03C
:1034A00085C20CF084C20BF075C012F074C011F02C
:1034B00073C010F072C00FF050EC08F00EC02DF089
:1034C0000DC02CF00CC02BF00BC02AF02DC00EF05C
:1034D0002CC00DF02BC00CF02AC00BF0DBC212F098
:1034E000DAC211F0D9C210F0D8C20FF050EC08F0D7
:1034F0000EC075F00DC074F00CC073F00BC072F00C
:1035000075C00EF074C00DF073C00CF072C00BF0FB
:1035100079C012F078C011F077C010F076C00FF0CB
:1035200050EC08F00EC087F20DC086F20CC085F298
:103530000BC084F2E40E0E6E4E0E0D6E690E0C6E14
:10354000750E0B6ED7C212F0D6C211F0D5C210F0B4
:10355000D4C20FF04AEC09F00EC075F00DC074F043
:103560000CC073F00BC072F023C20EF022C20DF03B
:1035700021C20CF020C20BF075C012F074C011F023
:1035800073C010F072C00FF04EEC08F00EC023F2C2
:103590000DC022F20CC021F20BC020F2E80E0E6E1C
:1035A000860E0D6E260E0C6E760E0B6E88C112F016
:1035B00087C111F086C110F085C10FF04AEC09F007
:1035C0000EC075F00DC074F00CC073F00BC072F03B
:1035D000F10E0E6E2B0E0D6E560E0C6E740E0B6EE3
:1035E000D7C212F0D6C211F0D5C210F0D4C20FF07B
:1035F0004AEC09F00EC079F00DC078F00CC077F0FD
:103600000BC076F0DBC20EF0DAC20DF0D9C20CF0BE
:10361000D8C20BF075C012F074C011F073C010F076
:1036200072C00FF050EC08F00EC075F00DC074F0D1
:103630000CC073F00BC072F075C00EF074C00DF0CA
:1036400073C00CF072C00BF079C012F078C011F0AA
:1036500077C010F076C00FF050EC08F00EC075F097
:103660000DC074F00CC073F00BC072F08BC20EF082
:103670008AC20DF089C20CF088C20BF075C012F03E
:1036800074C011F073C010F072C00FF050EC08F06D
:103690000EC08BF20DC08AF20CC089F20BC088F20A
:1036A000E50E0E6ED10E0D6E0D0E0C6E770E0B6EBE
:1036B000DFC212F0DEC211F0DDC210F0DCC20FF08A
:1036C0004AEC09F00EC075F00DC074F00CC073F038
:1036D0000BC072F0C80E0E6E440E0D6E4A0E0C6ECC
:1036E000790E0B6E88C112F087C111F086C110F0FF
:1036F00085C10FF04AEC09F00EC079F00DC078F0EA
:103700000CC077F00BC076F0CFC20EF0CEC20DF039
:10371000CDC20CF0CCC20BF0DBC212F0DAC211F059
:10372000D9C210F0D8C20FF050EC08F00EC07DF0F6
:103730000DC07CF00CC07BF00BC07AF07DC00EF0A9
:103740007CC00DF07BC00CF07AC00BF079C012F099
:1037500078C011F077C010F076C00FF04EEC08F092
:103760000EC07DF00DC07CF00CC07BF00BC07AF079
:103770007DC00EF07CC00DF07BC00CF07AC00BF069
:1037800075C012F074C011F073C010F072C00FF069
:103790004EEC08F00EC0CFF20DC0CEF20CC0CDF250
:1037A0000BC0CCF2740E0E6EB60E0D6E0C6A760E59
:1037B0000B6E88C112F087C111F086C110F085C16F
:1037C0000FF04AEC09F00EC075F00DC074F00CC09B
:1037D00073F00BC072F0FB0E0E6ECA0E0D6E030E70
:1037E0000C6E760E0B6ED7C212F0D6C211F0D5C297
:1037F00010F0D4C20FF04AEC09F00EC079F00DC001
:1038000078F00CC077F00BC076F0CBC20EF0CAC2D5
:103810000DF0C9C20CF0C8C20BF079C012F078C02C
:1038200011F077C010F076C00FF050EC08F00EC029
:103830007DF00DC07CF00CC07BF00BC07AF07DC039
:103840000EF07CC00DF07BC00CF07AC00BF0DBC238
:1038500012F0DAC211F0D9C210F0D8C20FF050EC59
:1038600008F00EC07DF00DC07CF00CC07BF00BC0EA
:103870007AF07DC00EF07CC00DF07BC00CF07AC0F9
:103880000BF075C012F074C011F073C010F072C06C
:103890000FF050EC08F00EC0CBF20DC0CAF20CC015
:1038A000C9F20BC0C8F24F0E0E6E540E0D6E7C0E98
:1038B0000C6E6D0E0B6E7CC112F07BC111F07AC1E3
:1038C00010F079C10FF04AEC09F00EC075F00DC090
:1038D00074F00CC073F00BC072F0270E0E6E830EE6
:1038E0000D6E230E0C6E760E0B6E75C012F074C04A
:1038F00011F073C010F072C00FF050EC08F00EC061
:1039000075F00DC074F00CC073F00BC072F075C090
:103910000EF074C00DF073C00CF072C00BF07CC1DF
:1039200012F07BC111F07AC110F079C10FF04AECAE
:1039300009F00EC075F00DC074F00CC073F00BC030
:1039400072F00E6A0D6A0C6A7F0E0B6E75C012F073
:1039500074C011F073C010F072C00FF04EEC08F09C
:103960000EC0E3F20DC0E2F20CC0E1F20BC0E0F2D7
:10397000E3C20EF0E2C20DF0E1C20CF0E0C20BF0C7
:10398000E3C212F0E2C211F0E1C210F0E0C20FF0A7
:103990004AEC09F00EC0E7F20DC0E6F20CC0E5F209
:1039A0000BC0E4F2340E0E6EFA0E0D6E0E0E0C6E9F
:1039B000790E0B6E87C212F086C211F085C210F02C
:1039C00084C20FF04AEC09F00EC087F20DC086F2F7
:1039D0000CC085F20BC084F2340E0E6EFA0E0D6E22
:1039E0000E0E0C6E790E0B6E23C212F022C211F075
:1039F00021C210F020C20FF04AEC09F00EC023F2F1
:103A00000DC022F20CC021F20BC020F2340E0E6E5B
:103A1000FA0E0D6E0E0E0C6E790E0B6ED3C212F0F6
:103A2000D2C211F0D1C210F0D0C20FF04AEC09F0AE
:103A30000EC0D3F20DC0D2F20CC0D1F20BC0D0F246
:103A4000340E0E6EFA0E0D6E0E0E0C6E790E0B6E9F
:103A5000CBC212F0CAC211F0C9C210F0C8C20FF036
:103A60004AEC09F00EC0CBF20DC0CAF20CC0C9F28C
:103A70000BC0C8F2340E0E6EFA0E0D6E0E0E0C6EEA
:103A8000790E0B6ECFC212F0CEC211F0CDC210F083
:103A9000CCC20FF04AEC09F00EC0CFF20DC0CEF24E
:103AA0000CC0CDF20BC0CCF2340E0E6EFA0E0D6EC1
:103AB0000E0E0C6E790E0B6E8BC212F08AC211F0D4
:103AC00089C210F088C20FF04AEC09F00EC08BF2E8
:103AD0000DC08AF20CC089F20BC088F2CBC2EBF2A7
:103AE000CAC2EAF2C9C2E9F20201C83D02D0368276
:103AF000C851E86FCBC2F3F2CAC2F2F2C9C2F1F206
:103B0000020EC82502E33682FF0EF06F8BC2FFF271
:103B10008AC2FEF289C2FDF2883D02D03682885107
:103B2000FC6F23C213F322C212F321C211F3203D12
:103B300002D0368220510301106F0E6A0D6A400ECA
:103B40000C6E800E0B6E8BC212F08AC211F089C20D
:103B500010F088C20FF04AEC09F00EC0F7F20DC069
:103B6000F6F20CC0F5F20BC0F4F2CFC207F3CEC2EE
:103B700006F3CDC205F30201CC3D02D03682CC5112
:103B80000301046F0E6A0D6A400E0C6E800E0B6E00
:103B9000CFC212F0CEC211F0CDC210F0CCC20FF0E5
:103BA0004AEC09F00EC00BF30DC00AF30CC009F388
:103BB0000BC008F30E6A0D6A400E0C6E800E0B6E81
:103BC000CBC212F0CAC211F0C9C210F0C8C20FF0C5
:103BD0004AEC09F00EC0EFF20DC0EEF20CC0EDF2AF
:103BE0000BC0ECF28BC203F38AC202F389C201F369
:103BF000020E0201882502E33682FF0E0301006FE8
:103C0000EBC20EF0EAC20DF0E9C20CF0E8C20BF014
:103C10008BC212F08AC211F089C210F088C20FF074
:103C20004EEC08F084EC05F00EC075F00DC074F099
:103C30000CC073F00BC072F0060E0E6E130E0D6EFC
:103C4000230E0C6E7F0E0B6E75C012F074C011F057
:103C500073C010F072C00FF04AEC09F00EC075F09E
:103C60000DC074F00CC073F00BC072F08BC20EF07C
:103C70008AC20DF089C20CF088C20BF084EC05F00A
:103C80000EC02DF00DC02CF00CC02BF00BC02AF094
:103C9000710E0E6E3D0E0D6E490E0C6E810E0B6E8A
:103CA0002DC012F02CC011F02BC010F02AC00FF064
:103CB0004AEC09F00EC079F00DC078F00CC077F036
:103CC0000BC076F079C00EF078C00DF077C00CF024
:103CD00076C00BF075C012F074C011F073C010F014
:103CE00072C00FF050EC08F00EC0FBF20DC0FAF2FB
:103CF0000CC0F9F20BC0F8F2EBC20EF0EAC20DF004
:103D0000E9C20CF0E8C20BF084EC05F00EC02DF017
:103D10000DC02CF00CC02BF00BC02AF0F00E0E6E74
:103D2000860E0D6E280E0C6E7E0E0B6E2DC012F0E0
:103D30002CC011F02BC010F02AC00FF04AEC09F093
:103D40000EC075F00DC074F00CC073F00BC072F0B3
:103D5000FBC20EF0FAC20DF0F9C20CF0F8C20BF083
:103D600075C012F074C011F073C010F072C00FF083
:103D700050EC08F00EC0FBF20DC0FAF20CC0F9F2E4
:103D80000BC0F8F2FFC20EF0FEC20DF0FDC20CF047
:103D9000FCC20BF084EC05F00EC075F00DC074F0A1
:103DA0000CC073F00BC072F0270E0E6EBE0E0D6EBF
:103DB0005A0E0C6E7C0E0B6E75C012F074C011F0B2
:103DC00073C010F072C00FF04AEC09F00EC075F02D
:103DD0000DC074F00CC073F00BC072F0FBC20EF09B
:103DE000FAC20DF0F9C20CF0F8C20BF075C012F077
:103DF00074C011F073C010F072C00FF050EC08F0F6
:103E00000EC0FBF20DC0FAF20CC0F9F20BC0F8F2D2
:103E100023C20EF022C20DF021C20CF020C20BF022
:103E200084EC05F00EC02DF00DC02CF00CC02BF072
:103E30000BC02AF0E10E0E6E0C0E0D6E3E0E0C6ED7
:103E40007C0E0B6E2DC012F02CC011F02BC010F0A8
:103E50002AC00FF04AEC09F00EC075F00DC074F0E6
:103E60000CC073F00BC072F0E3C20EF0E2C20DF0B2
:103E7000E1C20CF0E0C20BF075C012F074C011F09A
:103E800073C010F072C00FF04AEC09F00EC02DF0B4
:103E90000DC02CF00CC02BF00BC02AF0FBC20EF0B2
:103EA000FAC20DF0F9C20CF0F8C20BF02DC012F0FE
:103EB0002CC011F02BC010F02AC00FF04EEC08F00F
:103EC0000EC0FBF20DC0FAF20CC0F9F20BC0F8F212
:103ED00007C30EF006C30DF005C30CF004C30BF0CE
:103EE00084EC05F00EC075F00DC074F00CC073F0DA
:103EF0000BC072F0FE0E0E6E280E0D6E6A0E0C6E6A
:103F00007B0E0B6E75C012F074C011F073C010F010
:103F100072C00FF04AEC09F00EC075F00DC074F0DD
:103F20000CC073F00BC072F0FBC20EF0FAC20DF0C1
:103F3000F9C20CF0F8C20BF075C012F074C011F0A9
:103F400073C010F072C00FF04EEC08F00EC0FBF220
:103F50000DC0FAF20CC0F9F20BC0F8F2CBC20EF0B1
:103F6000CAC20DF0C9C20CF0C8C20BF08BC212F06D
:103F70008AC211F089C210F088C20FF04EEC08F02E
:103F80000EC075F00DC074F00CC073F00BC072F071
:103F900075C00EF074C00DF073C00CF00001723DDE
:103FA00002D0368272510B6E84EC05F00EC075F0B3
:103FB0000DC074F00CC073F00BC072F0EE0E0E6EFC
:103FC000D00E0D6E700E0C6E7A0E0B6E75C012F068
:103FD00074C011F073C010F072C00FF04AEC09F019
:103FE0000EC075F00DC074F00CC073F00BC072F011
:103FF000FBC20EF0FAC20DF0F9C20CF0F8C20BF0E1
:1040000075C012F074C011F073C010F072C00FF0E0
:1040100050EC08F00EC0FBF20DC0FAF20CC0F9F241
:104020000BC0F8F2EBC20EF0EAC20DF0E9C20CF0E0
:10403000E8C20BF023C212F022C211F021C210F02C
:1040400020C20FF04EEC08F00EC02DF00DC02CF089
:104050000CC02BF00BC02AF02DC00EF02CC00DF0C0
:104060002BC00CF02AC00BF08BC212F08AC211F0E8
:1040700089C210F088C20FF04EEC08F084EC05F015
:104080000EC075F00DC074F00CC073F00BC072F070
:10409000E3C20EF0E2C20DF0E1C20CF0E0C20BF0A0
:1040A00075C012F074C011F073C010F072C00FF040
:1040B0004AEC09F00EC075F00DC074F00CC073F03E
:1040C0000BC072F0210E0E6E570E0D6E6A0E0C6E46
:1040D0007A0E0B6E75C012F074C011F073C010F040
:1040E00072C00FF04AEC09F00EC075F00DC074F00C
:1040F0000CC073F00BC072F0FBC20EF0FAC20DF0F0
:10410000F9C20CF0F8C20BF075C012F074C011F0D7
:1041100073C010F072C00FF050EC08F00EC0FBF24C
:104120000DC0FAF20CC0F9F20BC0F8F2EBC20EF0BF
:10413000EAC20DF0E9C20CF0E8C20BF08BC212F03B
:104140008AC211F089C210F088C20FF050EC08F05A
:1041500084EC05F00EC075F00DC074F00CC073F067
:104160000BC072F0130E0E6E660E0D6E5A0E0C6EB4
:104170007A0E0B6E75C012F074C011F073C010F09F
:1041800072C00FF04AEC09F00EC075F00DC074F06B
:104190000CC073F00BC072F0FBC20EF0FAC20DF04F
:1041A000F9C20CF0F8C20BF075C012F074C011F037
:1041B00073C010F072C00FF050EC08F00EC0FBF2AC
:1041C0000DC0FAF20CC0F9F20BC0F8F2EBC20EF01F
:1041D000EAC20DF0E9C20CF0E8C20BF023C212F003
:1041E00022C211F021C210F020C20FF04EEC08F0F4
:1041F00084EC05F00EC075F00DC074F00CC073F0C7
:104200000BC072F0600E0E6EE60E0D6E3B0E0C6E65
:104210007A0E0B6EE3C212F0E2C211F0E1C210F0AE
:10422000E0C20FF04AEC09F00EC02DF00DC02CF0EA
:104230000CC02BF00BC02AF02DC00EF02CC00DF0DE
:104240002BC00CF02AC00BF075C012F074C011F036
:1042500073C010F072C00FF04AEC09F00EC075F098
:104260000DC074F00CC073F00BC072F0FBC20EF006
:10427000FAC20DF0F9C20CF0F8C20BF075C012F0E2
:1042800074C011F073C010F072C00FF050EC08F061
:104290000EC0FBF20DC0FAF20CC0F9F20BC0F8F23E
:1042A0008BC20EF08AC20DF089C20CF088C20BF0EE
:1042B00023C212F022C211F021C210F020C20FF06E
:1042C0004EEC08F084EC05F00EC075F00DC074F0F3
:1042D0000CC073F00BC072F0C80E0E6E080E0D6E9F
:1042E000280E0C6E7A0E0B6EE3C212F0E2C211F0D1
:1042F000E1C210F0E0C20FF04AEC09F00EC02DF060
:104300000DC02CF00CC02BF00BC02AF02DC00EF00D
:104310002CC00DF02BC00CF02AC00BF075C012F0B1
:1043200074C011F073C010F072C00FF04AEC09F0C5
:104330000EC075F00DC074F00CC073F00BC072F0BD
:10434000FBC20EF0FAC20DF0F9C20CF0F8C20BF08D
:1043500075C012F074C011F073C010F072C00FF08D
:1043600050EC08F00EC0FBF20DC0FAF20CC0F9F2EE
:104370000BC0F8F2CBC20EF0CAC20DF0C9C20CF0ED
:10438000C8C20BF084EC05F00EC075F00DC074F0DF
:104390000CC073F00BC072F0760E0E6E340E0D6E04
:1043A0000E0E0C6E7A0E0B6E75C012F074C011F00A
:1043B00073C010F072C00FF04AEC09F00EC079F033
:1043C0000DC078F00CC077F00BC076F023C20EF071
:1043D00022C20DF021C20CF020C20BF08BC212F0F1
:1043E0008AC211F089C210F088C20FF050EC08F0B8
:1043F00084EC05F00EC075F00DC074F00CC073F0C5
:104400000BC072F0BC0E0E6E910E0D6E790E0C6E1E
:104410000B6EE3C212F0E2C211F0E1C210F0E0C292
:104420000FF04AEC09F00EC02DF00DC02CF00CC0BE
:104430002BF00BC02AF02DC00EF02CC00DF02BC0BD
:104440000CF02AC00BF075C012F074C011F073C0EC
:1044500010F072C00FF04AEC09F00EC075F00DC0FC
:1044600074F00CC073F00BC072F0FBC20EF0FAC215
:104470000DF0F9C20CF0F8C20BF075C012F074C068
:1044800011F073C010F072C00FF04EEC08F00EC0C7
:104490002DF00DC02CF00CC02BF00BC02AF02DC05D
:1044A0000EF02CC00DF02BC00CF02AC00BF079C020
:1044B00012F078C011F077C010F076C00FF04EEC1B
:1044C00008F00EC0FBF20DC0FAF20CC0F9F20BC0FE
:1044D000F8F2CBC20EF0CAC20DF0C9C20CF0C8C2CD
:1044E0000BF0CFC212F0CEC211F0CDC210F0CCC290
:1044F0000FF04EEC08F00EC075F00DC074F00CC05B
:1045000073F00BC072F075C00EF074C00DF073C084
:104510000CF0723D02D0368272510B6E84EC05F0C5
:104520000EC075F00DC074F00CC073F00BC072F0CB
:10453000E70E0E6E190E0D6E7B0E0C6E780E0B6E66
:1045400075C012F074C011F073C010F072C00FF09B
:104550004AEC09F00EC075F00DC074F00CC073F099
:104560000BC072F075C00EF074C00DF073C00CF08B
:1045700072C00BF0FBC212F0FAC211F0F9C210F0D7
:10458000F8C20FF050EC08F00EC0FBF20DC0FAF2CA
:104590000CC0F9F20BC0F8F207C30EF006C30DF021
:1045A00005C30CF004C30BF08BC212F08AC211F0E9
:1045B00089C210F088C20FF050EC08F084EC05F0CE
:1045C0000EC075F00DC074F00CC073F00BC072F02B
:1045D0003E0E0E6E420E0D6E4D0E0C6E780E0B6E74
:1045E00075C012F074C011F073C010F072C00FF0FB
:1045F0004AEC09F00EC075F00DC074F00CC073F0F9
:104600000BC072F0FBC20EF0FAC20DF0F9C20CF052
:10461000F8C20BF075C012F074C011F073C010F046
:1046200072C00FF04EEC08F00EC0FBF20DC0FAF2B3
:104630000CC0F9F20BC0F8F207C30EF006C30DF080
:1046400005C30CF004C30BF08BC212F08AC211F048
:1046500089C210F088C20FF04EEC08F084EC05F02F
:104660000EC075F00DC074F00CC073F00BC072F08A
:10467000750E0E6EE50E0D6E330E0C6E780E0B6E13
:1046800075C012F074C011F073C010F072C00FF05A
:104690004AEC09F00EC075F00DC074F00CC073F058
:1046A0000BC072F0FBC20EF0FAC20DF0F9C20CF0B2
:1046B000F8C20BF075C012F074C011F073C010F0A6
:1046C00072C00FF04EEC08F00EC0FBF20DC0FAF213
:1046D0000CC0F9F20BC0F8F2F3C20EF0F2C20DF00A
:1046E000F1C20CF0F0C20BF08BC212F08AC211F0D2
:1046F00089C210F088C20FF04EEC08F084EC05F08F
:104700000EC075F00DC074F00CC073F00BC072F0E9
:104710000E6AE20E0D6E2E0E0C6E780E0B6E75C0CC
:1047200012F074C011F073C010F072C00FF04AECB8
:1047300009F00EC075F00DC074F00CC073F00BC022
:1047400072F0FBC20EF0FAC20DF0F9C20CF0F8C222
:104750000BF075C012F074C011F073C010F072C08D
:104760000FF050EC08F00EC0FBF20DC0FAF20CC0D6
:10477000F9F20BC0F8F2F7C20EF0F6C20DF0F5C276
:104780000CF0F4C20BF084EC05F00EC075F00DC017
:1047900074F00CC073F00BC072F0A50E0E6E650EB7
:1047A0000D6E240E0C6E780E0B6E75C012F074C078
:1047B00011F073C010F072C00FF04AEC09F00EC097
:1047C00075F00DC074F00CC073F00BC072F0FBC23A
:1047D0000EF0FAC20DF0F9C20CF0F8C20BF075C081
:1047E00012F074C011F073C010F072C00FF050ECF2
:1047F00008F00EC0FBF20DC0FAF20CC0F9F20BC0CB
:10480000F8F2F3C20EF0F2C20DF0F1C20CF0F0C2F9
:104810000BF0FFC212F0FEC211F0FDC210F0FCC29C
:104820000FF04EEC08F084EC05F00EC075F00DC0F2
:1048300074F00CC073F00BC072F0E90E0E6E0C0E2B
:104840000D6E0C6E780E0B6E75C012F074C011F008
:1048500073C010F072C00FF04AEC09F00EC075F092
:104860000DC074F00CC073F00BC072F0FBC20EF000
:10487000FAC20DF0F9C20CF0F8C20BF075C012F0DC
:1048800074C011F073C010F072C00FF050EC08F05B
:104890000EC0FBF20DC0FAF20CC0F9F20BC0F8F238
:1048A00023C20EF022C20DF021C20CF020C20BF088
:1048B0008BC212F08AC211F089C210F088C20FF0C8
:1048C0004EEC08F00EC02DF00DC02CF00CC02BF0FB
:1048D0000BC02AF02DC00EF02CC00DF02BC00CF038
:1048E0002AC00BF0EBC212F0EAC211F0E9C210F0DC
:1048F000E8C20FF050EC08F084EC05F00EC075F043
:104900000DC074F00CC073F00BC072F0F20E0E6E9E
:10491000980E0D6E010E0C6E780E0B6E75C012F0B7
:1049200074C011F073C010F072C00FF04AEC09F0BF
:104930000EC075F00DC074F00CC073F00BC072F0B7
:10494000E3C20EF0E2C20DF0E1C20CF0E0C20BF0E7
:1049500075C012F074C011F073C010F072C00FF087
:104960004AEC09F00EC075F00DC074F00CC073F085
:104970000BC072F0FBC20EF0FAC20DF0F9C20CF0DF
:10498000F8C20BF075C012F074C011F073C010F0D3
:1049900072C00FF04EEC08F00EC0FBF20DC0FAF240
:1049A0000CC0F9F20BC0F8F2EBC20EF0EAC20DF047
:1049B000E9C20CF0E8C20BF023C212F022C211F0DF
:1049C00021C210F020C20FF050EC08F084EC05F08A
:1049D0000EC075F00DC074F00CC073F00BC072F017
:1049E000EE0E0E6E430E0D6E5E0E0C6E770E0B6E9F
:1049F00075C012F074C011F073C010F072C00FF0E7
:104A00004AEC09F00EC075F00DC074F00CC073F0E4
:104A10000BC072F0E3C20EF0E2C20DF0E1C20CF086
:104A2000E0C20BF075C012F074C011F073C010F04A
:104A300072C00FF04AEC09F00EC075F00DC074F0B2
:104A40000CC073F00BC072F0FBC20EF0FAC20DF096
:104A5000F9C20CF0F8C20BF075C012F074C011F07E
:104A600073C010F072C00FF04EEC08F00EC0FBF2F5
:104A70000DC0FAF20CC0F9F20BC0F8F28BC20EF0C6
:104A80008AC20DF089C20CF088C20BF0CBC212F0C2
:104A9000CAC211F0C9C210F0C8C20FF04EEC08F043
:104AA00084EC05F00EC075F00DC074F00CC073F00E
:104AB0000BC072F00E68250E0D6E290E0C6E770E6F
:104AC0000B6E75C012F074C011F073C010F072C09C
:104AD0000FF04AEC09F00EC075F00DC074F00CC078
:104AE00073F00BC072F0FBC20EF0FAC20DF0F9C207
:104AF0000CF0F8C20BF075C012F074C011F073C066
:104B000010F072C00FF050EC08F00EC0FBF20DC0B8
:104B1000FAF20CC0F9F20BC0F8F223C20EF022C276
:104B20000DF021C20CF020C20BF0CBC212F0CAC2B1
:104B300011F0C9C210F0C8C20FF050EC08F084ECBC
:104B400005F00EC075F00DC074F00CC073F00BC012
:104B500072F00A0E0E6ED70E0D6E230E0C6E770ECF
:104B60000B6E75C012F074C011F073C010F072C0FB
:104B70000FF04AEC09F00EC075F00DC074F00CC0D7
:104B800073F00BC072F0E3C20EF0E2C20DF0E1C2AE
:104B90000CF0E0C20BF075C012F074C011F073C0DD
:104BA00010F072C00FF04AEC09F00EC075F00DC0A5
:104BB00074F00CC073F00BC072F0FBC20EF0FAC2BE
:104BC0000DF0F9C20CF0F8C20BF075C012F074C011
:104BD00011F073C010F072C00FF050EC08F00EC06E
:104BE000FBF20DC0FAF20CC0F9F20BC0F8F2F3C2FE
:104BF0000EF0F2C20DF0F1C20CF0F0C20BF084EC3A
:104C000005F00EC075F00DC074F00CC073F00BC051
:104C100072F09C0E0E6E190E0D6E7D0E0C6E760EE1
:104C20000B6E75C012F074C011F073C010F072C03A
:104C30000FF04AEC09F00EC075F00DC074F00CC016
:104C400073F00BC072F0FBC20EF0FAC20DF0F9C2A5
:104C50000CF0F8C20BF075C012F074C011F073C004
:104C600010F072C00FF050EC08F00EC0FBF20DC057
:104C7000FAF20CC0F9F20BC0F8F28BC20EF08AC245
:104C80000DF089C20CF088C20BF023C212F022C2D0
:104C900011F021C210F020C20FF04EEC08F00EC04F
:104CA0002DF00DC02CF00CC02BF00BC02AF02DC045
:104CB0000EF02CC00DF02BC00CF02AC00BF0EBC294
:104CC00012F0EAC211F0E9C210F0E8C20FF050ECA5
:104CD00008F084EC05F00EC075F00DC074F00CC047
:104CE00073F00BC072F0790E0E6EAD0E0D6E040EE9
:104CF0000C6E770E0B6E75C012F074C011F073C09D
:104D000010F072C00FF04AEC09F00EC075F00DC043
:104D100074F00CC073F00BC072F0E3C20EF0E2C28C
:104D20000DF0E1C20CF0E0C20BF075C012F074C0DF
:104D300011F073C010F072C00FF04AEC09F00EC011
:104D400075F00DC074F00CC073F00BC072F0FBC2B4
:104D50000EF0FAC20DF0F9C20CF0F8C20BF075C0FB
:104D600012F074C011F073C010F072C00FF050EC6C
:104D700008F00EC0FBF20DC0FAF20CC0F9F20BC045
:104D8000F8F28BC20EF08AC20DF089C20CF088C214
:104D90000BF0CBC212F0CAC211F0C9C210F0C8C2E7
:104DA0000FF050EC08F00EC075F00DC074F00CC0A0
:104DB00073F00BC072F075C00EF074C00DF073C0CC
:104DC0000CF0723D02D0368272510B6E84EC05F00D
:104DD0000EC075F00DC074F00CC073F00BC072F013
:104DE000E10E0E6EF00E0D6E020E0C6E770E0B6E57
:104DF00075C012F074C011F073C010F072C00FF0E3
:104E00004AEC09F00EC075F00DC074F00CC073F0E0
:104E10000BC072F0FBC20EF0FAC20DF0F9C20CF03A
:104E2000F8C20BF075C012F074C011F073C010F02E
:104E300072C00FF050EC08F00EC0FBF20DC0FAF299
:104E40000CC0F9F20BC0F8F2EBC20EF0EAC20DF0A2
:104E5000E9C20CF0E8C20BF0F7C212F0F6C211F092
:104E6000F5C210F0F4C20FF04EEC08F084EC05F03F
:104E70000EC075F00DC074F00CC073F00BC072F072
:104E80007F0E0E6E300E0D6E700E0C6E760E0B6E6B
:104E900075C012F074C011F073C010F072C00FF042
:104EA0004AEC09F00EC075F00DC074F00CC073F040
:104EB0000BC072F0FBC20EF0FAC20DF0F9C20CF09A
:104EC000F8C20BF075C012F074C011F073C010F08E
:104ED00072C00FF050EC08F00EC0FBF20DC0FAF2F9
:104EE0000CC0F9F20BC0F8F2FFC20EF0FEC20DF0DA
:104EF000FDC20CF0FCC20BF023C212F022C211F072
:104F000021C210F020C20FF04EEC08F084EC05F046
:104F10000EC075F00DC074F00CC073F00BC072F0D1
:104F2000990E0E6E9E0E0D6E300E0C6E760E0B6E82
:104F300075C012F074C011F073C010F072C00FF0A1
:104F40004AEC09F00EC075F00DC074F00CC073F09F
:104F50000BC072F0E3C20EF0E2C20DF0E1C20CF041
:104F6000E0C20BF075C012F074C011F073C010F005
:104F700072C00FF04AEC09F00EC075F00DC074F06D
:104F80000CC073F00BC072F0FBC20EF0FAC20DF051
:104F9000F9C20CF0F8C20BF075C012F074C011F039
:104FA00073C010F072C00FF050EC08F00EC0FBF2AE
:104FB0000DC0FAF20CC0F9F20BC0F8F2CFC20EF03D
:104FC000CEC20DF0CDC20CF0CCC20BF0CBC212F0B1
:104FD000CAC211F0C9C210F0C8C20FF050EC08F0FC
:104FE0000EC075F00DC074F00CC073F00BC072F001
:104FF000723F02D0368272078BC20EF08AC20DF069
:1050000089C20CF088C20BF075C012F074C011F0A8
:1050100073C010F072C00FF04EEC08F084EC05F095
:105020000EC075F00DC074F00CC073F00BC072F0C0
:10503000510E0E6E860E0D6E2A0E0C6E760E0B6ED7
:1050400075C012F074C011F073C010F072C00FF090
:105050004AEC09F00EC075F00DC074F00CC073F08E
:105060000BC072F0FBC20EF0FAC20DF0F9C20CF0E8
:10507000F8C20BF075C012F074C011F073C010F0DC
:1050800072C00FF050EC08F00EC0FBF20DC0FAF247
:105090000CC0F9F20BC0F8F2CBC20EF0CAC20DF090
:1050A000C9C20CF0C8C20BF08BC212F08AC211F058
:1050B00089C210F088C20FF04EEC08F00EC075F0F7
:1050C0000DC074F00CC073F00BC072F0723F02D0D0
:1050D0003682720775C00EF074C00DF073C00CF00C
:1050E00072C00BF023C212F022C211F021C210F0E4
:1050F00020C20FF04EEC08F084EC05F00EC075F005
:105100000DC074F00CC073F00BC072F0360E0E6E52
:10511000060E0D6E1D0E0C6E760E0B6E75C012F027
:1051200074C011F073C010F072C00FF04AEC09F0B7
:105130000EC075F00DC074F00CC073F00BC072F0AF
:10514000E3C20EF0E2C20DF0E1C20CF0E0C20BF0DF
:1051500075C012F074C011F073C010F072C00FF07F
:105160004AEC09F00EC075F00DC074F00CC073F07D
:105170000BC072F0FBC20EF0FAC20DF0F9C20CF0D7
:10518000F8C20BF075C012F074C011F073C010F0CB
:1051900072C00FF050EC08F00EC0FBF20DC0FAF236
:1051A0000CC0F9F20BC0F8F28BC20EF08AC20DF0FF
:1051B00089C20CF088C20BF0CBC212F0CAC211F047
:1051C000C9C210F0C8C20FF050EC08F084EC05F032
:1051D0000EC075F00DC074F00CC073F00BC072F00F
:1051E000AE0E0E6EF10E0D6E190E0C6E760E0B6E6F
:1051F00075C012F074C011F073C010F072C00FF0DF
:105200004AEC09F00EC075F00DC074F00CC073F0DC
:105210000BC072F0FBC20EF0FAC20DF0F9C20CF036
:10522000F8C20BF075C012F074C011F073C010F02A
:1052300072C00FF04EEC08F00EC0FBF20DC0FAF297
:105240000CC0F9F20BC0F8F2CBC20EF0CAC20DF0DE
:10525000C9C20CF0C8C20BF023C212F022C211F076
:1052600021C210F020C20FF04EEC08F00EC075F015
:105270000DC074F00CC073F00BC072F075C00EF06E
:1052800074C00DF073C00CF0723D02D036827251C2
:105290000B6E84EC05F00EC075F00DC074F00CC000
:1052A00073F00BC072F0F50E0E6E630E0D6E130EE2
:1052B0000C6E760E0B6E75C012F074C011F073C0D8
:1052C00010F072C00FF04AEC09F00EC075F00DC07E
:1052D00074F00CC073F00BC072F0E7C20EF0E6C2BF
:1052E0000DF0E5C20CF0E4C20BF075C012F074C012
:1052F00011F073C010F072C00FF04AEC09F00EC04C
:1053000075F00DC074F00CC073F00BC072F0FBC2EE
:105310000EF0FAC20DF0F9C20CF0F8C20BF075C035
:1053200012F074C011F073C010F072C00FF050ECA6
:1053300008F00EC0FBF20DC0FAF20CC0F9F20BC07F
:10534000F8F2FFC20EF0FEC20DF0FDC20CF0FCC27E
:105350000BF023C212F022C211F021C210F020C2C1
:105360000FF050EC08F084EC05F00EC075F00DC0A5
:1053700074F00CC073F00BC072F0960E0E6E430EFC
:105380000D6E0B0E0C6E760E0B6E75C012F074C0A7
:1053900011F073C010F072C00FF04AEC09F00EC0AB
:1053A00075F00DC074F00CC073F00BC072F0E3C266
:1053B0000EF0E2C20DF0E1C20CF0E0C20BF075C0DD
:1053C00012F074C011F073C010F072C00FF04AEC0C
:1053D00009F00EC075F00DC074F00CC073F00BC076
:1053E00072F0FBC20EF0FAC20DF0F9C20CF0F8C276
:1053F0000BF075C012F074C011F073C010F072C0E1
:105400000FF04EEC08F00EC0FBF20DC0FAF20CC02B
:10541000F9F20BC0F8F213C30EF012C30DF011C372
:105420000CF010C30BF084EC05F00EC075F00DC04D
:1054300074F00CC073F00BC072F0D50E0E6E3F0E00
:105440000D6E080E0C6E760E0B6E75C012F074C0E9
:1054500011F073C010F072C00FF04AEC09F00EC0EA
:1054600075F00DC074F00CC073F00BC072F0E7C2A1
:105470000EF0E6C20DF0E5C20CF0E4C20BF075C010
:1054800012F074C011F073C010F072C00FF04AEC4B
:1054900009F00EC075F00DC074F00CC073F00BC0B5
:1054A00072F0FBC20EF0FAC20DF0F9C20CF0F8C2B5
:1054B0000BF075C012F074C011F073C010F072C020
:1054C0000FF04EEC08F00EC0FBF20DC0FAF20CC06B
:1054D000F9F20BC0F8F2CBC20EF0CAC20DF0C9C28D
:1054E0000CF0C8C20BF023C212F022C211F021C28C
:1054F00010F020C20FF04EEC08F00EC02DF00DC0E1
:105500002CF00CC02BF00BC02AF02DC075F02CC075
:1055100074F02BC073F02A3C02D036822A50726F8E
:1055200075C00EF074C00DF073C00CF072C00BF0BB
:105530008BC212F08AC211F089C210F088C20FF03B
:105540004EEC08F084EC05F00EC075F00DC074F060
:105550000CC073F00BC072F04A0E0E6EF00E0D6EA2
:10556000060E0C6E760E0B6EE7C212F0E6C211F05C
:10557000E5C210F0E4C20FF04AEC09F00EC02DF0C5
:105580000DC02CF00CC02BF00BC02AF02DC00EF07B
:105590002CC00DF02BC00CF02AC00BF075C012F01F
:1055A00074C011F073C010F072C00FF04AEC09F033
:1055B0000EC075F00DC074F00CC073F00BC072F02B
:1055C000FBC20EF0FAC20DF0F9C20CF0F8C20BF0FB
:1055D00075C012F074C011F073C010F072C00FF0FB
:1055E00050EC08F00EC0FBF20DC0FAF20CC0F9F25C
:1055F0000BC0F8F2CBC20EF0CAC20DF0C9C20CF05B
:10560000C8C20BF0CFC212F0CEC211F0CDC210F062
:10561000CCC20FF04EEC08F00EC02DF00DC02CF0F7
:105620000CC02BF00BC02AF02DC075F02CC074F00C
:105630002BC073F02A3C02D036822A50726F8BC284
:105640000EF08AC20DF089C20CF088C20BF075C052
:1056500012F074C011F073C010F072C00FF050EC73
:1056600008F084EC05F00EC075F00DC074F00CC0AD
:1056700073F00BC072F0020E0E6E640E0D6E680EAB
:105680000C6E750E0B6E75C012F074C011F073C005
:1056900010F072C00FF04AEC09F00EC02DF00DC0F2
:1056A0002CF00CC02BF00BC02AF0FBC20EF0FAC29B
:1056B0000DF0F9C20CF0F8C20BF02DC012F02CC0A6
:1056C00011F02BC010F02AC00FF04EEC08F00EC005
:1056D000FBF20DC0FAF20CC0F9F20BC0F8F2CFC227
:1056E0000EF0CEC20DF0CDC20CF0CCC20BF0CBC28E
:1056F00012F0CAC211F0C9C210F0C8C20FF050ECCB
:1057000008F00EC02DF00DC02CF00CC02BF00BC01B
:105710002AF02DC00EF02CC00DF02BC00CF02A3C4E
:1057200002D036822A500B6E84EC05F00EC075F064
:105730000DC074F00CC073F00BC072F0520E0E6E00
:105740000F0E0D6E510E0C6E750E0B6E75C012F0B5
:1057500074C011F073C010F072C00FF04AEC09F081
:105760000EC02DF00DC02CF00CC02BF00BC02AF099
:10577000FBC20EF0FAC20DF0F9C20CF0F8C20BF049
:105780002DC012F02CC011F02BC010F02AC00FF069
:105790004EEC08F00EC0FBF20DC0FAF20CC0F9F2AC
:1057A0000BC0F8F2F3C20EF0F2C20DF0F1C20CF031
:1057B000F0C20BF023C212F022C211F021C210F08D
:1057C00020C20FF04EEC08F00EC02DF00DC02CF0F2
:1057D0000CC02BF00BC02AF02DC00EF02CC00DF029
:1057E0002BC00CF02AC00BF08BC212F08AC211F051
:1057F00089C210F088C20FF04EEC08F084EC05F07E
:105800000EC075F00DC074F00CC073F00BC072F0D8
:10581000680E0E6EE80E0D6E1F0E0C6E750E0B6E82
:10582000E3C212F0E2C211F0E1C210F0E0C20FF0E8
:105830004AEC09F00EC02DF00DC02CF00CC02BF07E
:105840000BC02AF02DC00EF02CC00DF02BC00CF0B8
:105850002AC00BF075C012F074C011F073C010F0C4
:1058600072C00FF04AEC09F00EC075F00DC074F074
:105870000CC073F00BC072F0FBC20EF0FAC20DF058
:10588000F9C20CF0F8C20BF075C012F074C011F040
:1058900073C010F072C00FF050EC08F00EC0FBF2B5
:1058A0000DC0FAF20CC0F9F20BC0F8F28BC20EF088
:1058B0008AC20DF089C20CF088C20BF0CFC212F080
:1058C000CEC211F0CDC210F0CCC20FF050EC08F0F7
:1058D0000EC02DF00DC02CF00CC02BF00BC02AF028
:1058E0002DC00EF02CC00DF02BC00CF02A3C02D0C5
:1058F00036822A500B6E84EC05F00EC075F00DC098
:1059000074F00CC073F00BC072F06B0E0E6E7D0E57
:105910000D6E110E0C6E750E0B6E75C012F074C00C
:1059200011F073C010F072C00FF04AEC09F00EC015
:105930002DF00DC02CF00CC02BF00BC02AF0FBC2D8
:105940000EF0FAC20DF0F9C20CF0F8C20BF02DC047
:1059500012F02CC011F02BC010F02AC00FF04EEC4A
:1059600008F00EC0FBF20DC0FAF20CC0F9F20BC049
:10597000F8F28BC20EF08AC20DF089C20CF088C218
:105980000BF0EFC212F0EEC211F0EDC210F0ECC25B
:105990000FF04EEC08F084EC05F00EC075F00DC071
:1059A00074F00CC073F00BC072F01B0E0E6ED50EAF
:1059B0000D6E690E0C6E740E0B6E75C012F074C015
:1059C00011F073C010F072C00FF04AEC09F00EC075
:1059D0002DF00DC02CF00CC02BF00BC02AF0FBC238
:1059E0000EF0FAC20DF0F9C20CF0F8C20BF02DC0A7
:1059F00012F02CC011F02BC010F02AC00FF050ECA8
:105A000008F00EC0FBF20DC0FAF20CC0F9F20BC0A8
:105A1000F8F223C20EF022C20DF021C20CF020C217
:105A20000BF08BC212F08AC211F089C210F088C24A
:105A30000FF050EC08F00EC02DF00DC02CF00CC093
:105A40002BF00BC02AF02DC00EF02CC00DF02BC097
:105A50000CF02AC00BF0EBC212F0EAC211F0E9C25E
:105A600010F0E8C20FF050EC08F084EC05F00EC026
:105A700075F00DC074F00CC073F00BC072F04A0EDC
:105A80000E6E990E0D6E540E0C6E740E0B6EE3C2FC
:105A900012F0E2C211F0E1C210F0E0C20FF04AECE5
:105AA00009F00EC02DF00DC02CF00CC02BF00BC077
:105AB0002AF02DC00EF02CC00DF02BC00CF02AC027
:105AC0000BF075C012F074C011F073C010F072C00A
:105AD0000FF04AEC09F00EC075F00DC074F00CC068
:105AE00073F00BC072F0FBC20EF0FAC20DF0F9C2F7
:105AF0000CF0F8C20BF075C012F074C011F073C056
:105B000010F072C00FF04EEC08F00EC0FBF20DC0AA
:105B1000FAF20CC0F9F20BC0F8F2F3C20EF0F2C2C6
:105B20000DF0F1C20CF0F0C20BF023C212F022C251
:105B300011F021C210F020C20FF04EEC08F00EC0A0
:105B40002DF00DC02CF00CC02BF00BC02AF02DC096
:105B50000EF02CC00DF02BC00CF02AC00BF0FFC2D1
:105B600012F0FEC211F0FDC210F0FCC20FF04EECBC
:105B700008F084EC05F00EC075F00DC074F00CC098
:105B800073F00BC072F0D80E0E6E7D0E0D6E470EC8
:105B90000C6E740E0B6EE3C212F0E2C211F0E1C2A1
:105BA00010F0E0C20FF04AEC09F00EC02DF00DC06D
:105BB0002CF00CC02BF00BC02AF02DC00EF02CC026
:105BC0000DF02BC00CF02AC00BF075C012F074C0A1
:105BD00011F073C010F072C00FF04AEC09F00EC063
:105BE00075F00DC074F00CC073F00BC072F0FBC206
:105BF0000EF0FAC20DF0F9C20CF0F8C20BF075C04D
:105C000012F074C011F073C010F072C00FF050ECBD
:105C100008F00EC0FBF20DC0FAF20CC0F9F20BC096
:105C2000F8F223C20EF022C20DF021C20CF020C205
:105C30000BF0CBC212F0CAC211F0C9C210F0C8C238
:105C40000FF050EC08F00EC02DF00DC02CF00CC081
:105C50002BF00BC02AF02DC075F02CC074F02BC0B7
:105C600073F02A3C02D036822A50726F8BC20EF03B
:105C70008AC20DF089C20CF088C20BF075C012F018
:105C800074C011F073C010F072C00FF04EEC08F049
:105C900084EC05F00EC075F00DC074F00CC073F00C
:105CA0000BC072F0A40E0E6E8C0E0D6E380E0C6EC4
:105CB000740E0B6EE7C212F0E6C211F0E5C210F0EE
:105CC000E4C20FF04AEC09F00EC02DF00DC02CF02C
:105CD0000CC02BF00BC02AF02DC00EF02CC00DF024
:105CE0002BC00CF02AC00BF075C012F074C011F07C
:105CF00073C010F072C00FF04AEC09F00EC075F0DE
:105D00000DC074F00CC073F00BC072F0FBC20EF04B
:105D1000FAC20DF0F9C20CF0F8C20BF075C012F027
:105D200074C011F073C010F072C00FF050EC08F0A6
:105D30000EC0FBF20DC0FAF20CC0F9F20BC0F8F283
:105D40008BC20EF08AC20DF089C20CF088C20BF033
:105D5000CBC212F0CAC211F0C9C210F0C8C20FF013
:105D60004EEC08F00EC02DF00DC02CF00CC02BF046
:105D70000BC02AF02DC075F02CC074F02BC073F04E
:105D80002A3C02D036822A50726F23C20EF022C201
:105D90000DF021C20CF020C20BF075C012F074C0DF
:105DA00011F073C010F072C00FF04EEC08F084ECEC
:105DB00005F00EC075F00DC074F00CC073F00BC090
:105DC00072F0710E0E6EAA0E0D6E350E0C6E740E04
:105DD0000B6EE3C212F0E2C211F0E1C210F0E0C2B9
:105DE0000FF04AEC09F00EC02DF00DC02CF00CC0E5
:105DF0002BF00BC02AF02DC00EF02CC00DF02BC0E4
:105E00000CF02AC00BF075C012F074C011F073C012
:105E100010F072C00FF04AEC09F00EC075F00DC022
:105E200074F00CC073F00BC072F0FBC20EF0FAC23B
:105E30000DF0F9C20CF0F8C20BF075C012F074C08E
:105E400011F073C010F072C00FF050EC08F00EC0EB
:105E5000FBF20DC0FAF20CC0F9F20BC0F8F2CBC2A3
:105E60000EF0CAC20DF0C9C20CF0C8C20BF0CFC20E
:105E700012F0CEC211F0CDC210F0CCC20FF04EEC39
:105E800008F00EC02DF00DC02CF00CC02BF00BC094
:105E90002AF02DC075F02CC074F02BC073F02A3C92
:105EA00002D036822A50726F75C00EF074C00DF0A9
:105EB00073C00CF072C00BF023C212F022C211F0BA
:105EC00021C210F020C20FF04EEC08F084EC05F077
:105ED0000EC075F00DC074F00CC073F00BC072F002
:105EE0001A0E0E6EC30E0D6E1C0E0C6E740E0B6E23
:105EF000E3C212F0E2C211F0E1C210F0E0C20FF012
:105F00004AEC09F00EC02DF00DC02CF00CC02BF0A7
:105F10000BC02AF02DC00EF02CC00DF02BC00CF0E1
:105F20002AC00BF075C012F074C011F073C010F0ED
:105F300072C00FF04AEC09F00EC075F00DC074F09D
:105F40000CC073F00BC072F0FBC20EF0FAC20DF081
:105F5000F9C20CF0F8C20BF075C012F074C011F069
:105F600073C010F072C00FF050EC08F00EC0FBF2DE
:105F70000DC0FAF20CC0F9F20BC0F8F28BC20EF0B1
:105F80008AC20DF089C20CF088C20BF0F3C212F085
:105F9000F2C211F0F1C210F0F0C20FF050EC08F0B4
:105FA00084EC05F00EC075F00DC074F00CC073F0F9
:105FB0000BC072F0E00E0E6E2D0E0D6E100E0C6EFC
:105FC000740E0B6E75C012F074C011F073C010F037
:105FD00072C00FF04AEC09F00EC075F00DC074F0FD
:105FE0000CC073F00BC072F003C30EF002C30DF0CF
:105FF00001C30CF000C30BF084EC05F00EC079F087
:106000000DC078F00CC077F00BC076F0920E0E6EDB
:10601000080E0D6E0D0E0C6E740E0B6E79C012F024
:1060200078C011F077C010F076C00FF04AEC09F09C
:106030000EC079F00DC078F00CC077F00BC076F090
:10604000FBC20EF0FAC20DF0F9C20CF0F8C20BF070
:1060500075C012F074C011F073C010F072C00FF070
:1060600050EC08F00EC02DF00DC02CF00CC02BF041
:106070000BC02AF02DC00EF02CC00DF02BC00CF080
:106080002AC00BF079C012F078C011F077C010F080
:1060900076C00FF050EC08F00EC0FBF20DC0FAF223
:1060A0000CC0F9F20BC0F8F2F3C20EF0F2C20DF020
:1060B000F1C20CF0F0C20BF023C212F022C211F0B8
:1060C00021C210F020C20FF04EEC08F084EC05F075
:1060D0000EC075F00DC074F00CC073F00BC072F000
:1060E00075C00EF074C00DF073C00CF072C00BF0F0
:1060F000E3C212F0E2C211F0E1C210F0E0C20FF010
:106100004AEC09F00EC02DF00DC02CF00CC02BF0A5
:106110000BC02AF0B80E0E6E930E0D6E080E0C6EAC
:10612000740E0B6E2DC012F02CC011F02BC010F0AD
:106130002AC00FF04AEC09F00EC075F00DC074F0E3
:106140000CC073F00BC072F0FBC20EF0FAC20DF07F
:10615000F9C20CF0F8C20BF075C012F074C011F067
:1061600073C010F072C00FF050EC08F00EC0FBF2DC
:106170000DC0FAF20CC0F9F20BC0F8F2FFC20EF03B
:10618000FEC20DF0FDC20CF0FCC20BF0CBC212F04F
:10619000CAC211F0C9C210F0C8C20FF04EEC08F02C
:1061A00084EC05F00EC075F00DC074F00CC073F0F7
:1061B0000BC072F0D10E0E6ECD0E0D6E7E0E0C6EFB
:1061C000730E0B6E75C012F074C011F073C010F036
:1061D00072C00FF04AEC09F00EC02DF00DC02CF08B
:1061E0000CC02BF00BC02AF02DC00EF02CC00DF00F
:1061F0002BC00CF02AC00BF0FBC212F0FAC211F057
:10620000F9C210F0F8C20FF050EC08F00EC0FBF22B
:106210000DC0FAF20CC0F9F20BC0F8F28BC20EF00E
:106220008AC20DF089C20CF088C20BF013C312F0C1
:1062300012C311F011C310F010C30FF04EEC08F0B0
:1062400084EC05F00EC075F00DC074F00CC073F056
:106250000BC072F00E0E0E6EF50E0D6E3B0E0C6E38
:10626000740E0B6E75C012F074C011F073C010F094
:1062700072C00FF04AEC09F00EC02DF00DC02CF0EA
:106280000CC02BF00BC02AF02DC00EF02CC00DF06E
:106290002BC00CF02AC00BF0E7C212F0E6C211F0DE
:1062A000E5C210F0E4C20FF04AEC09F00EC075F040
:1062B0000DC074F00CC073F00BC072F075C00EF01E
:1062C00074C00DF073C00CF072C00BF0FBC212F082
:1062D000FAC211F0F9C210F0F8C20FF050EC08F059
:1062E0000EC0FBF20DC0FAF20CC0F9F20BC0F8F2CE
:1062F000340E0E6EFA0E0D6E0E0E0C6E790E0B6EC7
:10630000FBC212F0FAC211F0F9C210F0F8C20FF09D
:106310004AEC09F00EC02DF00DC02CF00CC02BF093
:106320000BC02AF087C20EF086C20DF085C20CF0B9
:1063300084C20BF02DC012F02CC011F02BC010F055
:106340002AC00FF050EC08F00EC00FF30DC00EF392
:106350000CC00DF30BC00CF303010C53000121E042
:10636000D89603010DAFD88600011BE4DA0E0E6E3D
:106370000F0E0D6E490E0C6E810E0B6E0FC312F0D8
:106380000EC311F00DC310F00CC30FF050EC08F069
:106390000EC00FF30DC00EF30CC00DF30BC00CF3C9
:1063A000DBD7DA0E0E6E0F0E0D6E490E0C6E810EDF
:1063B0000B6E0FC312F00EC311F00DC310F00CC31F
:1063C0000FF09EEC07F001081BE0DA0E126E0F0EC4
:1063D000116E490E106E810E0F6E0FC30EF00EC3BC
:1063E0000DF00DC30CF00CC30BF04EEC08F00EC01A
:1063F0000FF30DC00EF30CC00DF30BC00CF3D1D78F
:10640000CFC20EF0CEC20DF0CDC20CF0CCC20BF05C
:1064100084EC05F00EC02DF00DC02CF00CC02BF05C
:106420000BC02AF0200E0E6E1A0E0D6E240E0C6E8E
:10643000810E0B6E2DC012F02CC011F02BC010F08D
:106440002AC00FF04AEC09F00EC075F00DC074F0D0
:106450000CC073F00BC072F08BC20EF08AC20DF04C
:1064600089C20CF088C20BF0CFC212F0CEC211F07C
:10647000CDC210F0CCC20FF050EC08F084EC05F067
:106480000EC079F00DC078F00CC077F00BC076F03C
:10649000970E0E6EAB0E0D6E0F0E0C6E7D0E0B6E0C
:1064A00079C012F078C011F077C010F076C00FF00C
:1064B0004AEC09F00EC02DF00DC02CF00CC02BF0F2
:1064C0000BC02AF02DC00EF02CC00DF02BC00CF02C
:1064D0002AC00BF075C012F074C011F073C010F038
:1064E00072C00FF050EC08F00EC017F30DC016F399
:1064F0000CC015F30BC014F38BC20EF08AC20DF062
:1065000089C20CF088C20BF0CFC212F0CEC211F0DB
:10651000CDC210F0CCC20FF04EEC08F084EC05F0C8
:106520000EC075F00DC074F00CC073F00BC072F0AB
:10653000C70E0E6E2D0E0D6E0E0E0C6E7D0E0B6EBA
:1065400075C012F074C011F073C010F072C00FF07B
:106550004AEC09F00EC02DF00DC02CF00CC02BF051
:106560000BC02AF02DC00EF02CC00DF02BC00CF08B
:106570002AC00BF017C312F016C311F015C310F0A8
:1065800014C30FF050EC08F00EC017F30DC016F353
:106590000CC015F30BC014F3EBC20EF0EAC20DF001
:1065A000E9C20CF0E8C20BF0CFC212F0CEC211F07B
:1065B000CDC210F0CCC20FF04EEC08F084EC05F028
:1065C0000EC075F00DC074F00CC073F00BC072F00B
:1065D0004D0E0E6E650E0D6E310E0C6E7C0E0B6E3A
:1065E00075C012F074C011F073C010F072C00FF0DB
:1065F0004AEC09F00EC02DF00DC02CF00CC02BF0B1
:106600000BC02AF02DC00EF02CC00DF02BC00CF0EA
:106610002AC00BF017C312F016C311F015C310F007
:1066200014C30FF050EC08F00EC017F30DC016F3B2
:106630000CC015F30BC014F3EBC20EF0EAC20DF060
:10664000E9C20CF0E8C20BF0CFC212F0CEC211F0DA
:10665000CDC210F0CCC20FF050EC08F00EC02DF0FF
:106660000DC02CF00CC02BF00BC02AF02DC00EF08A
:106670002CC00DF02BC00CF02AC00BF08BC212F016
:106680008AC211F089C210F088C20FF04EEC08F0F7
:1066900084EC05F00EC075F00DC074F00CC073F002
:1066A0000BC072F0BE0E0E6EF80E0D6E620E0C6E0A
:1066B0007A0E0B6E75C012F074C011F073C010F03A
:1066C00072C00FF04AEC09F00EC02DF00DC02CF096
:1066D0000CC02BF00BC02AF017C30EF016C30DF040
:1066E00015C30CF014C30BF02DC012F02CC011F028
:1066F0002BC010F02AC00FF050EC08F00EC017F3BA
:106700000DC016F30CC015F30BC014F3EBC20EF062
:10671000EAC20DF0E9C20CF0E8C20BF0CFC212F0F1
:10672000CEC211F0CDC210F0CCC20FF04EEC08F08A
:106730000EC02DF00DC02CF00CC02BF00BC02AF0B9
:106740002DC00EF02CC00DF02BC00CF02AC00BF0A9
:106750008BC212F08AC211F089C210F088C20FF009
:106760004EEC08F084EC05F00EC075F00DC074F02E
:106770000CC073F00BC072F0B50E0E6E870E0D6E6E
:106780003D0E0C6E7A0E0B6E75C012F074C011F0D7
:1067900073C010F072C00FF04AEC09F00EC075F033
:1067A0000DC074F00CC073F00BC072F017C30EF084
:1067B00016C30DF015C30CF014C30BF075C012F026
:1067C00074C011F073C010F072C00FF050EC08F0FC
:1067D0000EC017F30DC016F30CC015F30BC014F365
:1067E000EBC20EF0EAC20DF0E9C20CF0E8C20BF009
:1067F000CFC212F0CEC211F0CDC210F0CCC20FF059
:1068000050EC08F084EC05F00EC075F00DC074F08B
:106810000CC073F00BC072F0440E0E6E6B0E0D6E5A
:10682000050E0C6E7A0E0B6E75C012F074C011F06E
:1068300073C010F072C00FF04AEC09F00EC075F092
:106840000DC074F00CC073F00BC072F017C30EF0E3
:1068500016C30DF015C30CF014C30BF075C012F085
:1068600074C011F073C010F072C00FF050EC08F05B
:106870000EC017F30DC016F30CC015F30BC014F3C4
:10688000FFC20EF0FEC20DF0FDC20CF0FCC20BF018
:10689000CFC212F0CEC211F0CDC210F0CCC20FF0B8
:1068A00050EC08F084EC05F00EC075F00DC074F0EB
:1068B0000CC073F00BC072F0D20E0E6EE20E0D6EB5
:1068C0000C0E0C6E790E0B6E75C012F074C011F0C8
:1068D00073C010F072C00FF04AEC09F00EC075F0F2
:1068E0000DC074F00CC073F00BC072F017C30EF043
:1068F00016C30DF015C30CF014C30BF075C012F0E5
:1069000074C011F073C010F072C00FF050EC08F0BA
:106910000EC017F30DC016F30CC015F30BC014F323
:10692000EBC20EF0EAC20DF0E9C20CF0E8C20BF0C7
:106930008BC212F08AC211F089C210F088C20FF027
:1069400050EC08F00EC02DF00DC02CF00CC02BF058
:106950000BC02AF02DC00EF02CC00DF02BC00CF097
:106960002AC00BF0CFC212F0CEC211F0CDC210F08F
:10697000CCC20FF04EEC08F084EC05F00EC075F0C0
:106980000DC074F00CC073F00BC072F09D0E0E6E53
:10699000D40E0D6E170E0C6E780E0B6E75C012F0C5
:1069A00074C011F073C010F072C00FF04AEC09F01F
:1069B0000EC075F00DC074F00CC073F00BC072F017
:1069C00017C30EF016C30DF015C30CF014C30BF073
:1069D00075C012F074C011F073C010F072C00FF0E7
:1069E00050EC08F00EC017F30DC016F30CC015F3F1
:1069F0000BC014F3FFC20EF0FEC20DF0FDC20CF08E
:106A0000FCC20BF0CFC212F0CEC211F0CDC210F01A
:106A1000CCC20FF04EEC08F084EC05F00EC075F01F
:106A20000DC074F00CC073F00BC072F0580E0E6EF7
:106A30008E0E0D6E100E0C6E780E0B6E75C012F071
:106A400074C011F073C010F072C00FF04AEC09F07E
:106A50000EC075F00DC074F00CC073F00BC072F076
:106A600017C30EF016C30DF015C30CF014C30BF0D2
:106A700075C012F074C011F073C010F072C00FF046
:106A800050EC08F00EC017F30DC016F30CC015F350
:106A90000BC014F3EBC20EF0EAC20DF0E9C20CF029
:106AA000E8C20BF023C212F022C211F021C210F092
:106AB00020C20FF04EEC08F00EC02DF00DC02CF0EF
:106AC0000CC02BF00BC02AF02DC00EF02CC00DF026
:106AD0002BC00CF02AC00BF0CFC212F0CEC211F0C6
:106AE000CDC210F0CCC20FF04EEC08F084EC05F0F3
:106AF0000EC075F00DC074F00CC073F00BC072F0D6
:106B00006D0E0E6E1E0E0D6E070E0C6E780E0B6E59
:106B100075C012F074C011F073C010F072C00FF0A5
:106B20004AEC09F00EC075F00DC074F00CC073F0A3
:106B30000BC072F0E3C20EF0E2C20DF0E1C20CF045
:106B4000E0C20BF075C012F074C011F073C010F009
:106B500072C00FF04AEC09F00EC075F00DC074F071
:106B60000CC073F00BC072F017C30EF016C30DF01B
:106B700015C30CF014C30BF075C012F074C011F003
:106B800073C010F072C00FF050EC08F00EC017F395
:106B90000DC016F30CC015F30BC014F3CBC20EF0EE
:106BA000CAC20DF0C9C20CF0C8C20BF08BC212F001
:106BB0008AC211F089C210F088C20FF04EEC08F0C2
:106BC0000EC075F00DC074F00CC073F00BC072F005
:106BD000723F02D03682720775C00EF074C00DF09D
:106BE00073C00CF072C00BF0CFC212F0CEC211F025
:106BF000CDC210F0CCC20FF04EEC08F084EC05F0E2
:106C00000EC075F00DC074F00CC073F00BC072F0C4
:106C1000F40E0E6EA70E0D6E0D0E0C6E770E0B6E33
:106C200075C012F074C011F073C010F072C00FF094
:106C30004AEC09F00EC075F00DC074F00CC073F092
:106C40000BC072F017C30EF016C30DF015C30CF095
:106C500014C30BF075C012F074C011F073C010F0C3
:106C600072C00FF050EC08F00EC017F30DC016F311
:106C70000CC015F30BC014F3EBC20EF0EAC20DF01A
:106C8000E9C20CF0E8C20BF0CFC212F0CEC211F094
:106C9000CDC210F0CCC20FF050EC08F00EC02DF0B9
:106CA0000DC02CF00CC02BF00BC02AF02DC00EF044
:106CB0002CC00DF02BC00CF02AC00BF08BC212F0D0
:106CC0008AC211F089C210F088C20FF050EC08F0AF
:106CD00084EC05F00EC075F00DC074F00CC073F0BC
:106CE0000BC072F0270E0E6EA00E0D6E090E0C6E0C
:106CF000770E0B6E75C012F074C011F073C010F0F7
:106D000072C00FF04AEC09F00EC075F00DC074F0BF
:106D10000CC073F00BC072F017C30EF016C30DF069
:106D200015C30CF014C30BF075C012F074C011F051
:106D300073C010F072C00FF050EC08F00EC017F3E3
:106D40000DC016F30CC015F30BC014F3CFC20EF038
:106D5000CEC20DF0CDC20CF0CCC20BF023C212F0AB
:106D600022C211F021C210F020C20FF04EEC08F048
:106D70000EC02DF00DC02CF00CC02BF00BC02AF073
:106D80002DC00EF02CC00DF02BC00CF02AC00BF063
:106D9000EBC212F0EAC211F0E9C210F0E8C20FF043
:106DA0004EEC08F084EC05F00EC075F00DC074F0E8
:106DB0000CC073F00BC072F0C60E0E6EFC0E0D6EA2
:106DC0005C0E0C6E760E0B6E75C012F074C011F076
:106DD00073C010F072C00FF04AEC09F00EC075F0ED
:106DE0000DC074F00CC073F00BC072F0E3C20EF073
:106DF000E2C20DF0E1C20CF0E0C20BF075C012F07F
:106E000074C011F073C010F072C00FF04AEC09F0BA
:106E10000EC075F00DC074F00CC073F00BC072F0B2
:106E200017C30EF016C30DF015C30CF014C30BF00E
:106E300075C012F074C011F073C010F072C00FF082
:106E400050EC08F00EC017F30DC016F30CC015F38C
:106E50000BC014F3EBC20EF0EAC20DF0E9C20CF065
:106E6000E8C20BF0CFC212F0CEC211F0CDC210F0CA
:106E7000CCC20FF050EC08F00EC075F00DC074F0ED
:106E80000CC073F00BC072F075C00EF074C00DF042
:106E900073C00CF072C00BF023C212F022C211F0CA
:106EA00021C210F020C20FF04EEC08F00EC02DF001
:106EB0000DC02CF00CC02BF00BC02AF02DC00EF032
:106EC0002CC00DF02BC00CF02AC00BF08BC212F0BE
:106ED0008AC211F089C210F088C20FF04EEC08F09F
:106EE00084EC05F00EC075F00DC074F00CC073F0AA
:106EF0000BC072F0470E0E6E010E0D6E220E0C6E60
:106F0000760E0B6E75C012F074C011F073C010F0E5
:106F100072C00FF04AEC09F00EC075F00DC074F0AD
:106F20000CC073F00BC072F0E3C20EF0E2C20DF0C1
:106F3000E1C20CF0E0C20BF075C012F074C011F0A9
:106F400073C010F072C00FF04AEC09F00EC075F07B
:106F50000DC074F00CC073F00BC072F017C30EF0CC
:106F600016C30DF015C30CF014C30BF075C012F06E
:106F700074C011F073C010F072C00FF050EC08F044
:106F80000EC017F30DC016F30CC015F30BC014F3AD
:106F9000EBC20EF0EAC20DF0E9C20CF0E8C20BF051
:106FA000CFC212F0CEC211F0CDC210F0CCC20FF0A1
:106FB00050EC08F00EC02DF00DC02CF00CC02BF0E2
:106FC0000BC02AF02DC00EF02CC00DF02BC00CF021
:106FD0002AC00BF023C212F022C211F021C210F01D
:106FE00020C20FF04EEC08F084EC05F00EC075F0F6
:106FF0000DC074F00CC073F00BC072F0F90E0E6E81
:107000009E0E0D6E110E0C6E760E0B6E75C012F08C
:1070100074C011F073C010F072C00FF04AEC09F0A8
:107020000EC075F00DC074F00CC073F00BC072F0A0
:10703000E3C20EF0E2C20DF0E1C20CF0E0C20BF0D0
:1070400075C012F074C011F073C010F072C00FF070
:107050004AEC09F00EC075F00DC074F00CC073F06E
:107060000BC072F017C30EF016C30DF015C30CF071
:1070700014C30BF075C012F074C011F073C010F09F
:1070800072C00FF050EC08F00EC017F30DC016F3ED
:107090000CC015F30BC014F3EBC20EF0EAC20DF0F6
:1070A000E9C20CF0E8C20BF0CFC212F0CEC211F070
:1070B000CDC210F0CCC20FF04EEC08F00EC075F04F
:1070C0000DC074F00CC073F00BC072F075C00EF000
:1070D00074C00DF073C00CF072C00BF023C212F03C
:1070E00022C211F021C210F020C20FF04EEC08F0C5
:1070F0000EC02DF00DC02CF00CC02BF00BC02AF0F0
:107100002DC00EF02CC00DF02BC00CF02AC00BF0DF
:107110008BC212F08AC211F089C210F088C20FF03F
:107120004EEC08F084EC05F00EC075F00DC074F064
:107130000CC073F00BC072F0640E0E6ECA0E0D6EB2
:10714000070E0C6E760E0B6E75C012F074C011F047
:1071500073C010F072C00FF04AEC09F00EC075F069
:107160000DC074F00CC073F00BC072F0E3C20EF0EF
:10717000E2C20DF0E1C20CF0E0C20BF075C012F0FB
:1071800074C011F073C010F072C00FF04AEC09F037
:107190000EC075F00DC074F00CC073F00BC072F02F
:1071A00017C30EF016C30DF015C30CF014C30BF08B
:1071B00075C012F074C011F073C010F072C00FF0FF
:1071C00050EC08F00EC017F30DC016F30CC015F309
:1071D0000BC014F3CFC20EF0CEC20DF0CDC20CF036
:1071E000CCC20BF023C212F022C211F021C210F067
:1071F00020C20FF04EEC08F00EC02DF00DC02CF0A8
:107200000CC02BF00BC02AF02DC00EF02CC00DF0DE
:107210002BC00CF02AC00BF08BC212F08AC211F006
:1072200089C210F088C20FF050EC08F084EC05F031
:107230000EC075F00DC074F00CC073F00BC072F08E
:10724000AB0E0E6E050E0D6E760E0C6E750E0B6E81
:1072500075C012F074C011F073C010F072C00FF05E
:107260004AEC09F00EC075F00DC074F00CC073F05C
:107270000BC072F0E3C20EF0E2C20DF0E1C20CF0FE
:10728000E0C20BF075C012F074C011F073C010F0C2
:1072900072C00FF04AEC09F00EC075F00DC074F02A
:1072A0000CC073F00BC072F017C30EF016C30DF0D4
:1072B00015C30CF014C30BF075C012F074C011F0BC
:1072C00073C010F072C00FF050EC08F00EC017F34E
:1072D0000DC016F30CC015F30BC014F3F3C20EF07F
:1072E000F2C20DF0F1C20CF0F0C20BF0CFC212F0FE
:1072F000CEC211F0CDC210F0CCC20FF04EEC08F0AF
:107300000EC02DF00DC02CF00CC02BF00BC02AF0DD
:107310002DC00EF02CC00DF02BC00CF02AC00BF0CD
:107320008BC212F08AC211F089C210F088C20FF02D
:107330004EEC08F084EC05F00EC075F00DC074F052
:107340000CC073F00BC072F0800E0E6E990E0D6EB5
:107350006F0E0C6E750E0B6E75C012F074C011F0CE
:1073600073C010F072C00FF04AEC09F00EC075F057
:107370000DC074F00CC073F00BC072F017C30EF0A8
:1073800016C30DF015C30CF014C30BF075C012F04A
:1073900074C011F073C010F072C00FF050EC08F020
:1073A0000EC017F30DC016F30CC015F30BC014F389
:1073B000CFC20EF0CEC20DF0CDC20CF0CCC20BF09D
:1073C00023C212F022C211F021C210F020C20FF02D
:1073D00050EC08F084EC05F00EC075F00DC074F0B0
:1073E0000CC073F00BC072F0A40E0E6E520E0D6E38
:1073F0006C0E0C6E750E0B6E75C012F074C011F031
:1074000073C010F072C00FF04AEC09F00EC075F0B6
:107410000DC074F00CC073F00BC072F0E3C20EF03C
:10742000E2C20DF0E1C20CF0E0C20BF075C012F048
:1074300074C011F073C010F072C00FF04AEC09F084
:107440000EC079F00DC078F00CC077F00BC076F06C
:107450000BC30EF00AC30DF009C30CF008C30BF008
:1074600084EC05F00EC075F00DC074F00CC073F024
:107470000BC072F0420E0E6E600E0D6E650E0C6E3D
:10748000750E0B6E75C012F074C011F073C010F061
:1074900072C00FF04AEC09F00EC075F00DC074F028
:1074A0000CC073F00BC072F017C30EF016C30DF0D2
:1074B00015C30CF014C30BF079C012F078C011F0B2
:1074C00077C010F076C00FF04EEC08F00EC02DF033
:1074D0000DC02CF00CC02BF00BC02AF02DC00EF00C
:1074E0002CC00DF02BC00CF02AC00BF075C012F0B0
:1074F00074C011F073C010F072C00FF04EEC08F0C1
:107500000EC017F30DC016F30CC015F30BC014F327
:107510008BC20EF08AC20DF089C20CF088C20BF04B
:1075200023C212F022C211F021C210F020C20FF0CB
:107530004EEC08F00EC02DF00DC02CF00CC02BF05E
:107540000BC02AF02DC00EF02CC00DF02BC00CF09B
:107550002AC00BF0CFC212F0CEC211F0CDC210F093
:10756000CCC20FF04EEC08F084EC05F00EC075F0C4
:107570000DC074F00CC073F00BC072F0750E0E6E7F
:10758000C80E0D6E4D0E0C6E750E0B6E75C012F0A2
:1075900074C011F073C010F072C00FF04AEC09F023
:1075A0000EC075F00DC074F00CC073F00BC072F01B
:1075B000E3C20EF0E2C20DF0E1C20CF0E0C20BF04B
:1075C00075C012F074C011F073C010F072C00FF0EB
:1075D0004AEC09F00EC075F00DC074F00CC073F0E9
:1075E0000BC072F017C30EF016C30DF015C30CF0EC
:1075F00014C30BF075C012F074C011F073C010F01A
:1076000072C00FF050EC08F00EC017F30DC016F367
:107610000CC015F30BC014F3CFC20EF0CEC20DF0A8
:10762000CDC20CF0CCC20BF0CBC212F0CAC211F02A
:10763000C9C210F0C8C20FF050EC08F084EC05F09D
:107640000EC075F00DC074F00CC073F00BC072F07A
:10765000710E0E6EE70E0D6E420E0C6E750E0B6EF9
:1076600075C012F074C011F073C010F072C00FF04A
:107670004AEC09F00EC075F00DC074F00CC073F048
:107680000BC072F017C30EF016C30DF015C30CF04B
:1076900014C30BF075C012F074C011F073C010F079
:1076A00072C00FF04EEC08F00EC017F30DC016F3C9
:1076B0000CC015F30BC014F3CFC20EF0CEC20DF008
:1076C000CDC20CF0CCC20BF023C212F022C211F0DA
:1076D00021C210F020C20FF050EC08F00EC02DF0C7
:1076E0000DC02CF00CC02BF00BC02AF02DC00EF0FA
:1076F0002CC00DF02BC00CF02AC00BF08BC212F086
:107700008AC211F089C210F088C20FF050EC08F064
:1077100084EC05F00EC075F00DC074F00CC073F071
:107720000BC072F01D0E0E6E1E0E0D6E420E0C6E14
:10773000750E0B6E75C012F074C011F073C010F0AE
:1077400072C00FF04AEC09F00EC075F00DC074F075
:107750000CC073F00BC072F0E3C20EF0E2C20DF089
:10776000E1C20CF0E0C20BF075C012F074C011F071
:1077700073C010F072C00FF04AEC09F00EC075F043
:107780000DC074F00CC073F00BC072F017C30EF094
:1077900016C30DF015C30CF014C30BF075C012F036
:1077A00074C011F073C010F072C00FF04EEC08F00E
:1077B0000EC017F30DC016F30CC015F30BC014F375
:1077C000CFC20EF0CEC20DF0CDC20CF0CCC20BF089
:1077D00023C212F022C211F021C210F020C20FF019
:1077E0004EEC08F00EC02DF00DC02CF00CC02BF0AC
:1077F0000BC02AF02DC00EF02CC00DF02BC00CF0E9
:107800002AC00BF08BC212F08AC211F089C210F0AC
:1078100088C20FF04EEC08F084EC05F00EC075F055
:107820000DC074F00CC073F00BC072F0A10E0E6EA0
:10783000BA0E0D6E390E0C6E750E0B6E75C012F011
:1078400074C011F073C010F072C00FF04AEC09F070
:107850000EC075F00DC074F00CC073F00BC072F068
:10786000E3C20EF0E2C20DF0E1C20CF0E0C20BF098
:1078700075C012F074C011F073C010F072C00FF038
:107880004AEC09F00EC075F00DC074F00CC073F036
:107890000BC072F017C30EF016C30DF015C30CF039
:1078A00014C30BF075C012F074C011F073C010F067
:1078B00072C00FF050EC08F00EC017F30DC016F3B5
:1078C0000CC015F30BC014F3CFC20EF0CEC20DF0F6
:1078D000CDC20CF0CCC20BF023C212F022C211F0C8
:1078E00021C210F020C20FF04EEC08F084EC05F03D
:1078F0000EC075F00DC074F00CC073F00BC072F0C8
:107900007C0E0E6EF20E0D6E300E0C6E750E0B6E42
:1079100075C012F074C011F073C010F072C00FF097
:107920004AEC09F00EC075F00DC074F00CC073F095
:107930000BC072F0E3C20EF0E2C20DF0E1C20CF037
:10794000E0C20BF075C012F074C011F073C010F0FB
:1079500072C00FF04AEC09F00EC075F00DC074F063
:107960000CC073F00BC072F017C30EF016C30DF00D
:1079700015C30CF014C30BF075C012F074C011F0F5
:1079800073C010F072C00FF050EC08F00EC017F387
:107990000DC016F30CC015F30BC014F3CFC20EF0DC
:1079A000CEC20DF0CDC20CF0CCC20BF0CBC212F0A7
:1079B000CAC211F0C9C210F0C8C20FF04EEC08F0F4
:1079C00084EC05F00EC075F00DC074F00CC073F0BF
:1079D0000BC072F0650E0E6E530E0D6E2E0E0C6EF9
:1079E000750E0B6E75C012F074C011F073C010F0FC
:1079F00072C00FF04AEC09F00EC075F00DC074F0C3
:107A00000CC073F00BC072F017C30EF016C30DF06C
:107A100015C30CF014C30BF075C012F074C011F054
:107A200073C010F072C00FF050EC08F00EC017F3E6
:107A30000DC016F30CC015F30BC014F3CFC20EF03B
:107A4000CEC20DF0CDC20CF0CCC20BF0F7C212F0DA
:107A5000F6C211F0F5C210F0F4C20FF050EC08F0CD
:107A600084EC05F00EC075F00DC074F00CC073F01E
:107A70000BC072F0340E0E6EF70E0D6E100E0C6E03
:107A8000750E0B6E75C012F074C011F073C010F05B
:107A900072C00FF04AEC09F00EC075F00DC074F022
:107AA0000CC073F00BC072F0F3C20EF0F2C20DF016
:107AB000F1C20CF0F0C20BF0CFC212F0CEC211F046
:107AC000CDC210F0CCC20FF04EEC08F084EC05F003
:107AD0000EC079F00DC078F00CC077F00BC076F0D6
:107AE000850E0E6EB10E0D6E050E0C6E750E0B6EC4
:107AF00079C012F078C011F077C010F076C00FF0A6
:107B00004AEC09F00EC079F00DC078F00CC077F0A7
:107B10000BC076F075C00EF074C00DF073C00CF0A1
:107B200072C00BF079C012F078C011F077C010F07D
:107B300076C00FF050EC08F00EC075F00DC074F078
:107B40000CC073F00BC072F017C30EF016C30DF02B
:107B500015C30CF014C30BF075C012F074C011F013
:107B600073C010F072C00FF050EC08F00EC017F3A5
:107B70000DC016F30CC015F30BC014F3CFC20EF0FA
:107B8000CEC20DF0CDC20CF0CCC20BF0F3C212F09D
:107B9000F2C211F0F1C210F0F0C20FF050EC08F098
:107BA0000EC02DF00DC02CF00CC02BF00BC02AF035
:107BB0002DC00EF02CC00DF02BC00CF02AC00BF025
:107BC0008BC212F08AC211F089C210F088C20FF085
:107BD0004EEC08F084EC05F00EC075F00DC074F0AA
:107BE0000CC073F00BC072F0AF0E0E6E5D0E0D6E1A
:107BF0005A0E0C6E740E0B6E75C012F074C011F03C
:107C000073C010F072C00FF04AEC09F00EC075F0AE
:107C10000DC074F00CC073F00BC072F017C30EF0FF
:107C200016C30DF015C30CF014C30BF075C012F0A1
:107C300074C011F073C010F072C00FF050EC08F077
:107C40000EC017F30DC016F30CC015F30BC014F3E0
:107C50008BC20EF08AC20DF089C20CF088C20BF004
:107C60000BC312F00AC311F009C310F008C30FF0E0
:107C70004EEC08F084EC05F00EC075F00DC074F009
:107C80000CC073F00BC072F0060E0E6EBC0E0D6EC3
:107C90004C0E0C6E740E0B6E75C012F074C011F0A9
:107CA00073C010F072C00FF04AEC09F00EC075F00E
:107CB0000DC074F00CC073F00BC072F017C30EF05F
:107CC00016C30DF015C30CF014C30BF075C012F001
:107CD00074C011F073C010F072C00FF050EC08F0D7
:107CE0000EC017F30DC016F30CC015F30BC014F340
:107CF000CFC20EF0CEC20DF0CDC20CF0CCC20BF054
:107D0000F3C212F0F2C211F0F1C210F0F0C20FF0A3
:107D100050EC08F00EC02DF00DC02CF00CC02BF074
:107D20000BC02AF02DC00EF02CC00DF02BC00CF0B3
:107D30002AC00BF0FFC212F0FEC211F0FDC210F01B
:107D4000FCC20FF04EEC08F084EC05F00EC075F0AC
:107D50000DC074F00CC073F00BC072F0F00E0E6E1C
:107D6000A20E0D6E2F0E0C6E740E0B6E75C012F0FF
:107D700074C011F073C010F072C00FF04AEC09F03B
:107D80000EC075F00DC074F00CC073F00BC072F033
:107D900017C30EF016C30DF015C30CF014C30BF08F
:107DA00075C012F074C011F073C010F072C00FF003
:107DB00050EC08F00EC017F30DC016F30CC015F30D
:107DC0000BC014F3EBC20EF0EAC20DF0E9C20CF0E6
:107DD000E8C20BF00BC312F00AC311F009C310F094
:107DE00008C30FF04EEC08F084EC05F00EC075F0FF
:107DF0000DC074F00CC073F00BC072F0F90E0E6E73
:107E0000DB0E0D6E1E0E0C6E740E0B6E75C012F036
:107E100074C011F073C010F072C00FF04AEC09F09A
:107E20000EC075F00DC074F00CC073F00BC072F092
:107E300017C30EF016C30DF015C30CF014C30BF0EE
:107E400075C012F074C011F073C010F072C00FF062
:107E500050EC08F00EC017F30DC016F30CC015F36C
:107E60000BC014F3CBC20EF0CAC20DF0C9C20CF0A5
:107E7000C8C20BF08BC212F08AC211F089C210F096
:107E800088C20FF050EC08F00EC075F00DC074F011
:107E90000CC073F00BC072F0723F02D036827207D2
:107EA00075C00EF074C00DF073C00CF072C00BF012
:107EB000CFC212F0CEC211F0CDC210F0CCC20FF082
:107EC0004EEC08F084EC05F00EC075F00DC074F0B7
:107ED0000CC073F00BC072F0FE0E0E6E7F0E0D6EB6
:107EE0001C0E0C6E740E0B6E75C012F074C011F087
:107EF00073C010F072C00FF04AEC09F00EC075F0BC
:107F00000DC074F00CC073F00BC072F017C30EF00C
:107F100016C30DF015C30CF014C30BF075C012F0AE
:107F200074C011F073C010F072C00FF050EC08F084
:107F30000EC017F30DC016F30CC015F30BC014F3ED
:107F4000EBC20EF0EAC20DF0E9C20CF0E8C20BF091
:107F50008BC212F08AC211F089C210F088C20FF0F1
:107F600050EC08F00EC02DF00DC02CF00CC02BF022
:107F70000BC02AF02DC00EF02CC00DF02BC00CF061
:107F80002AC00BF023C212F022C211F021C210F05D
:107F900020C20FF04EEC08F00EC075F00DC074F06A
:107FA0000CC073F00BC072F075C00EF074C00DF011
:107FB00073C00CF072C00BF0CFC212F0CEC211F041
:107FC000CDC210F0CCC20FF04EEC08F084EC05F0FE
:107FD0000EC075F00DC074F00CC073F00BC072F0E1
:107FE000900E0E6EF90E0D6E0C6A740E0B6E75C04F
:107FF00012F074C011F073C010F072C00FF04AECB0
:1080000009F00EC075F00DC074F00CC073F00BC019
:1080100072F0E3C20EF0E2C20DF0E1C20CF0E0C279
:108020000BF075C012F074C011F073C010F072C084
:108030000FF04AEC09F00EC075F00DC074F00CC0E2
:1080400073F00BC072F017C30EF016C30DF015C31A
:108050000CF014C30BF075C012F074C011F073C0B3
:1080600010F072C00FF050EC08F00EC017F30DC006
:1080700016F30CC015F30BC014F38BC20EF08AC2BA
:108080000DF089C20CF088C20BF0CBC212F0CAC24C
:1080900011F0C9C210F0C8C20FF04EEC08F00EC0CB
:1080A00075F00DC074F00CC073F00BC072F0723F2D
:1080B00002D03682720775C00EF074C00DF073C026
:1080C0000CF072C00BF0CFC212F0CEC211F0CDC2D4
:1080D00010F0CCC20FF04EEC08F084EC05F00EC0AE
:1080E00075F00DC074F00CC073F00BC072F0FA0E96
:1080F0000E6EED0E0D6E6B0E0C6E730E0B6E75C06C
:1081000012F074C011F073C010F072C00FF04AEC9E
:1081100009F00EC075F00DC074F00CC073F00BC008
:1081200072F017C30EF016C30DF015C30CF014C394
:108130000BF075C012F074C011F073C010F072C073
:108140000FF050EC08F00EC017F30DC016F30CC082
:1081500015F30BC014F3F7C20EF0F6C20DF0F5C222
:108160000CF0F4C20BF0CFC212F0CEC211F0CDC2AF
:1081700010F0CCC20FF04EEC08F084EC05F00EC00D
:1081800075F00DC074F00CC073F00BC072F0950E5A
:108190000E6E290E0D6E660E0C6E730E0B6E75C094
:1081A00012F074C011F073C010F072C00FF04AECFE
:1081B00009F00EC075F00DC074F00CC073F00BC068
:1081C00072F017C30EF016C30DF015C30CF014C3F4
:1081D0000BF075C012F074C011F073C010F072C0D3
:1081E0000FF050EC08F00EC017F30DC016F30CC0E2
:1081F00015F30BC014F3CBC20EF0CAC20DF0C9C206
:108200000CF0C8C20BF08BC212F08AC211F089C206
:1082100010F088C20FF050EC08F00EC075F00DC0E1
:1082200074F00CC073F00BC072F0723F02D0368253
:10823000720775C00EF074C00DF073C00CF072C000
:108240000BF0CFC212F0CEC211F0CDC210F0CCC2F2
:108250000FF050EC08F084EC05F00EC075F00DC086
:1082600074F00CC073F00BC072F0190E0E6EC60ED7
:108270000D6E5D0E0C6E730E0B6E75C012F074C039
:1082800011F073C010F072C00FF04AEC09F00EC08C
:1082900075F00DC074F00CC073F00BC072F017C312
:1082A0000EF016C30DF015C30CF014C30BF075C01F
:1082B00012F074C011F073C010F072C00FF050ECE7
:1082C00008F00EC017F30DC016F30CC015F30BC069
:1082D00014F3EBC20EF0EAC20DF0E9C20CF0E8C2F2
:1082E0000BF0CFC212F0CEC211F0CDC210F0CCC252
:1082F0000FF04EEC08F00EC02DF00DC02CF00CC0AD
:108300002BF00BC02AF02DC00EF02CC00DF02BC0AE
:108310000CF02AC00BF0F7C212F0F6C211F0F5C251
:1083200010F0F4C20FF04EEC08F084EC05F00EC033
:1083300075F00DC074F00CC073F00BC072F0E20E5B
:108340000E6E3F0E0D6E5D0E0C6E730E0B6E75C0D5
:1083500012F074C011F073C010F072C00FF04AEC4C
:1083600009F00EC075F00DC074F00CC073F00BC0B6
:1083700072F017C30EF016C30DF015C30CF014C342
:108380000BF075C012F074C011F073C010F072C021
:108390000FF050EC08F00EC017F30DC016F30CC030
:1083A00015F30BC014F323C20EF022C20DF021C24C
:1083B0000CF020C20BF0CFC212F0CEC211F0CDC231
:1083C00010F0CCC20FF050EC08F00EC02DF00DC034
:1083D0002CF00CC02BF00BC02AF02DC00EF02CC0DE
:1083E0000DF02BC00CF02AC00BF0EBC212F0EAC269
:1083F00011F0E9C210F0E8C20FF050EC08F00EC026
:1084000075F00DC074F00CC073F00BC072F075C045
:108410000EF074C00DF073C00CF072C00BF08BC284
:1084200012F08AC211F089C210F088C20FF04EEC2F
:1084300008F084EC05F00EC075F00DC074F00CC0AF
:1084400073F00BC072F0E80E0E6E690E0D6E400EEA
:108450000C6E730E0B6E75C012F074C011F073C009
:1084600010F072C00FF04AEC09F00EC075F00DC0AC
:1084700074F00CC073F00BC072F0E3C20EF0E2C2F5
:108480000DF0E1C20CF0E0C20BF075C012F074C048
:1084900011F073C010F072C00FF04AEC09F00EC07A
:1084A00075F00DC074F00CC073F00BC072F017C300
:1084B0000EF016C30DF015C30CF014C30BF075C00D
:1084C00012F074C011F073C010F072C00FF04EECD7
:1084D00008F00EC017F30DC016F30CC015F30BC057
:1084E00014F323C20EF022C20DF021C20CF020C200
:1084F0000BF0CFC212F0CEC211F0CDC210F0CCC240
:108500000FF050EC08F00EC02DF00DC02CF00CC098
:108510002BF00BC02AF02DC00EF02CC00DF02BC09C
:108520000CF02AC00BF0EBC212F0EAC211F0E9C263
:1085300010F0E8C20FF050EC08F084EC05F00EC02B
:1085400075F00DC074F00CC073F00BC072F0DC0E4F
:108550000E6E120E0D6E390E0C6E730E0B6E75C014
:1085600012F074C011F073C010F072C00FF04AEC3A
:1085700009F00EC075F00DC074F00CC073F00BC0A4
:1085800072F0E3C20EF0E2C20DF0E1C20CF0E0C204
:108590000BF075C012F074C011F073C010F072C00F
:1085A0000FF04AEC09F00EC075F00DC074F00CC06D
:1085B00073F00BC072F017C30EF016C30DF015C3A5
:1085C0000CF014C30BF075C012F074C011F073C03E
:1085D00010F072C00FF04EEC08F00EC017F30DC093
:1085E00016F30CC015F30BC014F3CFC20EF0CEC2BD
:1085F0000DF0CDC20CF0CCC20BF0F3C212F0F2C2FF
:1086000011F0F1C210F0F0C20FF050EC08F084EC61
:1086100005F00EC075F00DC074F00CC073F00BC007
:1086200072F0110E0E6E8A0E0D6E2D0E0C6E730E04
:108630000B6E75C012F074C011F073C010F072C0F0
:108640000FF04AEC09F00EC075F00DC074F00CC0CC
:1086500073F00BC072F017C30EF016C30DF015C304
:108660000CF014C30BF075C012F074C011F073C09D
:1086700010F072C00FF050EC08F00EC017F30DC0F0
:1086800016F30CC015F30BC014F3EBC20EF0EAC2E4
:108690000DF0E9C20CF0E8C20BF0CFC212F0CEC26E
:1086A00011F0CDC210F0CCC20FF050EC08F00EC0AB
:1086B0002DF00DC02CF00CC02BF00BC02AF02DC0FB
:1086C0000EF02CC00DF02BC00CF02AC00BF023C212
:1086D00012F022C211F021C210F020C20FF04EECB5
:1086E00008F00EC075F00DC074F00CC073F00BC034
:1086F00072F075C00EF074C00DF073C00CF072C053
:108700000BF08BC212F08AC211F089C210F088C23D
:108710000FF050EC08F084EC05F00EC075F00DC0C1
:1087200074F00CC073F00BC072F0050E0E6E330EB9
:108730000D6E260E0C6E730E0B6E75C012F074C0AB
:1087400011F073C010F072C00FF04AEC09F00EC0C7
:1087500075F00DC074F00CC073F00BC072F0E3C282
:108760000EF0E2C20DF0E1C20CF0E0C20BF075C0F9
:1087700012F074C011F073C010F072C00FF04AEC28
:1087800009F00EC075F00DC074F00CC073F00BC092
:1087900072F017C30EF016C30DF015C30CF014C31E
:1087A0000BF075C012F074C011F073C010F072C0FD
:1087B0000FF050EC08F00EC017F30DC016F30CC00C
:1087C00015F30BC014F3CBC20EF0CAC20DF0C9C230
:1087D0000CF0C8C20BF023C212F022C211F021C269
:1087E00010F020C20FF04EEC08F00EC075F00DC076
:1087F00074F00CC073F00BC072F0723F02D036827E
:10880000720775C00EF074C00DF073C00CF072C02A
:108810000BF0CFC212F0CEC211F0CDC210F0CCC21C
:108820000FF04EEC08F084EC05F00EC075F00DC0B2
:1088300074F00CC073F00BC072F0A00E0E6E6E0ED2
:108840000D6E200E0C6E730E0B6E75C012F074C0A0
:1088500011F073C010F072C00FF04AEC09F00EC0B6
:1088600075F00DC074F00CC073F00BC072F0E7C26D
:108870000EF0E6C20DF0E5C20CF0E4C20BF075C0DC
:1088800012F074C011F073C010F072C00FF04AEC17
:1088900009F00EC075F00DC074F00CC073F00BC081
:1088A00072F017C30EF016C30DF015C30CF014C30D
:1088B0000BF075C012F074C011F073C010F072C0EC
:1088C0000FF050EC08F00EC017F30DC016F30CC0FB
:1088D00015F30BC014F38BC20EF08AC20DF089C2DF
:1088E0000CF088C20BF00BC312F00AC311F009C3DD
:1088F00010F008C30FF050EC08F084EC05F00EC047
:1089000075F00DC074F00CC073F00BC072F09E0EC9
:108910000E6E5F0E0D6E140E0C6E730E0B6E75C028
:1089200012F074C011F073C010F072C00FF04AEC76
:1089300009F00EC075F00DC074F00CC073F00BC0E0
:1089400072F017C30EF016C30DF015C30CF014C36C
:108950000BF075C012F074C011F073C010F072C04B
:108960000FF04EEC08F00EC017F30DC016F30CC05C
:1089700015F30BC014F3D3C20EF0D2C20DF0D1C266
:108980000CF0D0C20BF082EC05F00EC075F00DC0FB
:1089900074F00CC073F00BC072F0260E0E6E870ED2
:1089A0000D6E740E0C6E730E0B6E75C012F074C0EB
:1089B00011F073C010F072C00FF04AEC09F00EC055
:1089C0001BF30DC01AF30CC019F30BC018F34BC105
:1089D0000EF04AC10DF049C10CF048C10BF082EC19
:1089E00005F00EC075F00DC074F00CC073F00BC034
:1089F00072F0110E0E6E200E0D6E1E0E0C6E710EAC
:108A00000B6E75C012F074C011F073C010F072C01C
:108A10000FF04AEC09F00EC01FF30DC01EF30CC09E
:108A20001DF30BC01CF30E6A0D6A0C6A7F0E0B6EF1
:108A30001BC312F01AC311F019C310F018C30FF0C2
:108A40004EEC08F00EC02DF00DC02CF00CC02BF039
:108A50000BC02AF02DC00EF02CC00DF02BC00CF076
:108A60002AC00BF01FC312F01EC311F01DC310F07B
:108A70001CC30FF04EEC08F00EC075F00DC074F082
:108A80000CC073F00BC072F075C00EF074C00DF026
:108A900073C00CF072C00BF017C312F016C311F0C4
:108AA00015C310F014C30FF04AEC09F00EC02DF0FE
:108AB0000DC02CF00CC02BF00BC02AF0340E0E6E43
:108AC000FA0E0D6E0E0E0C6E790E0B6E2DC012F09E
:108AD0002CC011F02BC010F02AC00FF04AEC09F0A6
:108AE0000EC023F30DC022F30CC021F30BC020F302
:108AF0008BC20EF08AC20DF089C20CF088C20BF056
:108B000082EC05F00EC075F00DC074F00CC073F06F
:108B10000BC072F01C0E0E6E3F0E0D6E540E0C6EDE
:108B20007A0E0B6E75C012F074C011F073C010F0A5
:108B300072C00FF04AEC09F00EC075F00DC074F071
:108B40000CC073F00BC072F0A60E0E6E620E0D6EAE
:108B5000730E0C6E7E0E0B6E75C012F074C011F0A9
:108B600073C010F072C00FF050EC08F00EC027F385
:108B70000DC026F30CC025F30BC024F3EBC20EF09E
:108B8000EAC20DF0E9C20CF0E8C20BF08BC212F0A1
:108B90008AC211F089C210F088C20FF04EEC08F0C2
:108BA00082EC05F00EC075F00DC074F00CC073F0CF
:108BB0000BC072F0E90E0E6E270E0D6E1C0E0C6EC1
:108BC000780E0B6E75C012F074C011F073C010F007
:108BD00072C00FF04AEC09F00EC075F00DC074F0D1
:108BE0000CC073F00BC072F027C30EF026C30DF05B
:108BF00025C30CF024C30BF075C012F074C011F043
:108C000073C010F072C00FF050EC08F00EC027F3E4
:108C10000DC026F30CC025F30BC024F3EBC20EF0FD
:108C2000EAC20DF0E9C20CF0E8C20BF082EC05F0EC
:108C30000EC075F00DC074F00CC073F00BC072F074
:108C4000ED0E0E6E7F0E0D6E0C6A780E0B6E75C0FB
:108C500012F074C011F073C010F072C00FF04AEC43
:108C600009F00EC075F00DC074F00CC073F00BC0AD
:108C700072F027C30EF026C30DF025C30CF024C3F9
:108C80000BF075C012F074C011F073C010F072C018
:108C90000FF050EC08F00EC027F30DC026F30CC007
:108CA00025F30BC024F3FFC20EF0FEC20DF0FDC28F
:108CB0000CF0FCC20BF082EC05F00EC075F00DC09C
:108CC00074F00CC073F00BC072F0DC0E0E6E120E5E
:108CD0000D6E390E0C6E760E0B6E75C012F074C0F0
:108CE00011F073C010F072C00FF04AEC09F00EC022
:108CF00075F00DC074F00CC073F00BC072F027C398
:108D00000EF026C30DF025C30CF024C30BF075C084
:108D100012F074C011F073C010F072C00FF050EC7C
:108D200008F00EC027F30DC026F30CC025F30BC0CE
:108D300024F3EBC20EF0EAC20DF0E9C20CF0E8C277
:108D40000BF08BC212F08AC211F089C210F088C2F7
:108D50000FF050EC08F082EC05F00EC075F00DC07D
:108D600074F00CC073F00BC072F04C0E0E6EA80EB7
:108D70000D6E600E0C6E740E0B6E75C012F074C02A
:108D800011F073C010F072C00FF04AEC09F00EC081
:108D900075F00DC074F00CC073F00BC072F027C3F7
:108DA0000EF026C30DF025C30CF024C30BF075C0E4
:108DB00012F074C011F073C010F072C00FF050ECDC
:108DC00008F00EC027F30DC026F30CC025F30BC02E
:108DD00024F3EBC20EF0EAC20DF0E9C20CF0E8C2D7
:108DE0000BF023C212F022C211F021C210F020C2F7
:108DF0000FF04EEC08F082EC05F00EC075F00DC0DF
:108E000074F00CC073F00BC072F0060E0E6EB90E4B
:108E10000D6E0B0E0C6E740E0B6E75C012F074C0DE
:108E200011F073C010F072C00FF04AEC09F00EC0E0
:108E300075F00DC074F00CC073F00BC072F0E3C29B
:108E40000EF0E2C20DF0E1C20CF0E0C20BF075C012
:108E500012F074C011F073C010F072C00FF04AEC41
:108E600009F00EC075F00DC074F00CC073F00BC0AB
:108E700072F027C30EF026C30DF025C30CF024C3F7
:108E80000BF075C012F074C011F073C010F072C016
:108E90000FF050EC08F00EC027F30DC026F30CC005
:108EA00025F30BC024F3EBC20EF0EAC20DF0E9C2C9
:108EB0000CF0E8C20BF08BC212F08AC211F089C22A
:108EC00010F088C20FF04EEC08F00EC02DF00DC06F
:108ED0002CF00CC02BF00BC02AF02DC00EF02CC0D3
:108EE0000DF02BC00CF02AC00BF023C212F022C2EE
:108EF00011F021C210F020C20FF04EEC08F082EC0D
:108F000005F00EC075F00DC074F00CC073F00BC00E
:108F100072F04F0E0E6E3D0E0D6E520E0C6E730EF5
:108F20000B6E75C012F074C011F073C010F072C0F7
:108F30000FF04AEC09F00EC075F00DC074F00CC0D3
:108F400073F00BC072F0E3C20EF0E2C20DF0E1C2AA
:108F50000CF0E0C20BF075C012F074C011F073C0D9
:108F600010F072C00FF04AEC09F00EC075F00DC0A1
:108F700074F00CC073F00BC072F027C30EF026C360
:108F80000DF025C30CF024C30BF075C012F074C0B3
:108F900011F073C010F072C00FF050EC08F00EC06A
:108FA00027F30DC026F30CC025F30BC024F38BC2AE
:108FB0000EF08AC20DF089C20CF088C20BF023C2F9
:108FC00012F022C211F021C210F020C20FF04EECBC
:108FD00008F082EC05F00EC075F00DC074F00CC006
:108FE00073F00BC072F0AC0E0E6EC50E0D6E270E38
:108FF0000C6E730E0B6E75C012F074C011F073C05E
:1090000010F072C00FF04AEC09F00EC075F00DC000
:1090100074F00CC073F00BC072F0E3C20EF0E2C249
:109020000DF0E1C20CF0E0C20BF075C012F074C09C
:1090300011F073C010F072C00FF04AEC09F00EC0CE
:1090400075F00DC074F00CC073F00BC072F027C344
:109050000EF026C30DF025C30CF024C30BF075C031
:1090600012F074C011F073C010F072C00FF050EC29
:1090700008F00EC027F30DC026F30CC025F30BC07B
:1090800024F3CBC20EF0CAC20DF0C9C20CF0C8C2A4
:109090000BF082EC05F00EC075F00DC074F00CC042
:1090A00073F00BC072F0010E0E6E150E0D6E0E0EEB
:1090B0000C6E730E0B6E75C012F074C011F073C09D
:1090C00010F072C00FF04AEC09F00EC075F00DC040
:1090D00074F00CC073F00BC072F027C30EF026C3FF
:1090E0000DF025C30CF024C30BF075C012F074C052
:1090F00011F073C010F072C00FF04EEC08F00EC00B
:1091000027F30DC026F30CC025F30BC024F38BC24C
:109110000EF08AC20DF089C20CF088C20BF023C297
:1091200012F022C211F021C210F020C20FF050EC58
:1091300008F082EC05F00EC075F00DC074F00CC0A4
:1091400073F00BC072F07B0E0E6E690E0D6E0A0E80
:109150000C6E730E0B6E75C012F074C011F073C0FC
:1091600010F072C00FF04AEC09F00EC075F00DC09F
:1091700074F00CC073F00BC072F0E3C20EF0E2C2E8
:109180000DF0E1C20CF0E0C20BF075C012F074C03B
:1091900011F073C010F072C00FF04AEC09F00EC06D
:1091A00075F00DC074F00CC073F00BC072F027C3E3
:1091B0000EF026C30DF025C30CF024C30BF075C0D0
:1091C00012F074C011F073C010F072C00FF04EECCA
:1091D00008F00EC027F30DC026F30CC025F30BC01A
:1091E00024F307C30EF006C30DF005C30CF004C34F
:1091F0000BF08BC212F08AC211F089C210F088C243
:109200000FF04EEC08F082EC05F00EC075F00DC0CA
:1092100074F00CC073F00BC072F0380E0E6E9E0E20
:109220000D6E4F0E0C6E720E0B6E75C012F074C088
:1092300011F073C010F072C00FF04AEC09F00EC0CC
:1092400075F00DC074F00CC073F00BC072F027C342
:109250000EF026C30DF025C30CF024C30BF075C02F
:1092600012F074C011F073C010F072C00FF04EEC29
:1092700008F00EC027F30DC026F30CC025F30BC079
:1092800024F3F7C20EF0F6C20DF0F5C20CF0F4C2F2
:109290000BF082EC05F00EC075F00DC074F00CC040
:1092A00073F00BC072F0550E0E6E670E0D6E350E1C
:1092B0000C6E720E0B6E75C012F074C011F073C09C
:1092C00010F072C00FF04AEC09F00EC075F00DC03E
:1092D00074F00CC073F00BC072F027C30EF026C3FD
:1092E0000DF025C30CF024C30BF075C012F074C050
:1092F00011F073C010F072C00FF050EC08F00EC007
:1093000027F30DC026F30CC025F30BC024F3F3C2E2
:109310000EF0F2C20DF0F1C20CF0F0C20BF08BC2F5
:1093200012F08AC211F089C210F088C20FF04EEC20
:1093300008F082EC05F00EC075F00DC074F00CC0A2
:1093400073F00BC072F0B90E0E6E1C0E0D6E2F0E68
:109350000C6E720E0B6E75C012F074C011F073C0FB
:1093600010F072C00FF04AEC09F00EC075F00DC09D
:1093700074F00CC073F00BC072F027C30EF026C35C
:109380000DF025C30CF024C30BF075C012F074C0AF
:1093900011F073C010F072C00FF050EC08F00EC066
:1093A00027F30DC026F30CC025F30BC024F323C212
:1093B0000EF022C20DF021C20CF020C20BF082ECA4
:1093C00005F00EC075F00DC074F00CC073F00BC04A
:1093D00072F0AC0E0E6EC80E0D6E680E0C6E710E35
:1093E0000B6E75C012F074C011F073C010F072C033
:1093F0000FF04AEC09F00EC075F00DC074F00CC00F
:1094000073F00BC072F0E3C20EF0E2C20DF0E1C2E5
:109410000CF0E0C20BF075C012F074C011F073C014
:1094200010F072C00FF04AEC09F00EC075F00DC0DC
:1094300074F00CC073F00BC072F027C30EF026C39B
:109440000DF025C30CF024C30BF075C012F074C0EE
:1094500011F073C010F072C00FF04EEC08F00EC0A7
:1094600027F30DC026F30CC025F30BC024F3F3C281
:109470000EF0F2C20DF0F1C20CF0F0C20BF0FFC220
:1094800012F0FEC211F0FDC210F0FCC20FF04EEC63
:1094900008F082EC05F00EC075F00DC074F00CC041
:1094A00073F00BC072F0B40E0E6E010E0D6E580EFE
:1094B0000C6E710E0B6E75C012F074C011F073C09B
:1094C00010F072C00FF04AEC09F00EC075F00DC03C
:1094D00074F00CC073F00BC072F027C30EF026C3FB
:1094E0000DF025C30CF024C30BF075C012F074C04E
:1094F00011F073C010F072C00FF050EC08F00EC005
:1095000027F30DC026F30CC025F30BC024F3FFC2D4
:109510000EF0FEC20DF0FDC20CF0FCC20BF0EBC26F
:1095200012F0EAC211F0E9C210F0E8C20FF04EECFE
:1095300008F082EC05F00EC075F00DC074F00CC0A0
:1095400073F00BC072F0280E0E6E290E0D6E300EE9
:109550000C6E710E0B6E75C012F074C011F073C0FA
:1095600010F072C00FF04AEC09F00EC075F00DC09B
:1095700074F00CC073F00BC072F027C30EF026C35A
:109580000DF025C30CF024C30BF075C012F074C0AD
:1095900011F073C010F072C00FF04EEC08F00EC066
:1095A00027F30DC026F30CC025F30BC024F3EBC248
:1095B0000EF0EAC20DF0E9C20CF0E8C20BF023C2D3
:1095C00012F022C211F021C210F020C20FF050ECB4
:1095D00008F082EC05F00EC075F00DC074F00CC000
:1095E00073F00BC072F0490E0E6E100E0D6E2E0E43
:1095F0000C6E710E0B6E75C012F074C011F073C05A
:1096000010F072C00FF04AEC09F00EC075F00DC0FA
:1096100074F00CC073F00BC072F0E3C20EF0E2C243
:109620000DF0E1C20CF0E0C20BF075C012F074C096
:1096300011F073C010F072C00FF04AEC09F00EC0C8
:1096400075F00DC074F00CC073F00BC072F027C33E
:109650000EF026C30DF025C30CF024C30BF075C02B
:1096600012F074C011F073C010F072C00FF04EEC25
:1096700008F00EC027F30DC026F30CC025F30BC075
:1096800024F3EBC20EF0EAC20DF0E9C20CF0E8C21E
:109690000BF0FFC212F0FEC211F0FDC210F0FCC2CE
:1096A0000FF050EC08F082EC05F00EC075F00DC024
:1096B00074F00CC073F00BC072F0CD0E0E6EAC0ED9
:1096C0000D6E250E0C6E710E0B6E75C012F074C00F
:1096D00011F073C010F072C00FF04AEC09F00EC028
:1096E00075F00DC074F00CC073F00BC072F027C39E
:1096F0000EF026C30DF025C30CF024C30BF075C08B
:1097000012F074C011F073C010F072C00FF050EC82
:1097100008F00EC027F30DC026F30CC025F30BC0D4
:1097200024F3F3C20EF0F2C20DF0F1C20CF0F0C25D
:109730000BF082EC05F00EC075F00DC074F00CC09B
:1097400073F00BC072F0B50E0E6EFE0E0D6E160E9F
:109750000C6E710E0B6E75C012F074C011F073C0F8
:1097600010F072C00FF04AEC09F00EC075F00DC099
:1097700074F00CC073F00BC072F027C30EF026C358
:109780000DF025C30CF024C30BF075C012F074C0AB
:1097900011F073C010F072C00FF050EC08F00EC062
:1097A00027F30DC026F30CC025F30BC024F3EBC246
:1097B0000EF0EAC20DF0E9C20CF0E8C20BF023C2D1
:1097C00012F022C211F021C210F020C20FF04EECB4
:1097D00008F00EC02DF00DC02CF00CC02BF00BC00B
:1097E0002AF02DC00EF02CC00DF02BC00CF02AC0BA
:1097F0000BF08BC212F08AC211F089C210F088C23D
:109800000FF050EC08F082EC05F00EC075F00DC0C2
:1098100074F00CC073F00BC072F0BD0E0E6E370EFC
:109820000D6E060E0C6E710E0B6E75C012F074C0CC
:1098300011F073C010F072C00FF04AEC09F00EC0C6
:1098400075F00DC074F00CC073F00BC072F0E3C281
:109850000EF0E2C20DF0E1C20CF0E0C20BF075C0F8
:1098600012F074C011F073C010F072C00FF04AEC27
:1098700009F00EC075F00DC074F00CC073F00BC091
:1098800072F027C30EF026C30DF025C30CF024C3DD
:109890000BF075C012F074C011F073C010F072C0FC
:1098A0000FF050EC08F00EC027F30DC026F30CC0EB
:1098B00025F30BC024F3EBC20EF0EAC20DF0E9C2AF
:1098C0000CF0E8C20BF023C212F022C211F021C248
:1098D00010F020C20FF04EEC08F00EC02DF00DC0BD
:1098E0002CF00CC02BF00BC02AF02DC00EF02CC0B9
:1098F0000DF02BC00CF02AC00BF08BC212F08AC204
:1099000011F089C210F088C20FF04EEC08F082EC22
:1099100005F00EC075F00DC074F00CC073F00BC0F4
:1099200072F0DE0E0E6E1E0E0D6E040E0C6E710EBB
:109930000B6E75C012F074C011F073C010F072C0DD
:109940000FF04AEC09F00EC075F00DC074F00CC0B9
:1099500073F00BC072F0E3C20EF0E2C20DF0E1C290
:109960000CF0E0C20BF075C012F074C011F073C0BF
:1099700010F072C00FF04AEC09F00EC075F00DC087
:1099800074F00CC073F00BC072F027C30EF026C346
:109990000DF025C30CF024C30BF075C012F074C099
:1099A00011F073C010F072C00FF04EEC08F00EC052
:1099B00027F30DC026F30CC025F30BC024F323C2FC
:1099C0000EF022C20DF021C20CF020C20BF0CBC26F
:1099D00012F0CAC211F0C9C210F0C8C20FF050ECA8
:1099E00008F082EC05F00EC075F00DC074F00CC0EC
:1099F00073F00BC072F06A0E0E6EF70E0D6E2B0E2A
:109A00000C6E700E0B6E75C012F074C011F073C046
:109A100010F072C00FF04AEC09F00EC075F00DC0E6
:109A200074F00CC073F00BC072F0E3C20EF0E2C22F
:109A30000DF0E1C20CF0E0C20BF075C012F074C082
:109A400011F073C010F072C00FF04AEC09F00EC0B4
:109A500075F00DC074F00CC073F00BC072F027C32A
:109A60000EF026C30DF025C30CF024C30BF075C017
:109A700012F074C011F073C010F072C00FF050EC0F
:109A800008F00EC027F30DC026F30CC025F30BC061
:109A900024F3FFC20EF0FEC20DF0FDC20CF0FCC2BA
:109AA0000BF023C212F022C211F021C210F020C22A
:109AB0000FF04EEC08F082EC05F00EC075F00DC012
:109AC00074F00CC073F00BC072F0F70E0E6ECC0E7B
:109AD0000D6E120E0C6E700E0B6E75C012F074C00F
:109AE00011F073C010F072C00FF04AEC09F00EC014
:109AF00075F00DC074F00CC073F00BC072F0E3C2CF
:109B00000EF0E2C20DF0E1C20CF0E0C20BF075C045
:109B100012F074C011F073C010F072C00FF04AEC74
:109B200009F00EC075F00DC074F00CC073F00BC0DE
:109B300072F027C30EF026C30DF025C30CF024C32A
:109B40000BF075C012F074C011F073C010F072C049
:109B50000FF050EC08F00EC027F30DC026F30CC038
:109B600025F30BC024F3F7C20EF0F6C20DF0F5C2D8
:109B70000CF0F4C20BF0EBC212F0EAC211F0E9C231
:109B800010F0E8C20FF04EEC08F082EC05F00EC0C9
:109B900075F00DC074F00CC073F00BC072F07B0E4A
:109BA0000E6E690E0D6E0A0E0C6E700E0B6E75C089
:109BB00012F074C011F073C010F072C00FF04AECD4
:109BC00009F00EC075F00DC074F00CC073F00BC03E
:109BD00072F027C30EF026C30DF025C30CF024C38A
:109BE0000BF075C012F074C011F073C010F072C0A9
:109BF0000FF04EEC08F00EC027F30DC026F30CC09A
:109C000025F30BC024F38BC20EF08AC20DF089C27B
:109C10000CF088C20BF0CBC212F0CAC211F0C9C25C
:109C200010F0C8C20FF050EC08F082EC05F00EC046
:109C300075F00DC074F00CC073F00BC072F0820EA2
:109C40000E6EA80E0D6E7B0E0C6E6F0E0B6E75C039
:109C500012F074C011F073C010F072C00FF04AEC33
:109C600009F00EC075F00DC074F00CC073F00BC09D
:109C700072F027C30EF026C30DF025C30CF024C3E9
:109C80000BF075C012F074C011F073C010F072C008
:109C90000FF04EEC08F00EC027F30DC026F30CC0F9
:109CA00025F30BC024F3CFC20EF0CEC20DF0CDC20F
:109CB0000CF0CCC20BF0CBC212F0CAC211F0C9C278
:109CC00010F0C8C20FF04EEC08F00EC075F00DC0D9
:109CD00074F00CC073F00BC072F075C00EF074C05D
:109CE0000DF073C00CF0723D02D0368272510B6ED3
:109CF00082EC05F00EC075F00DC074F00CC073F06E
:109D00000BC072F0070E0E6E450E0D6E730E0C6ECC
:109D10006F0E0B6E75C012F074C011F073C010F0AE
:109D200072C00FF04AEC09F00EC075F00DC074F06F
:109D30000CC073F00BC072F027C30EF026C30DF0F9
:109D400025C30CF024C30BF075C012F074C011F0E1
:109D500073C010F072C00FF04EEC08F00EC027F385
:109D60000DC026F30CC025F30BC024F3FFC20EF088
:109D7000FEC20DF0FDC20CF0FCC20BF023C212F0CB
:109D800022C211F021C210F020C20FF050EC08F0F6
:109D900082EC05F00EC075F00DC074F00CC073F0CD
:109DA0000BC072F0070E0E6E450E0D6E730E0C6E2C
:109DB0006F0E0B6E75C012F074C011F073C010F00E
:109DC00072C00FF04AEC09F00EC075F00DC074F0CF
:109DD0000CC073F00BC072F0E3C20EF0E2C20DF0E3
:109DE000E1C20CF0E0C20BF075C012F074C011F0CB
:109DF00073C010F072C00FF04AEC09F00EC075F09D
:109E00000DC074F00CC073F00BC072F027C30EF0DD
:109E100026C30DF025C30CF024C30BF075C012F05F
:109E200074C011F073C010F072C00FF04EEC08F067
:109E30000EC027F30DC026F30CC025F30BC024F38E
:109E4000CBC20EF0CAC20DF0C9C20CF0C8C20BF0F2
:109E500023C212F022C211F021C210F020C20FF072
:109E60004EEC08F00EC075F00DC074F00CC073F02D
:109E70000BC072F075C00EF074C00DF073C00CF022
:109E8000723D02D0368272510B6E82EC05F00EC02C
:109E900075F00DC074F00CC073F00BC072F0930E2F
:109EA0000E6E1A0E0D6E5A0E0C6E6F0E0B6E75C086
:109EB00012F074C011F073C010F072C00FF04AECD1
:109EC00009F00EC075F00DC074F00CC073F00BC03B
:109ED00072F0E7C20EF0E6C20DF0E5C20CF0E4C28B
:109EE0000BF075C012F074C011F073C010F072C0A6
:109EF0000FF04AEC09F00EC075F00DC074F00CC004
:109F000073F00BC072F027C30EF026C30DF025C30B
:109F10000CF024C30BF075C012F074C011F073C0C4
:109F200010F072C00FF050EC08F00EC027F30DC017
:109F300026F30CC025F30BC024F3CFC20EF0CEC223
:109F40000DF0CDC20CF0CCC20BF0CBC212F0CAC2E5
:109F500011F0C9C210F0C8C20FF04EEC08F00EC0EC
:109F600075F00DC074F00CC073F00BC072F0723F4E
:109F700002D03682720775C00EF074C00DF073C047
:109F80000CF072C00BF08BC212F08AC211F089C2C1
:109F900010F088C20FF050EC08F082EC05F00EC013
:109FA00075F00DC074F00CC073F00BC072F0200E91
:109FB0000E6EF00E0D6E400E0C6E6F0E0B6E75C0B9
:109FC00012F074C011F073C010F072C00FF04AECC0
:109FD00009F00EC075F00DC074F00CC073F00BC02A
:109FE00072F027C30EF026C30DF025C30CF024C376
:109FF0000BF075C012F074C011F073C010F072C095
:10A000000FF04EEC08F00EC027F30DC026F30CC085
:10A0100025F30BC024F3F3C20EF0F2C20DF0F1C22F
:10A020000CF0F0C20BF023C212F022C211F021C2D8
:10A0300010F020C20FF04EEC08F00EC02DF00DC055
:10A040002CF00CC02BF00BC02AF02DC00EF02CC051
:10A050000DF02BC00CF02AC00BF08BC212F08AC29C
:10A0600011F089C210F088C20FF04EEC08F082ECBB
:10A0700005F00EC075F00DC074F00CC073F00BC08D
:10A0800072F0300E0E6E620E0D6E1F0E0C6E6F0EA5
:10A090000B6E75C012F074C011F073C010F072C076
:10A0A0000FF04AEC09F00EC075F00DC074F00CC052
:10A0B00073F00BC072F0E3C20EF0E2C20DF0E1C229
:10A0C0000CF0E0C20BF075C012F074C011F073C058
:10A0D00010F072C00FF04AEC09F00EC075F00DC020
:10A0E00074F00CC073F00BC072F027C30EF026C3DF
:10A0F0000DF025C30CF024C30BF075C012F074C032
:10A1000011F073C010F072C00FF050EC08F00EC0E8
:10A1100027F30DC026F30CC025F30BC024F3340E37
:10A120000E6EFA0E0D6E0E0E0C6E790E0B6E27C3B0
:10A1300012F026C311F025C310F024C30FF04AEC2F
:10A1400009F00EC01BF20DC01AF20CC019F20BC0C0
:10A1500018F21200010E0101136F8CC10EF08BC1B9
:10A160000DF08AC10CF089C10BF0126A116A106AF5
:10A170000F6A12EC08F0336E90C10EF08FC10DF033
:10A180008EC10CF08DC10BF0126A116A106A0F6A51
:10A1900012EC08F0331294C10EF093C10DF092C18D
:10A1A0000CF091C10BF0126A116A106A0F6A12EC7E
:10A1B00008F03312000103E0FF0E0101136F0001EC
:10A1C0008CC198F18BC197F18AC196F10101969FDC
:10A1D00089C195F190C19CF18FC19BF18EC19AF11B
:10A1E0009A9F8DC199F194C1A0F193C19FF192C141
:10A1F0009EF19E9F91C19DF1126A116A700E106EC0
:10A20000840E0F6EA0C10EF09FC10DF09EC10CF028
:10A210009DC10BF0E2EC08F00EC05CF10DC05BF1EB
:10A220000CC05AF10BC059F15CC10EF05BC10DF0CE
:10A230005AC10CF059C10BF09CC112F09BC111F036
:10A240009AC110F099C10FF050EC08F00EC05CF10B
:10A250000DC05BF10CC05AF10BC059F1126A116AC2
:10A26000700E106E840E0F6E5CC10EF05BC10DF0AF
:10A270005AC10CF059C10BF0E2EC08F00EC05CF1D1
:10A280000DC05BF10CC05AF10BC059F15CC10EF06E
:10A290005BC10DF05AC10CF059C10BF098C112F01E
:10A2A00097C111F096C110F095C10FF050EC08F075
:10A2B0000EC05CF10DC05BF10CC05AF10BC059F13E
:10A2C0001351EAEC09F05CC112F05BC111F05AC104
:10A2D00010F059C10FF04AEC09F00EC0A4F10DC006
:10A2E000A3F10CC0A2F10BC0A1F100011200366A6B
:10A2F00021C122F12FC133F12EC132F12DC131F133
:10A300002CC130F10101436B426B416B406B030E7A
:10A31000215D000109E20C0E01012125226F3007A9
:10A32000000E315B325B335B000133C11AF032C186
:10A3300019F031C118F030C117F0226A216A206A81
:10A34000640E1F6E30EC03F01AC037F119C036F1FD
:10A3500018C035F117C034F1010134510208406FC3
:10A36000000E3555416F000E3655426F000E3755C1
:10A37000436F37C11AF036C119F035C118F034C136
:10A3800017F0226A216A206A040E1F6E30EC03F077
:10A390001AC058F119C057F118C056F117C055F13D
:10A3A0005551402756514123575142235851432379
:10A3B00033C10EF032C10DF031C10CF030C10BF0E1
:10A3C000EEEC09F0126AA00E116E360E106E870EBA
:10A3D0000F6E4AEC09F00EC05CF10DC05BF10CC0D1
:10A3E0005AF10BC059F1900E126E700E116E290EBB
:10A3F000106E920E0F6E5CC10EF05BC10DF05AC173
:10A400000CF059C10BF04EEC08F09AEC09F00BC0BF
:10A410004FF10CC04EF10DC04DF14C6F222B22516B
:10A42000EAEC09F0010E126ECD0E116E740E106E74
:10A43000830E0F6E4AEC09F00EC05CF10DC05BF1AB
:10A440000CC05AF10BC059F15CC10EF05BC10DF0AC
:10A450005AC10CF059C10BF09AEC09F00BC053F142
:10A460000CC052F10DC051F1506F4C5140250B6E94
:10A470004D5141210C6E4E5142210D6E4F514321E1
:10A480000E6EEEEC09F00EC070F10DC06FF10CC055
:10A490006EF10BC06DF153C10EF052C10DF051C100
:10A4A0000CF050C10BF0EEEC09F070C112F06FC16E
:10A4B00011F06EC110F06DC10FF050EC08F00EC03D
:10A4C00070F10DC06FF10CC06EF10BC06DF170C179
:10A4D0000EF06FC10DF06EC10CF06DC10BF027C115
:10A4E00012F026C111F025C110F024C10FF050EC7C
:10A4F00008F00EC070F10DC06FF10CC06EF10BC012
:10A500006DF1126A116A106A7E0E0F6E70C10EF044
:10A510006FC10DF06EC10CF06DC10BF04EEC08F088
:10A520000EC070F10DC06FF10CC06EF10BC06DF17B
:10A53000400E366E0001120045BA83D121C123F1CD
:10A5400027C12BF126C12AF125C129F124C128F107
:10A55000458ACDDE70C174F16FC173F16EC172F1C5
:10A560006DC171F1010E0101216F276B266B256B07
:10A57000246B0001BCDE126AAD0E116E0E0E106E61
:10A580008E0E0F6E70C10EF06FC10DF06EC10CF02B
:10A590006DC10BF0E2EC08F00EC07CF10DC07BF158
:10A5A0000CC07AF10BC079F18E0E0E6E820E0D6E1C
:10A5B000580E0C6E6F0E0B6E7CC112F07BC111F049
:10A5C0007AC110F079C10FF04AEC09F00EC05CF1CD
:10A5D0000DC05BF10CC05AF10BC059F11A0E0E6E92
:10A5E000F80E0D6E510E0C6E7A0E0B6E5CC112F0F1
:10A5F0005BC111F05AC110F059C10FF050EC08F0D6
:10A600000EC05CF10DC05BF10CC05AF10BC059F1EA
:10A610005CC10EF05BC10DF05AC10CF059C10BF0DA
:10A620007CC112F07BC111F07AC110F079C10FF03A
:10A630004AEC09F00EC05CF10DC05BF10CC05AF1A0
:10A640000BC059F1920E0E6EAC0E0D6E540E0C6EC8
:10A65000810E0B6E5CC112F05BC111F05AC110F09B
:10A6600059C10FF050EC08F00EC080F10DC07FF121
:10A670000CC07EF10BC07DF12FC10EF02EC10DF08C
:10A680002DC10CF02CC10BF0EEEC09F0126A800E1B
:10A69000116E6D0E106E890E0F6E4EEC08F00EC02E
:10A6A0005CF10DC05BF10CC05AF10BC059F1126A9C
:10A6B000116A480E106E850E0F6E5CC10EF05BC104
:10A6C0000DF05AC10CF059C10BF0E2EC08F00EC0CD
:10A6D0005CF10DC05BF10CC05AF10BC059F17CC1AB
:10A6E0000EF07BC10DF07AC10CF079C10BF05CC1AA
:10A6F00012F05BC111F05AC110F059C10FF04EECCD
:10A7000008F00EC05CF10DC05BF10CC05AF10BC03B
:10A7100059F10E6A0D6A160E0C6E8A0E0B6E5CC134
:10A7200012F05BC111F05AC110F059C10FF04AECA0
:10A7300009F00EC084F10DC083F10CC082F10BC092
:10A7400081F10E6A0D6A400E0C6E830E0B6E80C195
:10A7500012F07FC111F07EC110F07DC10FF04EEC00
:10A7600008F00EC047F10DC046F10CC045F10BC01A
:10A7700044F147C10EF046C10DF045C10CF044C193
:10A780000BF084C112F083C111F082C110F081C1BD
:10A790000FF04EEC08F00EC047F10DC046F10CC0B2
:10A7A00045F10BC044F174C10EF073C10DF072C1DC
:10A7B0000CF071C10BF070C112F06FC111F06EC1DD
:10A7C00010F06DC10FF04EEC08F00EC05CF10DC042
:10A7D0005BF10CC05AF10BC059F1DC0E0E6E920EFB
:10A7E0000D6E060E0C6E7B0E0B6E5CC112F05BC123
:10A7F00011F05AC110F059C10FF04AEC09F00EC027
:10A800005CF10DC05BF10CC05AF10BC059F15CC199
:10A810000EF05BC10DF05AC10CF059C10BF047C1ED
:10A8200012F046C111F045C110F044C10FF04EECDA
:10A8300008F00EC0A8F10DC0A7F10CC0A6F10BC026
:10A84000A5F1B70E0E6E590E0D6E0C6A7F0E0B6ED3
:10A85000B0C112F0AFC111F0AEC110F0ADC10FF038
:10A860004AEC09F00EC05CF10DC05BF10CC05AF16E
:10A870000BC059F15CC10EF05BC10DF05AC10CF078
:10A8800059C10BF0A8C112F0A7C111F0A6C110F078
:10A89000A5C10FF050EC08F00EC0ACF10DC0ABF14B
:10A8A0000CC0AAF10BC0A9F10E6A0D6A400E0C6E25
:10A8B000830E0B6EACC112F0ABC111F0AAC110F047
:10A8C000A9C10FF09EEC07F0010819E0126A116AA5
:10A8D000400E106E830E0F6EACC10EF0ABC10DF0CA
:10A8E000AAC10CF0A9C10BF04EEC08F00EC0ACF1FF
:10A8F0000DC0ABF10CC0AAF10BC0A9F1D5D7010175
:10A90000A95300011FE0D8960101AAAFD886000123
:10A9100019E40E6A0D6A400E0C6E830E0B6EACC10C
:10A9200012F0ABC111F0AAC110F0A9C10FF050ECA8
:10A9300008F00EC0ACF10DC0ABF10CC0AAF10BC019
:10A94000A9F1DDD7ACC1A4F1ABC1A3F1AAC1A2F1B9
:10A95000A9C1A1F123C121F12BC127F12AC126F1FF
:10A9600029C125F128C124F174C170F173C16FF1BF
:10A9700072C16EF171C16DF1120045BC25D0B8C134
:10A980000EF0B7C10DF0B6C10CF0B5C10BF082EC02
:10A9900005F00EC0B4F10DC0B3F10CC0B2F10BC0A4
:10A9A000B1F1B8C10EF0B7C10DF0B6C10CF0B5C130
:10A9B0000BF084EC05F00EC0BCF10DC0BBF10CC077
:10A9C000BAF10BC0B9F1458CC4C10EF0C3C10DF092
:10A9D000C2C10CF0C1C10BF084EC05F00EC0C0F197
:10A9E0000DC0BFF10CC0BEF10BC0BDF1C4C10EF073
:10A9F000C3C10DF0C2C10CF0C1C10BF082EC05F077
:10AA00000EC0C8F10DC0C7F10CC0C6F10BC0C5F136
:10AA1000A4C10EF0A3C10DF0A2C10CF0A1C10BF0B6
:10AA200084EC05F00EC0CCF10DC0CBF10CC0CAF126
:10AA30000BC0C9F1A4C10EF0A3C10DF0A2C10CF06E
:10AA4000A1C10BF082EC05F00EC0D0F10DC0CFF12A
:10AA50000CC0CEF10BC0CDF1C0C10EF0BFC10DF0E6
:10AA6000BEC10CF0BDC10BF0BCC112F0BBC111F0F6
:10AA7000BAC110F0B9C10FF04AEC09F00EC05CF198
:10AA80000DC05BF10CC05AF10BC059F1C8C10EF0FA
:10AA9000C7C10DF0C6C10CF0C5C10BF0B4C112F0B6
:10AAA000B3C111F0B2C110F0B1C10FF04AEC09F01E
:10AAB0000EC060F10DC05FF10CC05EF10BC05DF126
:10AAC00060C10EF05FC10DF05EC10CF05DC10BF016
:10AAD000D0C112F0CFC111F0CEC110F0CDC10FF036
:10AAE0004AEC09F00EC060F10DC05FF10CC05EF1E0
:10AAF0000BC05DF15CC10EF05BC10DF05AC10CF0F2
:10AB000059C10BF060C112F05FC111F05EC110F0CD
:10AB10005DC10FF050EC08F00EC0D4F10DC0D3F1C0
:10AB20000CC0D2F10BC0D1F1D4C10EF0D3C10DF0E5
:10AB3000D2C10CF0D1C10BF0FBEC03F00EC0D8F188
:10AB40000DC0D7F10CC0D6F10BC0D5F1D8C10EF0B5
:10AB5000D7C10DF0D6C10CF0D5C10BF082EC05F0D9
:10AB60000EC0DCF10DC0DBF10CC0DAF10BC0D9F185
:10AB7000B4C10EF0B3C10DF0B2C10CF0B1C10BF015
:10AB8000DCC112F0DBC111F0DAC110F0D9C10FF055
:10AB90004AEC09F00EC03BF10DC03AF10CC039F19E
:10ABA0000BC038F1010139BF0AD0FF0E3B5DE60E44
:10ABB0003A595B0E39595D0E3859000108E201011E
:10ABC0003B69E60E3A6F5B0E396F5D0E386F000120
:10ABD000BCC10EF0BBC10DF0BAC10CF0B9C10BF095
:10ABE000D4C112F0D3C111F0D2C110F0D1C10FF015
:10ABF0004AEC09F00EC05CF10DC05BF10CC05AF1DB
:10AC00000BC059F1C0C10EF0BFC10DF0BEC10CF0B8
:10AC1000BDC10BF05CC112F05BC111F05AC110F064
:10AC200059C10FF04EEC08F00EC05CF10DC05BF1A5
:10AC30000CC05AF10BC059F15CC10EF05BC10DF0B4
:10AC40005AC10CF059C10BF03BC112F03AC111F0DE
:10AC500039C110F038C10FF0E2EC08F0EEEC03F06F
:10AC60000EC0E4F10DC0E3F10CC0E2F10BC0E1F164
:10AC70000E6A0D6A0C6A0B6ACCC112F0CBC111F0DE
:10AC8000CAC110F0C9C10FF09EEC07F001081AE02C
:10AC9000DA0E0E6E0F0E0D6E490E0C6E810E0B6EDF
:10ACA000E4C112F0E3C111F0E2C110F0E1C10FF014
:10ACB0004EEC08F00EC0E4F10DC0E3F10CC0E2F17F
:10ACC0000BC0E1F1120045BE1200458E126AAD0EB6
:10ACD000116E0E0E106E8E0E0F6E70C10EF06FC1E3
:10ACE0000DF06EC10CF06DC10BF0E2EC08F00EC07F
:10ACF0007CF10DC07BF10CC07AF10BC079F1860EAE
:10AD00000E6E3D0E0D6EED0E0C6E750E0B6E7CC153
:10AD100012F07BC111F07AC110F079C10FF04AEC4A
:10AD200009F00EC05CF10DC05BF10CC05AF10BC014
:10AD300059F1CA0E0E6E540E0D6E410E0C6E770E4A
:10AD40000B6E5CC112F05BC111F05AC110F059C119
:10AD50000FF050EC08F00EC05CF10DC05BF10CC0C0
:10AD60005AF10BC059F15CC10EF05BC10DF05AC134
:10AD70000CF059C10BF07CC112F07BC111F07AC10B
:10AD800010F079C10FF04AEC09F00EC05CF10DC073
:10AD90005BF10CC05AF10BC059F1480E0E6E610EFA
:10ADA0000D6E3B0E0C6E840E0B6E5CC112F05BC11F
:10ADB00011F05AC110F059C10FF050EC08F00EC05C
:10ADC0005CF10DC05BF10CC05AF10BC059F15CC1D4
:10ADD0000EF05BC10DF05AC10CF059C10BF07CC1F3
:10ADE00012F07BC111F07AC110F079C10FF04AEC7A
:10ADF00009F00EC04BF10DC04AF10CC049F10BC077
:10AE000048F1126A116A610E106E8A0E0F6E4BC104
:10AE10000EF04AC10DF049C10CF048C10BF0E2EC54
:10AE200008F00EC05CF10DC05BF10CC05AF10BC014
:10AE300059F14D0E0E6E9E0E0D6E3B0E0C6E830E76
:10AE40000B6E5CC112F05BC111F05AC110F059C118
:10AE50000FF04EEC08F00EC063F20DC062F20CC0B1
:10AE600061F20BC060F2350E0E6EFA0E0D6E0E0E14
:10AE70000C6E790E0B6E63C212F062C211F061C2E9
:10AE800010F060C20FF04AEC09F00EC067F20DC07E
:10AE900066F20CC065F20BC064F2120001011431BD
:10AEA000000107E3D896010114A1D8860001D8A6B5
:10AEB0005CD001011481000106DF63C20EF062C2A2
:10AEC0000DF061C20CF060C20BF06BC212F06AC2EE
:10AED00011F069C210F068C20FF050EC08F00EC01B
:10AEE0005CF10DC05BF10CC05AF10BC059F1340E8E
:10AEF0000E6EFA0E0D6E0E0E0C6E790E0B6E5CC1A0
:10AF000012F05BC111F05AC110F059C10FF04AECB8
:10AF100009F00EC077F20DC076F20CC075F20BC0CE
:10AF200074F277C20EF076C20DF075C20CF074C2E6
:10AF30000BF084EC05F00EC073F20DC072F20CC081
:10AF400071F20BC070F277C20EF076C20DF075C2CE
:10AF50000CF074C20BF082EC05F00EC06FF20DC065
:10AF60006EF20CC06DF20BC06CF2C4C10EF0C3C126
:10AF70000DF0C2C10CF0C1C10BF082EC05F00EC0A7
:10AF8000C8F10DC0C7F10CC0C6F10BC0C5F1C4C1FA
:10AF90000EF0C3C10DF0C2C10CF0C1C10BF084ECC6
:10AFA00005F00EC0C0F10DC0BFF10CC0BEF10BC06A
:10AFB000BDF1C8C15CF1C7C15BF1C6C15AF1010165
:10AFC0005A9FC5C159F15ABF0AD0FF0E5C5DE60E0B
:10AFD0005B595B0E5A595D0E5959000108E2010197
:10AFE000C869E60EC76F5B0EC66F5D0EC56F0001C8
:10AFF000C0C10EF0BFC10DF0BEC10CF0BDC10BF061
:10B00000C8C112F0C7C111F0C6C110F0C5C10FF020
:10B01000E2EC08F00EC07BF20DC07AF20CC079F2BF
:10B020000BC078F2A4C10EF0A3C10DF0A2C10CF0C8
:10B03000A1C10BF082EC05F00EC0D0F10DC0CFF134
:10B040000CC0CEF10BC0CDF1A4C10EF0A3C10DF028
:10B05000A2C10CF0A1C10BF084EC05F00EC0CCF144
:10B060000DC0CBF10CC0CAF10BC0C9F1C0C10EF0CC
:10B07000BFC10DF0BEC10CF0BDC10BF06FC212F02C
:10B080006EC211F06DC210F06CC20FF04AEC09F004
:10B090000EC05CF10DC05BF10CC05AF10BC059F150
:10B0A000C8C10EF0C7C10DF0C6C10CF0C5C10BF090
:10B0B00073C212F072C211F071C210F070C20FF0C0
:10B0C0004AEC09F00EC060F10DC05FF10CC05EF1FA
:10B0D0000BC05DF160C10EF05FC10DF05EC10CF000
:10B0E0005DC10BF0CCC112F0CBC111F0CAC110F0A0
:10B0F000C9C10FF04AEC09F00EC060F10DC05FF15C
:10B100000CC05EF10BC05DF11CC10EF01BC10DF057
:10B110001AC10CF019C10BF0EEEC09F060C112F08D
:10B120005FC111F05EC110F05DC10FF04AEC09F093
:10B130000EC060F10DC05FF10CC05EF10BC05DF19F
:10B140005CC10EF05BC10DF05AC10CF059C10BF09F
:10B1500060C112F05FC111F05EC110F05DC10FF06F
:10B160004EEC08F0FBEC03F00EC0D8F10DC0D7F1A7
:10B170000CC0D6F10BC0D5F1CCC10EF0CBC10DF097
:10B18000CAC10CF0C9C10BF06FC212F06EC211F04F
:10B190006DC210F06CC20FF04AEC09F00EC05CF109
:10B1A0000DC05BF10CC05AF10BC059F17BC20EF01F
:10B1B0007AC20DF079C20CF078C20BF073C212F0B3
:10B1C00072C211F071C210F070C20FF04AEC09F0B7
:10B1D0000EC060F10DC05FF10CC05EF10BC05DF1FF
:10B1E0001CC10EF01BC10DF01AC10CF019C10BF0FF
:10B1F000EEEC09F060C112F05FC111F05EC110F019
:10B200005DC10FF04AEC09F00EC060F10DC05FF1B6
:10B210000CC05EF10BC05DF15CC10EF05BC10DF0C6
:10B220005AC10CF059C10BF060C112F05FC111F0AE
:10B230005EC110F05DC10FF050EC08F00EC03FF1A0
:10B240000DC03EF10CC03DF10BC03CF13FC10EF012
:10B250003EC10DF03DC10CF03CC10BF0D0C112F06D
:10B26000CFC111F0CEC110F0CDC10FF0E2EC08F06B
:10B270002CEC04F00EC0E4F10DC0E3F10CC0E2F1DF
:10B280000BC0E1F10101CD53000120E0D89601018E
:10B29000CEAFD88600011AE4DC0E0E6E0F0E0D6ED6
:10B2A000490E0C6E800E0B6EE4C112F0E3C111F07A
:10B2B000E2C110F0E1C10FF050EC08F00EC0E4F173
:10B2C0000DC0E3F10CC0E2F10BC0E1F1DA0E0E6E3D
:10B2D0000F0E0D6E490E0C6E810E0B6EE4C112F056
:10B2E000E3C111F0E2C110F0E1C10FF09EEC07F0F4
:10B2F00001081AE0DA0E126E0F0E116E490E106E72
:10B30000810E0F6EE4C10EF0E3C10DF0E2C10CF04E
:10B31000E1C10BF04EEC08F00EC0E4F10DC0E3F11A
:10B320000CC0E2F10BC0E1F10101E153000120E0AA
:10B33000D8960101E2AFD88600011AE4DA0E0E6E4B
:10B340000F0E0D6E490E0C6E810E0B6EE4C112F0E5
:10B35000E3C111F0E2C110F0E1C10FF050EC08F0D0
:10B360000EC0E4F10DC0E3F10CC0E2F10BC0E1F15D
:10B370001200126A116A700E106E820E0F6EF0C10A
:10B380000EF0EFC10DF0EEC10CF0EDC10BF0E2ECF0
:10B3900008F00EC05CF10DC05BF10CC05AF10BC09F
:10B3A00059F1ECC10EF0EBC10DF0EAC10CF0E9C1AE
:10B3B0000BF05CC112F05BC111F05AC110F059C121
:10B3C0000FF050EC08F00EC0DAF00DC0D9F00CC050
:10B3D000D8F00BC0D7F00E6A0D6A400E0C6E830ECB
:10B3E0000B6EDAC012F0D9C011F0D8C010F0D7C07F
:10B3F0000FF09EEC07F0010818E0126A116A400E87
:10B40000106E830E0F6EDAC00EF0D9C00DF0D8C0EA
:10B410000CF0D7C00BF04EEC08F00EC0DAF00DC007
:10B42000D9F00CC0D8F00BC0D7F0D7531CE0D89699
:10B43000D8AFD88618E40E6A0D6A400E0C6E830EE3
:10B440000B6EDAC012F0D9C011F0D8C010F0D7C01E
:10B450000FF050EC08F00EC0DAF00DC0D9F00CC0BF
:10B46000D8F00BC0D7F0DAC00EF0D9C00DF0D8C0BC
:10B470000CF0D7C00BF0A4C112F0A3C111F0A2C10F
:10B4800010F0A1C10FF04EEC08F00EC0E4F10DC0B9
:10B49000E3F10CC0E2F10BC0E1F10101E153000165
:10B4A0001EE0D8960101E2AFD886000118E40E6ACA
:10B4B0000D6A400E0C6E830E0B6EE4C112F0E3C1F8
:10B4C00011F0E2C110F0E1C10FF050EC08F00EC035
:10B4D000E4F10DC0E3F10CC0E2F10BC0E1F11200A8
:10B4E0001BD8C4C10EF0C3C10DF0C2C10CF0C1C164
:10B4F0000BF080C112F07FC111F07EC110F07DC150
:10B500000FF050EC08F00EC0C4F10DC0C3F10CC038
:10B51000C2F10BC0C1F112000101C2BF0AD0920EEC
:10B52000C45D0A0EC359060EC2597D0EC1590001F1
:10B53000D8A046D0C4C10EF0C3C10DF0C2C10CF0FA
:10B54000C1C10BF05EEC05F00EC02DF00DC02CF06B
:10B550000CC02BF00BC02AF00E6A800E0D6E120E7E
:10B560000C6E870E0B6E2DC012F02CC011F02BC08C
:10B5700010F02AC00FF04AEC09F00EC060F10DC0C7
:10B580005FF10CC05EF10BC05DF12E0E0E6EAA0EC7
:10B590000D6E230E0C6E7B0E0B6E60C112F05FC140
:10B5A00011F05EC110F05DC10FF0E2EC08F00EC0CA
:10B5B00080F10DC07FF10CC07EF10BC07DF1120057
:10B5C000D8960101C2AFD886000112E40F0E010126
:10B5D000C45D2D0EC359B20EC2597B0EC159000174
:10B5E00007E30101806B7F6B7E6B7D6B00011200B6
:10B5F000E10E0E6E2E0E0D6E650E0C6E840E0B6E31
:10B60000C4C112F0C3C111F0C2C110F0C1C10FF02A
:10B610004AEC09F00EC0ABF20DC0AAF20CC0A9F2C0
:10B620000BC0A8F2AC0E0E6EC50E0D6E270E0C6E82
:10B630006F0E0B6EABC212F0AAC211F0A9C210F0CD
:10B64000A8C20FF04AEC09F00EC05CF10DC05BF12E
:10B650000CC05AF10BC059F12E0E0E6E900E0D6EED
:10B66000200E0C6E790E0B6E5CC112F05BC111F0F6
:10B670005AC110F059C10FF050EC08F00EC05CF147
:10B680000DC05BF10CC05AF10BC059F15CC10EF05A
:10B690005BC10DF05AC10CF059C10BF0ABC212F0F6
:10B6A000AAC211F0A9C210F0A8C20FF04AEC09F02A
:10B6B0000EC05CF10DC05BF10CC05AF10BC059F12A
:10B6C000C10E0E6E390E0D6E230E0C6E7C0E0B6EBF
:10B6D0005CC112F05BC111F05AC110F059C10FF0FA
:10B6E00050EC08F00EC05CF10DC05BF10CC05AF1DB
:10B6F0000BC059F10E6A0D6A7A0E0C6E880E0B6E35
:10B700005CC112F05BC111F05AC110F059C10FF0C9
:10B710004AEC09F00EC03FF10DC03EF10CC03DF106
:10B720000BC03CF1560E0E6E0E0E0D6E2D0E0C6EF5
:10B730007B0E0B6EABC212F0AAC211F0A9C210F0C0
:10B74000A8C20FF04AEC09F00EC060F10DC05FF125
:10B750000CC05EF10BC05DF1AE0E0E6E470E0D6EAD
:10B76000010E0C6E7E0E0B6E60C112F05FC111F007
:10B770005EC110F05DC10FF050EC08F00EC060F13A
:10B780000DC05FF10CC05EF10BC05DF160C10EF049
:10B790005FC10DF05EC10CF05DC10BF0ABC212F0E9
:10B7A000AAC211F0A9C210F0A8C20FF04AEC09F029
:10B7B0000EC060F10DC05FF10CC05EF10BC05DF119
:10B7C0000E6A0D6A0C6A7F0E0B6E60C112F05FC1CB
:10B7D00011F05EC110F05DC10FF050EC08F00EC02A
:10B7E00060F10DC05FF10CC05EF10BC05DF10E6A3F
:10B7F000800E0D6E120E0C6E870E0B6E60C112F075
:10B800005FC111F05EC110F05DC10FF04AEC09F0AC
:10B810000EC047F10DC046F10CC045F10BC044F11C
:10B820003FC10EF03EC10DF03DC10CF03CC10BF02C
:10B8300047C112F046C111F045C110F044C10FF0EC
:10B84000E2EC08F00EC05CF10DC05BF10CC05AF1E7
:10B850000BC059F1340E0E6EFA0E0D6E0E0E0C6EFC
:10B86000790E0B6E5CC112F05BC111F05AC110F081
:10B8700059C10FF04AEC09F00EC080F10DC07FF104
:10B880000CC07EF10BC07DF112000301DE530001FC
:10B89000D8B412000301DE6B126AAD0E116E0E0EEB
:10B8A000106E8E0E0F6E70C10EF06FC10DF06EC176
:10B8B0000CF06DC10BF0E2EC08F00EC07CF10DC095
:10B8C0007BF10CC07AF10BC079F17CC10EF07BC129
:10B8D0000DF07AC10CF079C10BF07CC112F07BC184
:10B8E00011F07AC110F079C10FF04AEC09F00EC0E6
:10B8F0006DF00DC06CF00CC06BF00BC06AF0180E50
:10B900000E6E010E0D6E480E0C6E850E0B6E7CC118
:10B9100012F07BC111F07AC110F079C10FF04AEC3E
:10B9200009F00EC03FF10DC03EF10CC03DF10BC05F
:10B930003CF100016FEC6CF0F90E0E6EDB0E0D6E3B
:10B940001E0E0C6E730E0B6E6DC012F06CC011F0FB
:10B950006BC010F06AC00FF04AEC09F00EC05CF149
:10B960000DC05BF10CC05AF10BC059F12D0E0E6EDB
:10B97000D90E0D6E0B0E0C6E870E0B6E5CC112F0A5
:10B980005BC111F05AC110F059C10FF050EC08F032
:10B990000EC05CF10DC05BF10CC05AF10BC059F147
:10B9A0005CC10EF05BC10DF05AC10CF059C10BF037
:10B9B00047C112F046C111F045C110F044C10FF06B
:10B9C00050EC08F00EC01FF20DC01EF20CC01DF2AC
:10B9D0000BC01CF25E0E0E6E1B0E0D6E270E0C6E53
:10B9E000890E0B6E7CC112F07BC111F07AC110F090
:10B9F00079C10FF04AEC09F00EC03FF10DC03EF1E5
:10BA00000CC03DF10BC03CF16FEC6CF02C0E0E6ED7
:10BA1000810E0D6E140E0C6E750E0B6E6DC012F055
:10BA20006CC011F06BC010F06AC00FF04AEC09F066
:10BA30000EC05CF10DC05BF10CC05AF10BC059F1A6
:10BA4000940E0E6E370E0D6E070E0C6E870E0B6E7B
:10BA50005CC112F05BC111F05AC110F059C10FF076
:10BA60004EEC08F00EC05CF10DC05BF10CC05AF159
:10BA70000BC059F15CC10EF05BC10DF05AC10CF066
:10BA800059C10BF047C112F046C111F045C110F089
:10BA900044C10FF050EC08F00EC087F20DC086F2E2
:10BAA0000CC085F20BC084F2A60E0E6EFE0E0D6E5B
:10BAB000470E0C6E850E0B6E7CC112F07BC111F02F
:10BAC0007AC110F079C10FF04AEC09F00EC03FF1D5
:10BAD0000DC03EF10CC03DF10BC03CF16FEC6CF0C1
:10BAE000520E0E6E490E0D6E1D0E0C6E720E0B6E0A
:10BAF0006DC012F06CC011F06BC010F06AC00FF096
:10BB00004AEC09F00EC05CF10DC05BF10CC05AF1BB
:10BB10000BC059F1E70E0E6E3C0E0D6E330E0C6E1F
:10BB2000870E0B6E5CC112F05BC111F05AC110F0B0
:10BB300059C10FF04EEC08F00EC05CF10DC05BF186
:10BB40000CC05AF10BC059F15CC10EF05BC10DF095
:10BB50005AC10CF059C10BF047C112F046C111F0A7
:10BB600045C110F044C10FF050EC08F00EC023F2B4
:10BB70000DC022F20CC021F20BC020F2640E0E6E3A
:10BB8000430E0D6E4A0E0C6E960E0B6E7CC112F0BB
:10BB90007BC111F07AC110F079C10FF04AEC09F0C5
:10BBA0000EC03FF10DC03EF10CC03DF10BC03CF1A9
:10BBB0006FEC6CF00B0E0E6E9A0E0D6E160E0C6E78
:10BBC000780E0B6E6DC012F06CC011F06BC010F0EF
:10BBD0006AC00FF04AEC09F00EC05CF10DC05BF1D9
:10BBE0000CC05AF10BC059F1640E0E6E0D0E0D6EA5
:10BBF000140E0C6E870E0B6E5CC112F05BC111F05F
:10BC00005AC110F059C10FF050EC08F00EC05CF1B1
:10BC10000DC05BF10CC05AF10BC059F15CC10EF0C4
:10BC20005BC10DF05AC10CF059C10BF047C112F0C5
:10BC300046C111F045C110F044C10FF050EC08F0BE
:10BC40000EC08BF20DC08AF20CC089F20BC088F2D4
:10BC50007A0E0E6EEC0E0D6E2B0E0C6E810E0B6EB0
:10BC60007CC112F07BC111F07AC110F079C10FF0E4
:10BC70004AEC09F00EC03FF10DC03EF10CC03DF1A1
:10BC80000BC03CF16FEC6CF00E0E0E6E2F0E0D6EB5
:10BC9000080E0C6E760E0B6E6DC012F06CC011F0BB
:10BCA0006BC010F06AC00FF04AEC09F00EC05CF1F6
:10BCB0000DC05BF10CC05AF10BC059F1760E0E6E3F
:10BCC000970E0D6E010E0C6E870E0B6E5CC112F09E
:10BCD0005BC111F05AC110F059C10FF050EC08F0DF
:10BCE0000EC05CF10DC05BF10CC05AF10BC059F1F4
:10BCF0005CC10EF05BC10DF05AC10CF059C10BF0E4
:10BD000047C112F046C111F045C110F044C10FF017
:10BD10004EEC08F00EC083F20DC082F20CC081F22E
:10BD20000BC080F2340E0E6EFA0E0D6E0E0E0C6EFF
:10BD3000790E0B6E1FC212F01EC211F01DC210F060
:10BD40001CC20FF04AEC09F00EC05CF10DC05BF1B3
:10BD50000CC05AF10BC059F15CC17FF25BC17EF29D
:10BD60005AC17DF20101593D02D03682595102017A
:10BD70007C6F340E0E6EFA0E0D6E0E0E0C6E790E7A
:10BD80000B6E83C212F082C211F081C210F080C229
:10BD90000FF04AEC09F00EC083F20DC082F20CC025
:10BDA00081F20BC080F2340E0E6EFA0E0D6E0E0E86
:10BDB0000C6E790E0B6E83C212F082C211F081C23A
:10BDC00010F080C20FF04AEC09F00EC05CF10DC01B
:10BDD0005BF10CC05AF10BC059F15CC18FF25BC131
:10BDE0008EF25AC18DF20101593D02D0368259516D
:10BDF00002018C6F340E0E6EFA0E0D6E0E0E0C6E6E
:10BE0000790E0B6E23C212F022C211F021C210F083
:10BE100020C20FF04AEC09F00EC023F20DC022F24E
:10BE20000CC021F20BC020F2340E0E6EFA0E0D6E15
:10BE30000E0E0C6E790E0B6E87C212F086C211F0D8
:10BE400085C210F084C20FF04AEC09F00EC05CF11C
:10BE50000DC05BF10CC05AF10BC059F15CC193F2FB
:10BE60005BC192F25AC191F20101593D02D0368272
:10BE700059510201906F340E0E6EFA0E0D6E0E0EB9
:10BE80000C6E790E0B6E8BC212F08AC211F089C251
:10BE900010F088C20FF04AEC09F00EC08BF20DC012
:10BEA0008AF20CC089F20BC088F2880E0E6E4B0E1F
:10BEB0000D6E0E0E0C6E790E0B6E7CC112F07BC1F6
:10BEC00011F07AC110F079C10FF04AEC09F00EC000
:10BED0005CF10DC05BF10CC05AF10BC059F1920E30
:10BEE0000E6EDC0E0D6E890E0C6E830E0B6E5CC139
:10BEF00012F05BC111F05AC110F059C10FF04EECB5
:10BF000008F00EC05CF10DC05BF10CC05AF10BC023
:10BF100059F183C20EF082C20DF081C20CF080C2D2
:10BF20000BF084EC05F00EC060F10DC05FF10CC0A9
:10BF30005EF10BC05DF15CC10EF05BC10DF05AC14A
:10BF40000CF059C10BF060C112F05FC111F05EC17D
:10BF500010F05DC10FF04AEC09F00EC05CF10DC0AD
:10BF60005BF10CC05AF10BC059F19C0E0E6E500ED5
:10BF70000D6E080E0C6E720E0B6E7CC112F07BC142
:10BF800011F07AC110F079C10FF04AEC09F00EC03F
:10BF900064F10DC063F10CC062F10BC061F1630E7E
:10BFA0000E6EEE0E0D6EA20E0C6E7F0E0B6E64C149
:10BFB00012F063C111F062C110F061C10FF04EECDC
:10BFC00008F00EC064F10DC063F10CC062F10BC04B
:10BFD00061F17FC20EF07EC20DF07DC20CF07CC21A
:10BFE0000BF084EC05F00EC060F10DC05FF10CC0E9
:10BFF0005EF10BC05DF164C10EF063C10DF062C172
:10C000000CF061C10BF060C112F05FC111F05EC1B4
:10C0100010F05DC10FF04AEC09F00EC064F10DC0E4
:10C0200063F10CC062F10BC061F15CC10EF05BC149
:10C030000DF05AC10CF059C10BF064C112F063C18C
:10C0400011F062C110F061C10FF050EC08F00EC0A9
:10C0500068F10DC067F10CC066F10BC065F18FC2CD
:10C060000EF08EC20DF08DC20CF08CC20BF084EC81
:10C0700005F00EC05CF10DC05BF10CC05AF10BC0B5
:10C0800059F1AB0E0E6ECF0E0D6E550E0C6E7C0E72
:10C090000B6E5CC112F05BC111F05AC110F059C1B6
:10C0A0000FF04AEC09F00EC05CF10DC05BF10CC062
:10C0B0005AF10BC059F168C10EF067C10DF066C1AD
:10C0C0000CF065C10BF05CC112F05BC111F05AC1FC
:10C0D00010F059C10FF050EC08F00EC068F10DC01F
:10C0E00067F10CC066F10BC065F193C20EF092C20D
:10C0F0000DF091C20CF090C20BF084EC05F00EC074
:10C100005CF10DC05BF10CC05AF10BC059F1BC0ED3
:10C110000E6E960E0D6E500E0C6E7C0E0B6E5CC18C
:10C1200012F05BC111F05AC110F059C10FF04AEC86
:10C1300009F00EC05CF10DC05BF10CC05AF10BC0F0
:10C1400059F168C10EF067C10DF066C10CF065C110
:10C150000BF05CC112F05BC111F05AC110F059C173
:10C160000FF04EEC08F00EC068F10DC067F10CC086
:10C1700066F10BC065F17F0E0E6E870E0D6E220EFE
:10C180000C6E730E0B6E7CC112F07BC111F07AC184
:10C1900010F079C10FF04AEC09F00EC05CF10DC04F
:10C1A0005BF10CC05AF10BC059F15C0E0E6E200E03
:10C1B0000D6E010E0C6E7C0E0B6E5CC112F05BC13D
:10C1C00011F05AC110F059C10FF04EEC08F00EC03A
:10C1D0005CF10DC05BF10CC05AF10BC059F123C2E8
:10C1E0000EF022C20DF021C20CF020C20BF084EC44
:10C1F00005F00EC060F10DC05FF10CC05EF10BC028
:10C200005DF15CC10EF05BC10DF05AC10CF059C17B
:10C210000BF060C112F05FC111F05EC110F05DC1A2
:10C220000FF04AEC09F00EC05CF10DC05BF10CC0E0
:10C230005AF10BC059F168C10EF067C10DF066C12B
:10C240000CF065C10BF05CC112F05BC111F05AC17A
:10C2500010F059C10FF050EC08F00EC068F10DC09D
:10C2600067F10CC066F10BC065F18BC20EF08AC29B
:10C270000DF089C20CF088C20BF084EC05F00EC002
:10C280005CF10DC05BF10CC05AF10BC059F1710E9D
:10C290000E6E3D0E0D6E0A0E0C6E7B0E0B6E5CC1AB
:10C2A00012F05BC111F05AC110F059C10FF04AEC05
:10C2B00009F00EC05CF10DC05BF10CC05AF10BC06F
:10C2C00059F168C10EF067C10DF066C10CF065C18F
:10C2D0000BF05CC112F05BC111F05AC110F059C1F2
:10C2E0000FF050EC08F00EC068F10DC067F10CC003
:10C2F00066F10BC065F17FC20EF07EC20DF07DC20B
:10C300000CF07CC20BF023C212F022C211F021C249
:10C3100010F020C20FF050EC08F084EC05F00EC0D5
:10C320005CF10DC05BF10CC05AF10BC059F1820EEB
:10C330000E6EA80E0D6E7B0E0C6E710E0B6E7CC118
:10C3400012F07BC111F07AC110F079C10FF04AEC04
:10C3500009F00EC060F10DC05FF10CC05EF10BC0C2
:10C360005DF13A0E0E6E920E0D6E4B0E0C6E7A0E45
:10C370000B6E60C112F05FC111F05EC110F05DC1C3
:10C380000FF04EEC08F00EC064F10DC063F10CC06C
:10C3900062F10BC061F15CC10EF05BC10DF05AC1DE
:10C3A0000CF059C10BF064C112F063C111F062C10D
:10C3B00010F061C10FF04AEC09F00EC064F10DC03D
:10C3C00063F10CC062F10BC061F168C10EF067C18E
:10C3D0000DF066C10CF065C10BF064C112F063C1D1
:10C3E00011F062C110F061C10FF04EEC08F00EC008
:10C3F00068F10DC067F10CC066F10BC065F193C226
:10C400000EF092C20DF091C20CF090C20BF083C2FC
:10C4100012F082C211F081C210F080C20FF04EEC17
:10C4200008F084EC05F00EC05CF10DC05BF10CC0AF
:10C430005AF10BC059F14D0E0E6E150E0D6E0C0E0D
:10C440000C6E7A0E0B6E5CC112F05BC111F05AC11A
:10C4500010F059C10FF04AEC09F00EC05CF10DC0AC
:10C460005BF10CC05AF10BC059F168C10EF067C105
:10C470000DF066C10CF065C10BF05CC112F05BC140
:10C4800011F05AC110F059C10FF04EEC08F00EC077
:10C4900068F10DC067F10CC066F10BC065F193C285
:10C4A0000EF092C20DF091C20CF090C20BF08BC254
:10C4B00012F08AC211F089C210F088C20FF050EC5D
:10C4C00008F084EC05F00EC05CF10DC05BF10CC00F
:10C4D0005AF10BC059F1AB0E0E6ECF0E0D6E550E0C
:10C4E0000C6E790E0B6E5CC112F05BC111F05AC17B
:10C4F00010F059C10FF04AEC09F00EC05CF10DC00C
:10C500005BF10CC05AF10BC059F168C10EF067C164
:10C510000DF066C10CF065C10BF05CC112F05BC19F
:10C5200011F05AC110F059C10FF04EEC08F00EC0D6
:10C5300068F10DC067F10CC066F10BC065F17FC2F8
:10C540000EF07EC20DF07DC20CF07CC20BF023C257
:10C5500012F022C211F021C210F020C20FF04EECF6
:10C5600008F084EC05F00EC05CF10DC05BF10CC06E
:10C570005AF10BC059F10E0E0E6E4F0E0D6E2F0EAE
:10C580000C6E790E0B6E5CC112F05BC111F05AC1DA
:10C5900010F059C10FF04AEC09F00EC05CF10DC06B
:10C5A0005BF10CC05AF10BC059F168C10EF067C1C4
:10C5B0000DF066C10CF065C10BF05CC112F05BC1FF
:10C5C00011F05AC110F059C10FF050EC08F00EC034
:10C5D00068F10DC067F10CC066F10BC065F17FC258
:10C5E0000EF07EC20DF07DC20CF07CC20BF093C247
:10C5F00012F092C211F091C210F090C20FF04EEC06
:10C6000008F00EC02DF00DC02CF00CC02BF00BC0AC
:10C610002AF02DC00EF02CC00DF02BC00CF02AC05B
:10C620000BF08BC212F08AC211F089C210F088C2DE
:10C630000FF050EC08F084EC05F00EC05CF10DC07A
:10C640005BF10CC05AF10BC059F1210E0E6E1F0E9A
:10C650000D6E740E0C6E780E0B6E5CC112F05BC129
:10C6600011F05AC110F059C10FF04AEC09F00EC098
:10C670005CF10DC05BF10CC05AF10BC059F168C1FF
:10C680000EF067C10DF066C10CF065C10BF05CC126
:10C6900012F05BC111F05AC110F059C10FF04EEC0D
:10C6A00008F00EC068F10DC067F10CC066F10BC058
:10C6B00065F17FC20EF07EC20DF07DC20CF07CC22F
:10C6C0000BF083C212F082C211F081C210F080C25E
:10C6D0000FF04EEC08F084EC05F00EC05CF10DC0DC
:10C6E0005BF10CC05AF10BC059F15F0E0E6E290EB2
:10C6F0000D6E4B0E0C6E780E0B6E5CC112F05BC1B2
:10C7000011F05AC110F059C10FF04AEC09F00EC0F7
:10C710005CF10DC05BF10CC05AF10BC059F168C15E
:10C720000EF067C10DF066C10CF065C10BF05CC185
:10C7300012F05BC111F05AC110F059C10FF050EC6A
:10C7400008F00EC068F10DC067F10CC066F10BC0B7
:10C7500065F193C20EF092C20DF091C20CF090C23E
:10C760000BF08BC212F08AC211F089C210F088C29D
:10C770000FF04EEC08F084EC05F00EC05CF10DC03B
:10C780005BF10CC05AF10BC059F1110E0E6EC70EC1
:10C790000D6E3A0E0C6E780E0B6E5CC112F05BC122
:10C7A00011F05AC110F059C10FF04AEC09F00EC057
:10C7B0005CF10DC05BF10CC05AF10BC059F168C1BE
:10C7C0000EF067C10DF066C10CF065C10BF05CC1E5
:10C7D00012F05BC111F05AC110F059C10FF050ECCA
:10C7E00008F00EC097F20DC096F20CC095F20BC087
:10C7F00094F2110E0E6E8D0E0D6E6E0E0C6E740E8A
:10C800000B6E7CC112F07BC111F07AC110F079C1BE
:10C810000FF04AEC09F00EC05CF10DC05BF10CC0EA
:10C820005AF10BC059F1290E0E6E5C0E0D6E130EEF
:10C830000C6E820E0B6E5CC112F05BC111F05AC11E
:10C8400010F059C10FF050EC08F00EC05CF10DC0B3
:10C850005BF10CC05AF10BC059F183C20EF082C2D9
:10C860000DF081C20CF080C20BF082EC05F00EC01E
:10C8700060F10DC05FF10CC05EF10BC05DF15CC1F9
:10C880000EF05BC10DF05AC10CF059C10BF060C144
:10C8900012F05FC111F05EC110F05DC10FF04AEC03
:10C8A00009F00EC064F10DC063F10CC062F10BC061
:10C8B00061F1240E0E6E0B0E0D6E180E0C6E730EC3
:10C8C0000B6E7CC112F07BC111F07AC110F079C1FE
:10C8D0000FF04AEC09F00EC05CF10DC05BF10CC02A
:10C8E0005AF10BC059F1FB0E0E6E5C0E0D6E0D0E63
:10C8F0000C6E7E0E0B6E5CC112F05BC111F05AC162
:10C9000010F059C10FF04EEC08F00EC05CF10DC0F4
:10C910005BF10CC05AF10BC059F17FC20EF07EC220
:10C920000DF07DC20CF07CC20BF082EC05F00EC065
:10C9300060F10DC05FF10CC05EF10BC05DF15CC138
:10C940000EF05BC10DF05AC10CF059C10BF060C183
:10C9500012F05FC111F05EC110F05DC10FF04AEC42
:10C9600009F00EC05CF10DC05BF10CC05AF10BC0B8
:10C9700059F164C10EF063C10DF062C10CF061C1E8
:10C980000BF05CC112F05BC111F05AC110F059C13B
:10C990000FF050EC08F00EC064F10DC063F10CC054
:10C9A00062F10BC061F18FC20EF08EC20DF08DC22C
:10C9B0000CF08CC20BF082EC05F00EC05CF10DC0E7
:10C9C0005BF10CC05AF10BC059F1A30E0E6E230E91
:10C9D0000D6E390E0C6E7B0E0B6E5CC112F05BC1DE
:10C9E00011F05AC110F059C10FF04AEC09F00EC015
:10C9F0005CF10DC05BF10CC05AF10BC059F164C180
:10CA00000EF063C10DF062C10CF061C10BF05CC1AE
:10CA100012F05BC111F05AC110F059C10FF04EEC89
:10CA200008F00EC064F10DC063F10CC062F10BC0E0
:10CA300061F193C20EF092C20DF091C20CF090C25F
:10CA40000BF082EC05F00EC05CF10DC05BF10CC088
:10CA50005AF10BC059F10F0E0E6E0B0E0D6E350E06
:10CA60000C6E7B0E0B6E5CC112F05BC111F05AC1F3
:10CA700010F059C10FF04AEC09F00EC05CF10DC086
:10CA80005BF10CC05AF10BC059F164C10EF063C1E7
:10CA90000DF062C10CF061C10BF05CC112F05BC122
:10CAA00011F05AC110F059C10FF050EC08F00EC04F
:10CAB00064F10DC063F10CC062F10BC061F17FC283
:10CAC0000EF07EC20DF07DC20CF07CC20BF023C2D2
:10CAD00012F022C211F021C210F020C20FF050EC6F
:10CAE00008F082EC05F00EC05CF10DC05BF10CC0EB
:10CAF0005AF10BC059F17C0E0E6EF20E0D6E300E17
:10CB00000C6E790E0B6E5CC112F05BC111F05AC154
:10CB100010F059C10FF04AEC09F00EC05CF10DC0E5
:10CB20005BF10CC05AF10BC059F164C10EF063C146
:10CB30000DF062C10CF061C10BF05CC112F05BC181
:10CB400011F05AC110F059C10FF050EC08F00EC0AE
:10CB500064F10DC063F10CC062F10BC061F193C2CE
:10CB60000EF092C20DF091C20CF090C20BF083C295
:10CB700012F082C211F081C210F080C20FF04EECB0
:10CB800008F082EC05F00EC05CF10DC05BF10CC04A
:10CB90005AF10BC059F1E20E0E6EE90E0D6E150E34
:10CBA0000C6E790E0B6E5CC112F05BC111F05AC1B4
:10CBB00010F059C10FF04AEC09F00EC05CF10DC045
:10CBC0005BF10CC05AF10BC059F164C10EF063C1A6
:10CBD0000DF062C10CF061C10BF05CC112F05BC1E1
:10CBE00011F05AC110F059C10FF050EC08F00EC00E
:10CBF00064F10DC063F10CC062F10BC061F17FC242
:10CC00000EF07EC20DF07DC20CF07CC20BF08BC228
:10CC100012F08AC211F089C210F088C20FF050ECF5
:10CC200008F082EC05F00EC05CF10DC05BF10CC0A9
:10CC30005AF10BC059F1F40E0E6EFD0E0D6E540E2E
:10CC40000C6E780E0B6E5CC112F05BC111F05AC114
:10CC500010F059C10FF04AEC09F00EC05CF10DC0A4
:10CC60005BF10CC05AF10BC059F164C10EF063C105
:10CC70000DF062C10CF061C10BF05CC112F05BC140
:10CC800011F05AC110F059C10FF050EC08F00EC06D
:10CC900064F10DC063F10CC062F10BC061F17FC2A1
:10CCA0000EF07EC20DF07DC20CF07CC20BF023C2F0
:10CCB00012F022C211F021C210F020C20FF04EEC8F
:10CCC00008F082EC05F00EC05CF10DC05BF10CC009
:10CCD0005AF10BC059F1070E0E6E5F0E0D6E180E55
:10CCE0000C6E780E0B6E5CC112F05BC111F05AC174
:10CCF00010F059C10FF04AEC09F00EC05CF10DC004
:10CD00005BF10CC05AF10BC059F164C10EF063C164
:10CD10000DF062C10CF061C10BF05CC112F05BC19F
:10CD200011F05AC110F059C10FF04EEC08F00EC0CE
:10CD300064F10DC063F10CC062F10BC061F17FC200
:10CD40000EF07EC20DF07DC20CF07CC20BF083C2EF
:10CD500012F082C211F081C210F080C20FF04EECCE
:10CD600008F082EC05F00EC05CF10DC05BF10CC068
:10CD70005AF10BC059F1D00E0E6E440E0D6E580EC6
:10CD80000C6E770E0B6E5CC112F05BC111F05AC1D4
:10CD900010F059C10FF04AEC09F00EC05CF10DC063
:10CDA0005BF10CC05AF10BC059F164C10EF063C1C4
:10CDB0000DF062C10CF061C10BF05CC112F05BC1FF
:10CDC00011F05AC110F059C10FF04EEC08F00EC02E
:10CDD0006BF20DC06AF20CC069F20BC068F2126A05
:10CDE000116A610E106E8A0E0F6E97C20EF096C217
:10CDF0000DF095C20CF094C20BF0E2EC08F00EC0FE
:10CE000097F20DC096F20CC095F20BC094F2126A24
:10CE1000116A610E106E8A0E0F6E6BC20EF06AC23E
:10CE20000DF069C20CF068C20BF0E2EC08F00EC025
:10CE30006BF20DC06AF20CC069F20BC068F200011F
:10CE4000120001011431E8320001D8B012D1B8C18A
:10CE50000EF0B7C10DF0B6C10CF0B5C10BF082EC0D
:10CE600005F00EC0B4F10DC0B3F10CC0B2F10BC0AF
:10CE7000B1F1B8C10EF0B7C10DF0B6C10CF0B5C13B
:10CE80000BF084EC05F00EC0BCF10DC0BBF10CC082
:10CE9000BAF10BC0B9F1BCC10EF0BBC10DF0BAC103
:10CEA0000CF0B9C10BF0B4C112F0B3C111F0B2C1B2
:10CEB00010F0B1C10FF0E2EC08F00EC05CF10DC053
:10CEC0005BF10CC05AF10BC059F1420E0E6E240EEC
:10CED0000D6E7F0E0C6E7E0E0B6E5CC112F05BC190
:10CEE00011F05AC110F059C10FF04AEC09F00EC010
:10CEF0005CF10DC05BF10CC05AF10BC059F15CC183
:10CF00000EF05BC10DF05AC10CF059C10BF02CECC6
:10CF100004F00EC0F4F10DC0F3F10CC0F2F10BC03F
:10CF2000F1F1F4C10EF0F3C10DF0F2C10CF0F1C15A
:10CF30000BF082EC05F00EC0FBF10DC0FAF10CC055
:10CF4000F9F10BC0F8F1F4C10EF0F3C10DF0F2C12C
:10CF50000CF0F1C10BF084EC05F00EC0FFF10DC038
:10CF6000FEF10CC0FDF10BC0FCF10101148317C2EE
:10CF70000EF016C20DF015C20CF014C20BF0BCC1BD
:10CF800012F0BBC111F0BAC110F0B9C10FF04AECF8
:10CF900009F00EC05CF10DC05BF10CC05AF10BC082
:10CFA00059F1420E0E6E240E0D6E7F0E0C6E7E0E2B
:10CFB0000B6EFFC112F0FEC111F0FDC110F0FCC1FB
:10CFC0000FF04AEC09F00EC060F10DC05FF10CC02B
:10CFD0005EF10BC05DF15CC10EF05BC10DF05AC19A
:10CFE0000CF059C10BF060C112F05FC111F05EC1CD
:10CFF00010F05DC10FF050EC08F00EC00BF20DC048
:10D000000AF20CC009F20BC008F217C20EF016C2E9
:10D010000DF015C20CF014C20BF0B4C112F0B3C184
:10D0200011F0B2C110F0B1C10FF04AEC09F00EC01E
:10D030005CF10DC05BF10CC05AF10BC059F1FBC1A2
:10D040000EF0FAC10DF0F9C10CF0F8C10BF05CC1A3
:10D0500012F05BC111F05AC110F059C10FF050EC41
:10D0600008F00EC007F20DC006F20CC005F20BC0AE
:10D0700004F200011BC20EF01AC20DF019C20CF02E
:10D0800018C20BF084EC05F00EC05CF10DC05BF132
:10D090000CC05AF10BC059F10E6A0D6A0C6A7F0E72
:10D0A0000B6E5CC112F05BC111F05AC110F059C196
:10D0B0000FF0E2EC08F00EC003F20DC002F20CC05B
:10D0C00001F20BC000F2A4C10EF0A3C10DF0A2C189
:10D0D0000CF0A1C10BF082EC05F00EC0D0F10DC038
:10D0E000CFF10CC0CEF10BC0CDF1C4C10EF0C3C165
:10D0F0000DF0C2C10CF0C1C10BF084EC05F00EC004
:10D10000C0F10DC0BFF10CC0BEF10BC0BDF1C4C178
:10D110000EF0C3C10DF0C2C10CF0C1C10BF082EC26
:10D1200005F00EC0C8F10DC0C7F10CC0C6F10BC0B0
:10D13000C5F1A4C10EF0A3C10DF0A2C10CF0A1C1B4
:10D140000BF084EC05F00EC05CF10DC05BF10CC07F
:10D150005AF10BC059F15CC10EF05BC10DF05AC120
:10D160000CF059C10BF007C212F006C211F005C253
:10D1700010F004C20FF04AEC09F00EC05CF10DC0D3
:10D180005BF10CC05AF10BC059F103C20EF002C2A0
:10D190000DF001C20CF000C20BF0C8C112F0C7C103
:10D1A00011F0C6C110F0C5C10FF04AEC09F00EC075
:10D1B00060F10DC05FF10CC05EF10BC05DF107C204
:10D1C0000EF006C20DF005C20CF004C20BF0D0C187
:10D1D00012F0CFC111F0CEC110F0CDC10FF04AEC6A
:10D1E00009F00EC064F10DC063F10CC062F10BC018
:10D1F00061F160C10EF05FC10DF05EC10CF05DC168
:10D200000BF064C112F063C111F062C110F061C192
:10D210000FF04EEC08F00EC060F10DC05FF10CC0D5
:10D220005EF10BC05DF15CC10EF05BC10DF05AC147
:10D230000CF059C10BF060C112F05FC111F05EC17A
:10D2400010F05DC10FF0E2EC08F00EC013F20DC05B
:10D2500012F20CC011F20BC010F213C20EF012C287
:10D260000DF011C20CF010C20BF02CEC04F00EC04B
:10D270000FF20DC00EF20CC00DF20BC00CF2A4C1E7
:10D280000EF0A3C10DF0A2C10CF0A1C10BF00FC2B2
:10D2900012F00EC211F00DC210F00CC20FF050ECE3
:10D2A00008F00EC0E4F10DC0E3F10CC0E2F10BC0D8
:10D2B000E1F1E4C10EF0E3C10DF0E2C10CF0E1C117
:10D2C0000BF082EC05F00EC0E0F10DC0DFF10CC0F8
:10D2D000DEF10BC0DDF1DA0E0E6E0F0E0D6E490E93
:10D2E0000C6E810E0B6EE4C112F0E3C111F0E2C1CD
:10D2F00010F0E1C10FF09EEC07F001081AE0DA0E21
:10D30000126E0F0E116E490E106E810E0F6EE4C17B
:10D310000EF0E3C10DF0E2C10CF0E1C10BF04EECF8
:10D3200008F00EC0E4F10DC0E3F10CC0E2F10BC057
:10D33000E1F10101E153000120E0D8960101E2AFE3
:10D34000D88600011AE4DA0E0E6E0F0E0D6E490E2D
:10D350000C6E810E0B6EE4C112F0E3C111F0E2C15C
:10D3600010F0E1C10FF050EC08F00EC0E4F10DC078
:10D37000E3F10CC0E2F10BC0E1F103C20EF002C216
:10D380000DF001C20CF000C20BF0C0C112F0BFC121
:10D3900011F0BEC110F0BDC10FF04AEC09F00EC093
:10D3A0005CF10DC05BF10CC05AF10BC059F15CC1CE
:10D3B0000EF05BC10DF05AC10CF059C10BF00BC25D
:10D3C00012F00AC211F009C210F008C20FF04EECC0
:10D3D00008F00EC05CF10DC05BF10CC05AF10BC03F
:10D3E00059F1E0C10EF0DFC10DF0DEC10CF0DDC17E
:10D3F0000BF05CC112F05BC111F05AC110F059C1C1
:10D400000FF04AEC09F00EC05CF10DC05BF10CC0EE
:10D410005AF10BC059F103C20EF002C20DF001C265
:10D420000CF000C20BF0C8C112F0C7C111F0C6C1A8
:10D4300010F0C5C10FF04AEC09F00EC060F10DC04C
:10D440005FF10CC05EF10BC05DF160C10EF05FC119
:10D450000DF05EC10CF05DC10BF0D0C112F0CFC178
:10D4600011F0CEC110F0CDC10FF04AEC09F00EC0A2
:10D4700060F10DC05FF10CC05EF10BC05DF160C1E9
:10D480000EF05FC10DF05EC10CF05DC10BF007C284
:10D4900012F006C211F005C210F004C20FF04EECFB
:10D4A00008F00EC060F10DC05FF10CC05EF10BC062
:10D4B0005DF15CC10EF05BC10DF05AC10CF059C1B9
:10D4C0000BF060C112F05FC111F05EC110F05DC1E0
:10D4D0000FF0E2EC08F02CEC04F00EC0D8F10DC017
:10D4E000D7F10CC0D6F10BC0D5F11200DA0E126ED6
:10D4F0000F0E116E490E106E810E0F6E0AC10EF0E6
:10D5000009C10DF008C10CF007C10BF0E2EC08F006
:10D510000EC05CF10DC05BF10CC05AF10BC059F1AB
:10D52000366A5CC10EF05BC10DF05AC10CF059C1F6
:10D530000BF09AEC09F00BC058F10CC057F10DC07C
:10D5400056F10101556F400E366E58C10EF057C1AD
:10D550000DF056C10CF055C10BF0EEEC09F0DA0EEF
:10D56000126E0F0E116E490E106E810E0F6E4AEC88
:10D5700009F00EC05CF10DC05BF10CC05AF10BC09C
:10D5800059F10AC10EF009C10DF008C10CF007C134
:10D590000BF05CC112F05BC111F05AC110F059C11F
:10D5A0000FF04EEC08F00EC05BF20DC05AF20CC04A
:10D5B00059F20BC058F25BC253F25AC252F259C22E
:10D5C00051F258C250F2000153C20EF052C20DF097
:10D5D00051C20CF050C20BF084EC05F00EC05CF1AF
:10D5E0000DC05BF10CC05AF10BC059F15CC10EF0DB
:10D5F0005BC10DF05AC10CF059C10BF027C212F0FB
:10D6000026C211F025C210F024C20FF04AEC09F036
:10D610000EC05CF10DC05BF10CC05AF10BC059F1AA
:10D6200053C20EF052C20DF051C20CF050C20BF0BA
:10D630005CC112F05BC111F05AC110F059C10FF07A
:10D640004EEC08F00EC05CF10DC05BF10CC05AF15D
:10D650000BC059F15CC10EF05BC10DF05AC10CF06A
:10D6600059C10BF05BC212F05AC211F059C210F04E
:10D6700058C20FF04EEC08F00EC057F20DC056F233
:10D680000CC055F20BC054F257C25CF156C25BF1AC
:10D6900055C25AF101015A9F54C259F15ABF0AD0DA
:10D6A000BD0E5C5D370E5B59060E5A596B0E59590B
:10D6B0000001D8A078D053C20EF052C20DF051C272
:10D6C0000CF050C20BF082EC05F00EC060F10DC002
:10D6D0005FF10CC05EF10BC05DF160C10EF05FC187
:10D6E0000DF05EC10CF05DC10BF027C212F026C236
:10D6F00011F025C210F024C20FF04AEC09F00EC060
:10D7000060F10DC05FF10CC05EF10BC05DF10E6AFF
:10D710000D6A0C6A7F0E0B6E60C112F05FC111F0D2
:10D720005EC110F05DC10FF04EEC08F00EC060F16C
:10D730000DC05FF10CC05EF10BC05DF157C20EF081
:10D7400056C20DF055C20CF054C20BF060C112F07D
:10D750005FC111F05EC110F05DC10FF0E2EC08F0A6
:10D760000EC057F20DC056F20CC055F20BC054F269
:10D7700053C20EF052C20DF051C20CF050C20BF069
:10D7800057C212F056C211F055C210F054C20FF039
:10D790004EEC08F00EC053F20DC052F20CC051F224
:10D7A0000BC050F210D753C20EF052C20DF051C24E
:10D7B0000CF002015051D8B43684D8A450050B6E39
:10D7C0005EEC05F00EC05CF10DC05BF10CC05AF1CF
:10D7D0000BC059F10E6A0D6A0C6A7F0E0B6E27C2E0
:10D7E00012F026C211F025C210F024C20FF04EEC48
:10D7F00008F00EC060F10DC05FF10CC05EF10BC00F
:10D800005DF10E6A0D6A0C6A7F0E0B6E27C212F074
:10D8100026C211F025C210F024C20FF050EC08F01F
:10D820000EC064F10DC063F10CC062F10BC061F178
:10D8300064C10EF063C10DF062C10CF061C10BF068
:10D8400060C112F05FC111F05EC110F05DC10FF058
:10D85000E2EC08F00EC064F10DC063F10CC062F19F
:10D860000BC061F164C10EF063C10DF062C10CF038
:10D8700061C10BF0F4EC06F00EC064F10DC063F171
:10D880000CC062F10BC061F164C10EF063C10DF018
:10D8900062C10CF061C10BF05CC112F05BC111F010
:10D8A0005AC110F059C10FF04AEC09F02CEC04F009
:10D8B0000EC05CF10DC05BF10CC05AF10BC059F108
:10D8C0005CC14BF25BC14AF25AC149F20101593DB8
:10D8D00002D0368259510201486F00011200366AA7
:10D8E0003FC10EF03EC10DF03DC10CF03CC10BF04C
:10D8F0009AEC09F00BC058F10CC057F10DC056F16D
:10D900000101556F400E366E58C10EF057C10DF033
:10D9100056C10CF055C10BF0EEEC09F00EC012F040
:10D920000DC011F00CC010F00BC00FF03FC10EF095
:10D930003EC10DF03DC10CF03CC10BF04EEC08F0C7
:10D940000EC03FF10DC03EF10CC03DF10BC03CF1EB
:10D950000E6A0D6A340E0C6E870E0B6E3FC112F00C
:10D960003EC111F03DC110F03CC10FF04AEC09F08E
:10D970000EC047F10DC046F10CC045F10BC044F19B
:10D9800000011200180E0E6E010E0D6E480E0C6E88
:10D99000850E0B6E7CC112F07BC111F07AC110F0C4
:10D9A00079C10FF04AEC09F00EC03FF10DC03EF115
:10D9B0000CC03DF10BC03CF192DFDD0E0E6E980EF7
:10D9C0000D6E1E0E0C6E730E0B6E6DC012F06CC0E1
:10D9D00011F06BC010F06AC00FF04AEC09F00EC0F5
:10D9E0005CF10DC05BF10CC05AF10BC059F12D0E6A
:10D9F0000E6ED90E0D6E0B0E0C6E870E0B6E5CC18B
:10DA000012F05BC111F05AC110F059C10FF050EC87
:10DA100008F00EC05CF10DC05BF10CC05AF10BC0F8
:10DA200059F15CC10EF05BC10DF05AC10CF059C147
:10DA30000BF047C112F046C111F045C110F044C1CE
:10DA40000FF050EC08F00EC01FF20DC01EF20CC01B
:10DA50001DF20BC01CF2A60E0E6EFE0E0D6E470ED2
:10DA60000C6E850E0B6E7CC112F07BC111F07AC179
:10DA700010F079C10FF04AEC09F00EC03FF10DC073
:10DA80003EF10CC03DF10BC03CF129DF910E0E6E52
:10DA9000750E0D6E5D0E0C6E6C0E0B6E7CC112F071
:10DAA0007BC111F07AC110F079C10FF04AEC09F096
:10DAB0000EC05CF10DC05BF10CC05AF10BC059F106
:10DAC000520E0E6E490E0D6E1D0E0C6E720E0B6E0A
:10DAD0005CC112F05BC111F05AC110F059C10FF0D6
:10DAE00050EC08F00EC05CF10DC05BF10CC05AF1B7
:10DAF0000BC059F15CC10EF05BC10DF05AC10CF0C6
:10DB000059C10BF06DC012F06CC011F06BC010F079
:10DB10006AC00FF04AEC09F00EC05CF10DC05BF179
:10DB20000CC05AF10BC059F1E80E0E6E3C0E0D6E92
:10DB3000330E0C6E870E0B6E5CC112F05BC111F0E0
:10DB40005AC110F059C10FF04EEC08F00EC05CF154
:10DB50000DC05BF10CC05AF10BC059F15CC10EF065
:10DB60005BC10DF05AC10CF059C10BF047C112F066
:10DB700046C111F045C110F044C10FF050EC08F05F
:10DB80000EC023F20DC022F20CC021F20BC020F215
:10DB9000690E0E6E520E0D6E2F0E0C6E700E0B6E09
:10DBA0007CC112F07BC111F07AC110F079C10FF085
:10DBB0004AEC09F00EC05CF10DC05BF10CC05AF1EB
:10DBC0000BC059F19E0E0E6E4A0E0D6E070E0C6EB6
:10DBD000680E0B6E6DC012F06CC011F06BC010F0CF
:10DBE0006AC00FF04AEC09F00EC060F10DC05FF1A1
:10DBF0000CC05EF10BC05DF15CC10EF05BC10DF0BD
:10DC00005AC10CF059C10BF060C112F05FC111F0A4
:10DC10005EC110F05DC10FF050EC08F00EC05CF179
:10DC20000DC05BF10CC05AF10BC059F17A0E0E6EAB
:10DC3000390E0D6E090E0C6E790E0B6E5CC112F072
:10DC40005BC111F05AC110F059C10FF04EEC08F051
:10DC50000EC027F20DC026F20CC025F20BC024F234
:10DC6000340E0E6EFA0E0D6E0E0E0C6E790E0B6EDD
:10DC700023C212F022C211F021C210F020C20FF014
:10DC80004AEC09F00EC00AF10DC009F10CC008F110
:10DC90000BC007F176EC6AF0580E0E6E350E0D6E65
:10DCA0007A0E0C6E840E0B6E7CC112F07BC111F0EB
:10DCB0007AC110F079C10FF04AEC09F00EC03FF1C3
:10DCC0000DC03EF10CC03DF10BC03CF108DEE10E91
:10DCD0000E6E3A0E0D6E190E0C6E860E0B6E47C14F
:10DCE00012F046C111F045C110F044C10FF050ECE4
:10DCF00008F00EC05CF10DC05BF10CC05AF10BC016
:10DD000059F1340E0E6EFA0E0D6E0E0E0C6E790E6B
:10DD10000B6E5CC112F05BC111F05AC110F059C119
:10DD20000FF04AEC09F00EC03BF10DC03AF10CC007
:10DD300039F10BC038F1580E0E6E350E0D6E7A0E9D
:10DD40000C6E850E0B6E7CC112F07BC111F07AC196
:10DD500010F079C10FF04AEC09F00EC03FF10DC090
:10DD60003EF10CC03DF10BC03CF16FEC6CF0EC0EE1
:10DD70000E6E910E0D6E580E0C6E860E0B6E47C118
:10DD800012F046C111F045C110F044C10FF050EC43
:10DD900008F00EC05CF10DC05BF10CC05AF10BC075
:10DDA00059F1340E0E6EFA0E0D6E0E0E0C6E790ECB
:10DDB0000B6E5CC112F05BC111F05AC110F059C179
:10DDC0000FF04AEC09F00EC02BF20DC02AF20CC085
:10DDD00029F20BC028F2A40E0E6E220E0D6E370E25
:10DDE0000C6E850E0B6E7CC112F07BC111F07AC1F6
:10DDF00010F079C10FF04AEC09F00EC03FF10DC0F0
:10DE00003EF10CC03DF10BC03CF16FEC6CF0520EDA
:10DE10000E6E580E0D6E1C0E0C6E870E0B6E47C1EB
:10DE200012F046C111F045C110F044C10FF050ECA2
:10DE300008F00EC05CF10DC05BF10CC05AF10BC0D4
:10DE400059F1340E0E6EFA0E0D6E0E0E0C6E790E2A
:10DE50000B6E5CC112F05BC111F05AC110F059C1D8
:10DE60000FF04AEC09F00EC02FF20DC02EF20CC0DC
:10DE70002DF20BC02CF24D0E0E6E9B0E0D6E1A0E77
:10DE80000C6E890E0B6E7CC112F07BC111F07AC151
:10DE900010F079C10FF04AEC09F00EC03FF10DC04F
:10DEA0003EF10CC03DF10BC03CF16FEC6CF0620E2A
:10DEB0000E6EBE0E0D6E3C0E0C6E750E0B6E6DC0B2
:10DEC00012F06CC011F06BC010F06AC00FF04AEC99
:10DED00009F00EC05CF10DC05BF10CC05AF10BC033
:10DEE00059F1B80E0E6E5E0E0D6E2F0E0C6E870E73
:10DEF0000B6E5CC112F05BC111F05AC110F059C138
:10DF00000FF04EEC08F00EC05CF10DC05BF10CC0E0
:10DF10005AF10BC059F15CC10EF05BC10DF05AC152
:10DF20000CF059C10BF047C112F046C111F045C1C8
:10DF300010F044C10FF050EC08F00EC05CF10DC0C1
:10DF40005BF10CC05AF10BC059F1340E0E6EFA0E93
:10DF50000D6E0E0E0C6E790E0B6E5CC112F05BC175
:10DF600011F05AC110F059C10FF04AEC09F00EC07F
:10DF700033F20DC032F20CC031F20BC030F29A0E07
:10DF80000E6E990E0D6E210E0C6E830E0B6E7CC103
:10DF900012F07BC111F07AC110F079C10FF04AEC98
:10DFA00009F00EC05CF10DC05BF10CC05AF10BC062
:10DFB00059F1A40E0E6E300E0D6E670E0C6E860EAD
:10DFC0000B6E5CC112F05BC111F05AC110F059C167
:10DFD0000FF050EC08F00EC05CF10DC05BF10CC00E
:10DFE0005AF10BC059F1340E0E6EFA0E0D6E0E0E74
:10DFF0000C6E790E0B6E5CC112F05BC111F05AC150
:10E0000010F059C10FF04AEC09F00EC037F20DC004
:10E0100036F20CC035F20BC034F2A40E0E6E220E96
:10E020000D6E370E0C6E860E0B6E7CC112F07BC12E
:10E0300011F07AC110F079C10FF04AEC09F00EC06E
:10E040003FF10DC03EF10CC03DF10BC03CF16FEC57
:10E050006CF0330E0E6EB30E0D6E300E0C6E870E1E
:10E060000B6E47C112F046C111F045C110F044C11A
:10E070000FF050EC08F00EC05CF10DC05BF10CC06D
:10E080005AF10BC059F1340E0E6EFA0E0D6E0E0ED3
:10E090000C6E790E0B6E5CC112F05BC111F05AC1AF
:10E0A00010F059C10FF04AEC09F00EC03BF20DC060
:10E0B0003AF20CC039F20BC038F23BC10EF03AC153
:10E0C0000DF039C10CF038C10BF082EC05F00EC038
:10E0D0005CF10DC05BF10CC05AF10BC059F1F00EB0
:10E0E0000E6EA20E0D6E2F0E0C6E750E0B6E5CC1B9
:10E0F00012F05BC111F05AC110F059C10FF04AEC97
:10E1000009F00EC05CF10DC05BF10CC05AF10BC000
:10E1100059F12BC20EF02AC20DF029C20CF028C210
:10E120000BF082EC05F00EC060F10DC05FF10CC089
:10E130005EF10BC05DF1D30E0E6ED90E0D6E490E61
:10E140000C6E750E0B6E60C112F05FC111F05EC1F6
:10E1500010F05DC10FF04AEC09F00EC060F10DC087
:10E160005FF10CC05EF10BC05DF12FC20EF02EC24C
:10E170000DF02DC20CF02CC20BF082EC05F00EC09D
:10E1800064F10DC063F10CC062F10BC061F16F0E60
:10E190000E6E120E0D6E030E0C6E760E0B6E64C1BB
:10E1A00012F063C111F062C110F061C10FF04AECCE
:10E1B00009F00EC064F10DC063F10CC062F10BC038
:10E1C00061F133C20EF032C20DF031C20CF030C238
:10E1D0000BF084EC05F00EC068F10DC067F10CC0C7
:10E1E00066F10BC065F16F0E0E6E9E0E0D6E6A0E1F
:10E1F0000C6E750E0B6E68C112F067C111F066C12E
:10E2000010F065C10FF04AEC09F00EC068F10DC0C6
:10E2100067F10CC066F10BC065F137C20EF036C273
:10E220000DF035C20CF034C20BF084EC05F00EC0DA
:10E230006CF10DC06BF10CC06AF10BC069F1E40E1A
:10E240000E6E4E0E0D6E690E0C6E750E0B6E6CC161
:10E2500012F06BC111F06AC110F069C10FF04AEC05
:10E2600009F00EC06CF10DC06BF10CC06AF10BC06F
:10E2700069F15CC10EF05BC10DF05AC10CF059C1DF
:10E280000BF060C112F05FC111F05EC110F05DC112
:10E290000FF050EC08F00EC03FF20DC03EF20CC083
:10E2A0003DF20BC03CF23FC20EF03EC20DF03DC24B
:10E2B0000CF03CC20BF064C112F063C111F062C1FA
:10E2C00010F061C10FF050EC08F00EC03FF20DC02D
:10E2D0003EF20CC03DF20BC03CF23FC20EF03EC21B
:10E2E0000DF03DC20CF03CC20BF068C112F067C1EA
:10E2F00011F066C110F065C10FF050EC08F00EC0CF
:10E300003FF20DC03EF20CC03DF20BC03CF23FC2EA
:10E310000EF03EC20DF03DC20CF03CC20BF06CC1E1
:10E3200012F06BC111F06AC110F069C10FF050EC2E
:10E3300008F00EC03FF20DC03EF20CC03DF20BC023
:10E340003CF23BC10EF03AC10DF039C10CF038C1BE
:10E350000BF084EC05F00EC05CF10DC05BF10CC05D
:10E360005AF10BC059F1580E0E6E330E0D6E360E6B
:10E370000C6E6D0E0B6E5CC112F05BC111F05AC1D8
:10E3800010F059C10FF04AEC09F00EC05CF10DC05D
:10E390005BF10CC05AF10BC059F12BC20EF02AC22E
:10E3A0000DF029C20CF028C20BF084EC05F00EC071
:10E3B00060F10DC05FF10CC05EF10BC05DF1DE0ECF
:10E3C0000E6E1E0E0D6E040E0C6E6F0E0B6E60C187
:10E3D00012F05FC111F05EC110F05DC10FF04AECA8
:10E3E00009F00EC060F10DC05FF10CC05EF10BC012
:10E3F0005DF12FC20EF02EC20DF02DC20CF02CC21A
:10E400000BF084EC05F00EC064F10DC063F10CC09C
:10E4100062F10BC061F18F0E0E6E7B0E0D6E080E59
:10E420000C6E6F0E0B6E64C112F063C111F062C10D
:10E4300010F061C10FF04AEC09F00EC064F10DC09C
:10E4400063F10CC062F10BC061F133C20EF032C255
:10E450000DF031C20CF030C20BF082EC05F00EC0B2
:10E4600068F10DC067F10CC066F10BC065F14C0E90
:10E470000E6E040E0D6E010E0C6E700E0B6E68C1EA
:10E4800012F067C111F066C110F065C10FF04AECDF
:10E4900009F00EC068F10DC067F10CC066F10BC049
:10E4A00065F13BC20EF03AC20DF039C20CF038C231
:10E4B0000BF084EC05F00EC06CF10DC06BF10CC0DC
:10E4C0006AF10BC069F1590E0E6E860E0D6E1B0EB1
:10E4D0000C6E6E0E0B6E6CC112F06BC111F06AC146
:10E4E00010F069C10FF04AEC09F00EC06CF10DC0DC
:10E4F0006BF10CC06AF10BC069F15CC10EF05BC13D
:10E500000DF05AC10CF059C10BF060C112F05FC19F
:10E5100011F05EC110F05DC10FF050EC08F00EC0BC
:10E5200043F20DC042F20CC041F20BC040F243C2B4
:10E530000EF042C20DF041C20CF040C20BF064C1BB
:10E5400012F063C111F062C110F061C10FF050EC24
:10E5500008F00EC043F20DC042F20CC041F20BC0F5
:10E5600040F243C20EF042C20DF041C20CF040C274
:10E570000BF068C112F067C111F066C110F065C1FF
:10E580000FF050EC08F00EC043F20DC042F20CC088
:10E5900041F20BC040F243C20EF042C20DF041C244
:10E5A0000CF040C20BF06CC112F06BC111F06AC1EB
:10E5B00010F069C10FF050EC08F00EC043F20DC02E
:10E5C00042F20CC041F20BC040F21FC20EF01EC25C
:10E5D0000DF01DC20CF01CC20BF023C212F022C2BF
:10E5E00011F021C210F020C20FF04EEC08F00EC066
:10E5F0005CF10DC05BF10CC05AF10BC059F15CC16C
:10E600000EF05BC10DF05AC10CF059C10BF03FC2C6
:10E6100012F03EC211F03DC210F03CC20FF050ECBF
:10E6200008F00EC05CF10DC05BF10CC05AF10BC0DC
:10E6300059F1340E0E6EFA0E0D6E0E0E0C6E790E32
:10E640000B6E5CC112F05BC111F05AC110F059C1E0
:10E650000FF04AEC09F00EC05CF10DC05BF10CC08C
:10E660005AF10BC059F15CC10EF05BC10DF05AC1FB
:10E670000CF059C10BF04BC212F04AC211F049C262
:10E6800010F048C20FF050EC08F00EC047F20DC079
:10E6900046F20CC045F20BC044F253C20EF052C217
:10E6A0000DF051C20CF050C20BF082EC05F00EC020
:10E6B0005CF10DC05BF10CC05AF10BC059F127C2DF
:10E6C0000EF026C20DF025C20CF024C20BF05CC186
:10E6D00012F05BC111F05AC110F059C10FF04AECB1
:10E6E00009F00EC05CF10DC05BF10CC05AF10BC01B
:10E6F00059F10E6A0D6A0C6A7F0E0B6E5CC112F046
:10E700005BC111F05AC110F059C10FF04EEC08F086
:10E710000EC05CF10DC05BF10CC05AF10BC059F199
:10E72000020E0E6E0D6A0C6A7F0E0B6E5CC112F04B
:10E730005BC111F05AC110F059C10FF04AEC09F059
:10E740000EC05CF10DC05BF10CC05AF10BC059F169
:10E750005CC10EF05BC10DF05AC10CF059C10BF059
:10E7600043C212F042C211F041C210F040C20FF099
:10E7700050EC08F00EC04FF20DC04EF20CC04DF23E
:10E780000BC04CF202014453000121E0D896020173
:10E7900045AFD88600011BE4DA0E0E6E0F0E0D6E2B
:10E7A000490E0C6E810E0B6E47C212F046C211F07C
:10E7B00045C210F044C20FF050EC08F00EC047F212
:10E7C0000DC046F20CC045F20BC044F2DBD7DA0EA6
:10E7D0000E6E0F0E0D6E490E0C6E810E0B6E47C243
:10E7E00012F046C211F045C210F044C20FF09EEC88
:10E7F00007F001081BE0DA0E126E0F0E116E490EC3
:10E80000106E810E0F6E47C20EF046C20DF045C26B
:10E810000CF044C20BF04EEC08F00EC047F20DC0F5
:10E8200046F20CC045F20BC044F2D1D71200459A13
:10E830003E50EAEC09F00EC094F10DC093F10CC00B
:10E8400092F10BC091F13F50EAEC09F00EC090F14B
:10E850000DC08FF10CC08EF10BC08DF14050EAEC71
:10E8600009F00EC08CF10DC08BF10CC08AF10BC009
:10E8700089F14150EAEC09F00EC027F10DC026F1F4
:10E880000CC025F10BC024F144C021F101012F6B14
:10E890002E6B43C02DF142C02CF10001AAEC50F0C8
:10E8A000A4C1B0F1A3C1AFF1A2C1AEF1A1C1ADF15C
:10E8B000459A9CEC52F0ACC1ECF1ABC1EBF1AAC1B2
:10E8C000EAF1A9C1E9F14596010114910001AAEC10
:10E8D00050F0126A116A400E106E830E0F6EA4C1C2
:10E8E0000EF0A3C10DF0A2C10CF0A1C10BF0E2EC3F
:10E8F00008F00EC05CF10DC05BF10CC05AF10BC00A
:10E9000059F127C10EF026C10DF025C10CF024C12C
:10E910000BF05CC112F05BC111F05AC110F059C18B
:10E920000FF050EC08F00EC027F10DC026F10CC01E
:10E9300025F10BC024F177EC51F0126AAD0E116E87
:10E940000E0E106E8E0E0F6E70C10EF06FC10DF0B8
:10E950006EC10CF06DC10BF0E2EC08F00EC07CF162
:10E960000DC07BF10CC07AF10BC079F17CC10EF0C7
:10E970007BC10DF07AC10CF079C10BF07CC112F0B3
:10E980007BC111F07AC110F079C10FF04AEC09F0A7
:10E990000EC06DF00DC06CF00CC06BF00BC06AF0D7
:10E9A00081B2A7D0C2EC6CF0B50E0E6E150E0D6ED6
:10E9B000200E0C6E760E0B6E4FC212F04EC211F08E
:10E9C0004DC210F04CC20FF0E2EC08F00EC01BF28A
:10E9D0000DC01AF20CC019F20BC018F2340E0E6EF4
:10E9E000FA0E0D6E0E0E0C6E790E0B6E1BC212F02F
:10E9F0001AC211F019C210F018C20FF04AEC09F057
:10EA00000EC01BF20DC01AF20CC019F20BC018F2A6
:10EA100045EC5CF0E10E0E6E2E0E0D6E650E0C6E6A
:10EA2000840E0B6E47C212F046C211F045C210F0C0
:10EA300044C20FF04AEC09F00EC05CF10DC05BF16E
:10EA40000CC05AF10BC059F15CC10EF05BC10DF066
:10EA50005AC10CF059C10BF097C212F096C211F0D6
:10EA600095C210F094C20FF050EC08F00EC05CF1AB
:10EA70000DC05BF10CC05AF10BC059F12E0E126E95
:10EA8000730E116E3A0E106E770E0F6E5CC10EF0A3
:10EA90005BC10DF05AC10CF059C10BF04EEC08F0FF
:10EAA0000EC0AFF20DC0AEF20CC0ADF20BC0ACF2B6
:10EAB000340E0E6EFA0E0D6E0E0E0C6E790E0B6E7F
:10EAC000AFC212F0AEC211F0ADC210F0ACC20FF086
:10EAD0004AEC09F00EC0A4F10DC0A3F10CC0A2F1E4
:10EAE0000BC0A1F10101C46BC36BC26BC16B000110
:10EAF00045D0EBEC12F0040108530001D8A42CD946
:10EB000045EC5CF0340E0E6EFA0E0D6E0E0E0C6EB1
:10EB1000790E0B6E97C212F096C211F095C210F0EA
:10EB200094C20FF04AEC09F00EC05CF10DC05BF12D
:10EB30000CC05AF10BC059F10FC30EF00EC30DF00B
:10EB40000DC30CF00CC30BF05CC112F05BC111F0F3
:10EB50005AC110F059C10FF050EC08F00EC0A4F1EA
:10EB60000DC0A3F10CC0A2F10BC0A1F123C3C4F1ED
:10EB700022C3C3F121C3C2F120C3C1F101011C6949
:10EB80001B691A691969459E00014EEC57F0E10EA8
:10EB90000E6E2E0E0D6E650E0C6E840E0B6EE4C1A5
:10EBA00012F0E3C111F0E2C110F0E1C10FF04AEC44
:10EBB00009F00EC0A4F10DC0A3F10CC0A2F10BC06E
:10EBC000A1F1126A116A700E106E820E0F6EA4C14E
:10EBD0000EF0A3C10DF0A2C10CF0A1C10BF0E2EC4C
:10EBE00008F00EC0A4F10DC0A3F10CC0A2F10BC03F
:10EBF000A1F1B9EC59F00E6A0D6A700E0C6E820E1E
:10EC00000B6EE4C112F0E3C111F0E2C110F0E1C1FA
:10EC10000FF04AEC09F00EC0A4F10DC0A3F10CC036
:10EC2000A2F10BC0A1F1340E0E6EFA0E0D6E0E0E97
:10EC30000C6E790E0B6EA4C112F0A3C111F0A2C12B
:10EC400010F0A1C10FF04AEC09F00EC0A4F10DC004
:10EC5000A3F10CC0A2F10BC0A1F1D8C1C4F1D7C17E
:10EC6000C3F1D6C1C2F1D5C1C1F121EC67F0E4C155
:10EC7000A4F1E3C1A3F1E2C1A2F1E1C1A1F1D8C1C4
:10EC8000C4F1D7C1C3F1D6C1C2F1D5C1C1F1BDEC48
:10EC900054F0D8C1C4F1D7C1C3F1D6C1C2F1D5C1B6
:10ECA000C1F10301DD530001D8A470EC5AF0E10E6C
:10ECB0000E6E2E0E0D6E650E0C6E840E0B6EE4C184
:10ECC00012F0E3C111F0E2C110F0E1C10FF04AEC23
:10ECD00009F00EC003F10DC002F10CC001F10BC030
:10ECE00000F1E10E0E6E2E0E0D6E650E0C6E840E92
:10ECF0000B6EC4C112F0C3C111F0C2C110F0C1C18A
:10ED00000FF04AEC09F00EC0FFF00DC0FEF00CC091
:10ED1000FDF00BC0FCF0CEEC0AF012000300FED7B1
:10ED200004010D6B0C6B0B6B0A6B416B406B3F6B03
:10ED30003E6B426B70C135F46FC134F46EC133F475
:10ED40006DC132F41BC22DF41AC22CF419C22BF47B
:10ED500018C22AF400011200D896FDAFD8860BE441
:10ED6000010EFF5D000EFE59A00EFD59820EFC59EA
:10ED700002E3D6DF1200E4C10EF0E3C10DF0E2C100
:10ED80000CF0E1C10BF084EC05F00EC01DF40DC0D9
:10ED90001CF40CC01BF40BC01AF404011B9FD8C157
:10EDA0000EF0D7C10DF0D6C10CF0D5C10BF082EC3E
:10EDB00005F00EC025F40DC024F40CC023F40BC0E4
:10EDC00022F4239FFFC30EF0FEC30DF0FDC30CF031
:10EDD000FCC30BF01DC412F01CC411F01BC410F0D6
:10EDE0001AC40FF04AEC09F00EC02DF00DC02CF043
:10EDF0000CC02BF00BC02AF02DC00EF02CC00DF073
:10EE00002BC00CF02AC00BF025C412F024C411F062
:10EE100023C410F022C40FF04AEC09F00EC003F432
:10EE20000DC002F40CC001F40BC000F42A51020121
:10EE3000185D11E104012B510201195D0CE104017F
:10EE40002C5102011A5D07E104012D5102011B5DE5
:10EE50000001D8B431D170C10EF06FC10DF06EC198
:10EE60000CF06DC10BF035C412F034C411F033C492
:10EE700010F032C40FF04EEC08F00EC039F40DC0A3
:10EE800038F40CC037F40BC036F40E6AC00E0D6EA9
:10EE9000280E0C6E8F0E0B6E39C412F038C411F0B0
:10EEA00037C410F036C40FF04AEC09F00EC039F444
:10EEB0000DC038F40CC037F40BC036F40E6A0D6A7E
:10EEC000160E0C6E890E0B6E39C412F038C411F098
:10EED00037C410F036C40FF09EEC07F0010802E0D2
:10EEE0001FDFEBD01BC20EF01AC20DF019C20CF0DE
:10EEF00018C20BF084EC05F00EC03DF40DC03CF4DC
:10EF00000CC03BF40BC03AF4480E0E6E510E0D6E61
:10EF1000470E0C6E8B0E0B6E3DC412F03CC411F00C
:10EF20003BC410F03AC40FF0E2EC08F00EC015F448
:10EF30000DC014F40CC013F40BC012F42DC40EF069
:10EF40002CC40DF02BC40CF02AC40BF084EC05F09B
:10EF50000EC031F40DC030F40CC02FF40BC02EF4F1
:10EF6000480E0E6E510E0D6E470E0C6E8B0E0B6E14
:10EF700031C412F030C411F02FC410F02EC40FF0C1
:10EF8000E2EC08F00EC019F40DC018F40CC017F430
:10EF90000BC016F419C40EF018C40DF017C40CF011
:10EFA00016C40BF015C412F014C411F013C410F001
:10EFB00012C40FF04EEC08F00EC029F40DC028F476
:10EFC0000CC027F40BC026F429C40EF028C40DF0A1
:10EFD00027C40CF026C40BF039C412F038C411F069
:10EFE00037C410F036C40FF0E2EC08F00EC029F47C
:10EFF0000DC028F40CC027F40BC026F404014251C4
:10F00000EAEC09F041C412F040C411F03FC410F022
:10F010003EC40FF04AEC09F00EC02DF00DC02CF0EC
:10F020000CC02BF00BC02AF02DC00EF02CC00DF040
:10F030002BC00CF02AC00BF029C412F028C411F028
:10F0400027C410F026C40FF050EC08F00EC041F4B5
:10F050000DC040F40CC03FF40BC03EF4422B4251B3
:10F06000EAEC09F00EC012F00DC011F00CC010F067
:10F070000BC00FF041C40EF040C40DF03FC40CF0C3
:10F080003EC40BF0E2EC08F00EC041F40DC040F4B9
:10F090000CC03FF40BC03EF470C135F46FC134F4C2
:10F0A0006EC133F46DC132F41BC22DF41AC22CF4BC
:10F0B00019C22BF418C22AF400010E6A0D6A340E2C
:10F0C0000C6E860E0B6E03C112F002C111F001C16D
:10F0D00010F000C10FF09EEC07F0010816E00E6A78
:10F0E0000D6A0C6A0B6A03C412F002C411F001C469
:10F0F00010F000C40FF04EEC08F00EC003F40DC089
:10F1000002F40CC001F40BC000F403C40EF002C4FE
:10F110000DF001C40CF000C40BF041C412F040C467
:10F1200011F03FC410F03EC40FF050EC08F00EC0D8
:10F1300021F40DC020F40CC01FF40BC01EF4240EEB
:10F140000E6E7B0E0D6E550E0C6E810E0B6E21C475
:10F1500012F020C411F01FC410F01EC40FF04AECCE
:10F1600009F00EC007F40DC006F40CC005F40BC086
:10F1700004F407C40EF006C40DF005C40CF004C47A
:10F180000BF011C412F010C411F00FC410F00EC433
:10F190000FF04AEC09F09AEC09F00BC00DF40CC02A
:10F1A0000CF40DC00BF404010A6F0E6A0D6A0C6AB0
:10F1B0007F0E0B6E21C412F020C411F01FC410F09A
:10F1C0001EC40FF09EEC07F00108000105E00401E9
:10F1D0000D6B0C6B0B6B0A6B00011200800E016E45
:10F1E00026EC00F0470E1EEC02F0500E1EEC02F072
:10F1F000530E1EEC02F03D0E1EEC02F040507BEC74
:10F2000000F03A0E1EEC02F03F507BEC00F03A0E9C
:10F210001EEC02F03E507BEC00F0200E1EEC02F0E3
:10F22000550E1EEC02F0540E1EEC02F0430E1EECC6
:10F2300002F0480EF3EC02F0800E016EC00E26ECD8
:10F2400000F0B8C10EF0B7C10DF0B6C10CF0B5C1F9
:10F250000BF0030EADEC00F03A0E1EEC02F0F0C124
:10F260000EF0EFC10DF0EEC10CF0EDC10BF0030E8E
:10F27000ADEC00F01200126A116A480E106E850E95
:10F280000F6E04019751EAEC09F0E2EC08F00EC0B1
:10F2900096F40DC095F40CC094F40BC093F40101E6
:10F2A0000551EAEC09F096C412F095C411F094C42B
:10F2B00010F093C40FF050EC08F00EC096F40DC09F
:10F2C00095F40CC094F40BC093F4126A116A700E9A
:10F2D000106E840E0F6E96C40EF095C40DF094C49B
:10F2E0000CF093C40BF0E2EC08F00EC096F40DC0E5
:10F2F00095F40CC094F40BC093F482C40BF083C457
:10F300000CF0ECEC09F096C412F095C411F094C422
:10F3100010F093C40FF050EC08F00EC096F40DC03E
:10F3200095F40CC094F40BC093F40001120004EEA9
:10F3300086F014EE44F092C4F3FF020EE5EC03F005
:10F34000EF6A04EE86F02FEC00F00401976F0001E5
:10F35000120004EE89F014EE44F092C4F3FF030EA1
:10F36000E5EC03F0EF6A04EE89F02FEC00F0040105
:10F37000826F20C083F40001120004EE44F0040107
:10F380009251EB50986F922B2C0E985D0001F5E195
:10F390001200670EAF6E8386A0EC02F02408FCE139
:10F3A000A0EC02F04708F8E1A0EC02F05008F4E10C
:10F3B000A0EC02F05208F0E1A0EC02F04D08ECE104
:10F3C000A0EC02F04308E8E1A0EC02F02C08E4E134
:10F3D00004EE44F03C0EF36EA0EC02F0EE6EF32E61
:10F3E000FBD7010E0401926F0001A1DF97C440F02A
:10F3F000030E0401926F00019ADF97C43FF0050EDF
:10F400000401926F000193DF97C43EF0B6DF04EE73
:10F4100044F004019251EB50436F410E435D0001F3
:10F42000D8A4B9D7AADF0401922B000180DF040120
:10F43000836B97C482F4020E9227000178DF97C491
:10F4400005F1030E04019227000171DF14DF96C459
:10F45000B8F195C4B7F194C4B6F193C4B5F18DDF9A
:10F4600004EE44F004019251EB50846F530E845D1E
:10F47000000118E10E6A0D6A800E0C6E7F0E0B6E95
:10F48000B8C112F0B7C111F0B6C110F0B5C10FF09C
:10F490004AEC09F00EC0B8F10DC0B7F10CC0B6F1DE
:10F4A0000BC0B5F1AA6A1E0EA96E0101B551E5ECBB
:10F4B00002F0B651E5EC02F0B751E5EC02F0B851BC
:10F4C000E5EC02F0000159DF0401922B000141DF5D
:10F4D000030E0401922700012ADF97C405F1030EF1
:10F4E00004019227000123DFC6DE96C4F0F195C423
:10F4F000EFF194C4EEF193C4EDF13FDF04EE44F07C
:10F5000004019251EB50856F570E855D000118E1A3
:10F510000E6A0D6A800E0C6E7F0E0B6EF0C112F03B
:10F52000EFC111F0EEC110F0EDC10FF04AEC09F09F
:10F530000EC0F0F10DC0EFF10CC0EEF10BC0EDF11B
:10F54000AA6A1A0EA96E0101ED51E5EC02F0EE5126
:10F55000E5EC02F0EF51E5EC02F0F051E5EC02F0E1
:10F5600000010BDF0ADF09DF0401922B0001DFDE5F
:10F5700097C441F0020E040192270001D8DE97C41F
:10F5800044F0020E040192270001D1DED00E0401E6
:10F590009725436A426E070E432200011FDE83ACAB
:10F5A000FED78396330EAF6E1200D896030179A56D
:10F5B000D88600010EE40301DF53000103E18392CA
:10F5C000808A04D0FA0E18EC03F083820301798F4D
:10F5D000858D000112000301DF53000102E1809AD2
:10F5E00001D0839283EC85F01200D896030179A5AF
:10F5F000D886000111E40301DF53000106E1838294
:10F60000320E18EC03F0808A04D0FA0E18EC03F0E6
:10F6100084800301798F859D000112000301DF536F
:10F6200000010CE1809AD896030179A5D8860001E3
:10F6300003E4320E18EC03F0839201D0849083EC43
:10F6400085F0120003017931E83200010EE3030175
:10F65000DF53000103E18094848004D0FA0E18EC9B
:10F6600003F080840301798F859B00011200030160
:10F67000DF53000102E1849001D0809480EC85F09A
:10F68000120003017931E832000111E30301DF5375
:10F69000000106E18084320E18EC03F0848004D06F
:10F6A000FA0E18EC03F0808A0301798F858B000134
:10F6B00012000301DF5300010BE184900301793153
:10F6C000E832000103E3320E18EC03F0809401D01D
:10F6D000809A80EC85F0120003017931E832000154
:10F6E00011E3800E016E26EC00F0400EF3EC02F008
:10F6F000056A47C320F046C31FF07EEC00F0480EB9
:10F70000F3EC02F0120031C375F030C374F02FC374
:10F7100073F02EC372F035C379F034C378F033C37D
:10F7200077F032C376F00301F7BF0DD0F651F71131
:10F730000001D8A44CD0010E0301F45D100EF55960
:10F740000001D8B044D00E6A0D6A200E0C6E820EF5
:10F750000B6E31C312F030C311F02FC310F02EC363
:10F760000FF04AEC09F00EC075F00DC074F00CC03B
:10F7700073F00BC072F075C00EF074C00DF073C062
:10F780000CF072C00BF09AEC09F00BC04FF30CC0F8
:10F790004EF30DC04DF303014C6F126A116A200E37
:10F7A000106E820E0F6E4CC30BF04DC30CF04EC3A7
:10F7B0000DF04FC30EF0EEEC09F0E2EC08F00EC0D5
:10F7C00075F00DC074F00CC073F00BC072F0030143
:10F7D000FBBF0DD0FA51FB110001D8A44CD0010E93
:10F7E0000301F85D100EF9590001D8B044D00E6A3B
:10F7F0000D6A200E0C6E820E0B6E35C312F034C3F0
:10F8000011F033C310F032C30FF04AEC09F00EC010
:10F8100079F00DC078F00CC077F00BC076F079C0AD
:10F820000EF078C00DF077C00CF076C00BF09AECBB
:10F8300009F00BC04FF30CC04EF30DC04DF30301A4
:10F840004C6F126A116A200E106E820E0F6E4CC33E
:10F850000BF04DC30CF04EC30DF04FC30EF0EEECA9
:10F8600009F0E2EC08F00EC079F00DC078F00CC0A1
:10F8700077F00BC076F00001E86A030179B3010E5E
:10F88000336EE86A79B5010E3316000120E0800E70
:10F89000016E26EC00F05F0EF3EC02F075C00EF086
:10F8A00074C00DF073C00CF072C00BF0020EADEC22
:10F8B00000F03A0E1EEC02F079C00EF078C00DF0A8
:10F8C00077C00CF076C00BF0020EADEC00F0E86AE9
:10F8D000030179B3010E336E010E79B5E86A331670
:10F8E000000115E0800E016E26EC00F0010EAA6EFC
:10F8F000C70EA96EF5EC02F075C00EF074C00DF0E5
:10F9000073C00CF072C00BF0020EADEC00F0010EF3
:10F91000030179B3E86A336EE86A79B5010E3316EC
:10F92000000115E0800E016E26EC00F0010EAA6EBB
:10F93000CB0EA96EF5EC02F079C00EF078C00DF098
:10F9400077C00CF076C00BF0020EADEC00F0176A39
:10F95000030179B3172A000E06EC00F0336E176A24
:10F9600079B5172A000E06EC00F03312000115E0FD
:10F9700050C317F0000E06EC00F0336E51C317F0C1
:10F98000000E06EC00F0331203E02A0E1EEC02F02B
:10F99000800E016E480EF3EC02F01200800E016E34
:10F9A000C00E26EC00F0620EF3EC02F040507BEC4F
:10F9B00000F03A0E1EEC02F03F507BEC00F03A0EE5
:10F9C0001EEC02F03E507BEC00F0480EF3EC02F02F
:10F9D00012000301F0530001D8A481D004010D519D
:10F9E0000C110B110A11000105E1010E0401096F50
:10F9F00000010AD0186A3EC017F01C6A060E1B6E82
:10FA00008DEC03F01FC009F4010E04010953D8A4C2
:10FA1000000E336E08C417F0000E06EC00F033162B
:10FA2000E86A81B2010E3316010E80B8E86A331617
:10FA3000010E0301F353D8A4000E331600011AE09F
:10FA4000800E016EC00E26EC00F0030EAA6E510E61
:10FA5000A96EF5EC02F0056A0DC42DF00CC42CF073
:10FA60000BC42BF00AC42AF0E7EC01F0480EF3ECCB
:10FA700002F034D0800E016EC00E26EC00F08FC371
:10FA8000AAFF8EC3A9FFF5EC02F003C10EF002C17C
:10FA90000DF001C10CF000C10BF0020EADEC00F056
:10FAA0003A0E1EEC02F0FFC00EF0FEC00DF0FDC0DD
:10FAB0000CF0FCC00BF0020EADEC00F0010E0301E7
:10FAC000DA5D000106E1800E016E530EF3EC02F0E8
:10FAD00005D0800E016E480EF3EC02F002D0030157
:10FAE000F00700011200800E016EC00E26EC00F03F
:10FAF000030EAA6E480EA96EF5EC02F0480EF3EC68
:10FB000002F012006BC3D4F381A202D00301D48FA0
:10FB10000001010E0301F35D000102E10301D48D38
:10FB20000001560EA8EC02F0470EA8EC02F0410EC0
:10FB3000A8EC02F00301D451A8EC02F0010100513D
:10FB4000A8EC02F00151A8EC02F00251A8EC02F07E
:10FB50000351A8EC02F00001FC51A8EC02F0FD51A9
:10FB6000A8EC02F0FE51A8EC02F0FF51A8EC02F064
:10FB700003012E51A8EC02F02F51A8EC02F03051F5
:10FB8000A8EC02F03151A8EC02F03251A8EC02F0DE
:10FB90003351A8EC02F03451A8EC02F03551A8EC36
:10FBA00002F000011200F5D8D896030179A7D88693
:10FBB000000103E45FEC82F002D03FEC82F07DECC8
:10FBC00081F0D896030179A9D886000103E4EDEC11
:10FBD00083F002D02FEC83F01200030176516DEC1C
:10FBE00002F0010E066EF40E036E83EC02F00001CB
:10FBF0002FE30301766F83EC02F0000129E3030198
:10FC0000776F83EC02F0000123E30301786F1A6A37
:10FC1000196A010E186E176A226A216A206A77C370
:10FC20001FF0A4EC03F01AC02DF019C02CF018C07E
:10FC30002BF017C02AF078512A2400016E6F000EB5
:10FC40002B206F6F000E2C20706F000E2D20716F17
:10FC500012008380110E0301766F0001BEDFD8967B
:10FC600071BFD88610E4715307E1705105E1090EA8
:10FC70006E5D070E6F5907E3100E6E5F0E0E6F5B21
:10FC8000000E705B715B126A116A200E106E820E9C
:10FC90000F6E6EC00BF06FC00CF070C00DF071C035
:10FCA0000EF0EEEC09F0E2EC08F00EC035F30DC0FA
:10FCB00034F30CC033F30BC032F335C3EFF334C36A
:10FCC000EEF333C3EDF332C3ECF335C30EF034C3BC
:10FCD0000DF033C30CF032C30BF0E7C312F0E6C3F0
:10FCE00011F0E5C310F0E4C30FF050EC08F00EC0C3
:10FCF00035F30DC034F30CC033F30BC032F3100EE8
:10FD00000301766F000169DF126A116A200E106E1E
:10FD1000820E0F6E6EC00BF06FC00CF070C00DF055
:10FD200071C00EF0EEEC09F0E2EC08F00EC0A5F3A5
:10FD30000DC0A4F30CC0A3F30BC0A2F38390410E3B
:10FD40000301696F6A6FA5C3EBF3A4C3EAF3A3C30E
:10FD5000E9F3A2C3E8F3A5C30EF0A4C30DF0A3C357
:10FD60000CF0A2C30BF0E3C312F0E2C311F0E1C345
:10FD700010F0E0C30FF050EC08F00EC0A5F30DC07A
:10FD8000A4F30CC0A3F30BC0A2F300017DEC81F03F
:10FD9000120080B802D00301DA6B03017931E83236
:10FDA000000143E3D896030179A7D88600012DE42A
:10FDB00083848298010E066EF40E036E83EC02F0CB
:10FDC00020E30301696F83EC02F000011AE30301F1
:10FDD000466F83EC02F0000114E30301476F83ECEC
:10FDE00002F000010EE303014A6F83EC02F0000110
:10FDF00008E30301526F83EC02F0000102E3030108
:10FE0000536F0001828883940ED0F2AE02D0F29E2E
:10FE1000FCD7010E03EC03F00301466F2BC047F340
:10FE2000F28E410E696F000106D00301696B476BCA
:10FE3000466B536B526B0001D896030179A5D886A7
:10FE4000000143E4D896030179A9D88600012DE486
:10FE500083808492010E066EF40E036E83EC02F032
:10FE600020E303016A6F83EC02F000011AE303014F
:10FE7000486F83EC02F0000114E30301496F83EC47
:10FE800002F000010EE303014B6F83EC02F000016E
:10FE900008E30301546F83EC02F0000102E3030165
:10FEA000556F0001848283900ED0F2AE02D0F29E94
:10FEB000FCD7000E03EC03F00301486F2BC049F39D
:10FEC000F28E410E6A6F000106D003016A6B496B26
:10FED000486B556B546B0001120080A825D10301BB
:10FEE000853500010DE20101036B026B016B006BB4
:10FEF0000001FF6BFE6BFD6BFC6B0301858FD86B04
:10FF00000301D753000102E1828601D082968386E5
:10FF1000410EA8EC02F0200EA8EC02F0040E016ED7
:10FF200031C30EF030C30DF02FC30CF02EC30BF015
:10FF3000020EADEC00F0200EA8EC02F035C30EF07E
:10FF400034C30DF033C30CF032C30BF0020EADEC32
:10FF500000F0200EA8EC02F00301D8517BEC00F079
:10FF60000D0EA8EC02F00001ACA2FDD70301D7539F
:10FF7000000102E1829601D082860301D96B066AF4
:10FF8000320E036E326A056A33EC00F00001D8A02D
:10FF9000D0D00301D96F056A33EC00F00001D8A07E
:10FFA000C8D00301586F20C059F3056A33EC00F044
:10FFB0000001D8A0BED003015A6F20C05BF3056AD0
:10FFC00033EC00F00001D8A0B4D00301D86F8396C1
:10FFD000430ED95D0001D8A46AD0126A116A480E96
:10FFE000106E850E0F6E59C30CF058C30BF0ECEC7D
:10FFF00009F0E2EC08F00EC003F10DC002F10CC0F4
:020000040001F9
:1000000001F10BC000F18C0E03015B5D000139E3CF
:1000100005E1A10E03015A5D000133E3A00E0301C7
:100020005A5F8C0E5B5B126A116A480E106E850E69
:100030000F6E5BC30CF05AC30BF0ECEC09F0E2EC72
:1000400008F00EC02DF00DC02CF00CC02BF00BC032
:100050002AF00E6A0D6A0C6A0B6A2DC012F02CC0D1
:1000600011F02BC010F02AC00FF04EEC08F00EC0BB
:10007000FFF00DC0FEF00CC0FDF00BC0FCF0000165
:1000800016D0126A116A480E106E850E0F6E5BC391
:100090000CF05AC30BF0ECEC09F0E2EC08F00EC0E7
:1000A000FFF00DC0FEF00CC0FDF00BC0FCF0440EE4
:1000B0000301D95D000109E1440E0301D85D00018F
:1000C00003E1010E0301DA6F0001450E0301D95D62
:1000D000000108E1450E0301D85D000102E10301C2
:1000E000DA6B0001C00E0301D915766FC00E765D84
:1000F000000118E13F0E0301D9153E6E59C33FF0D0
:1001000058C340F05BC341F05AC344F0D00ED82529
:10011000436A426E070E4322000173EC7DF00F0E1E
:100120000301F06F000103D00301859FD86B00012C
:10013000120083961200060E03016B150A6A096EFF
:100140000A5009100001D8A466D031C30EF030C3A4
:100150000DF02FC30CF02EC30BF0A5C312F0A4C3F7
:1001600011F0A3C310F0A2C30FF04EEC08F00EC0C4
:10017000A9F30DC0A8F30CC0A7F30BC0A6F3A9C345
:100180000EF0A8C30DF0A7C30CF0A6C30BF00C9E95
:100190009AEC09F00DC0ABF30301AA6FAA51AB11A1
:1001A000000138E10E6A0D6A700E0C6E820E0B6E45
:1001B00031C312F030C311F02FC310F02EC30FF073
:1001C0004AEC09F00EC02DF00DC02CF00CC02BF045
:1001D0000BC02AF02DC00EF02CC00DF02BC00CF07F
:1001E0002AC00BF0A5C312F0A4C311F0A3C310F0F2
:1001F000A2C30FF050EC08F00EC0A5F30DC0A4F39D
:100200000CC0A3F30BC0A2F3040E0301A25F02E231
:100210003684A26B00011200180E03016B150A6AE6
:10022000096E0A5009100001D8A466D035C30EF03B
:1002300034C30DF033C30CF032C30BF0A5C312F07E
:10024000A4C311F0A3C310F0A2C30FF04EEC08F04A
:100250000EC0A9F30DC0A8F30CC0A7F30BC0A6F302
:10026000A9C30EF0A8C30DF0A7C30CF0A6C30BF0F2
:100270000C9E9AEC09F00DC0ABF30301AA6FAA51D2
:10028000AB11000138E10E6A0D6A700E0C6E820E21
:100290000B6E35C312F034C311F033C310F032C308
:1002A0000FF04AEC09F00EC02DF00DC02CF00CC080
:1002B0002BF00BC02AF02DC00EF02CC00DF02BC07F
:1002C0000CF02AC00BF0A5C312F0A4C311F0A3C315
:1002D00010F0A2C30FF050EC08F00EC0A5F30DC053
:1002E000A4F30CC0A3F30BC0A2F3040E0301A25F9E
:1002F00002E23684A26B00011200366AA5C30EF03A
:10030000A4C30DF0A3C30CF0A2C30BF09AEC09F048
:100310000DC0BCF30301BB6F400E366E010EBC5D19
:1003200000011FE305E1680E0301BB5D000119E355
:10033000126A116A340E106E870E0F6EA5C30EF08E
:10034000A4C30DF0A3C30CF0A2C30BF04EEC08F055
:100350000EC031F30DC030F30CC02FF30BC02EF3E1
:1003600008D0A5C331F3A4C330F3A3C32FF3A2C3B2
:100370002EF30301A25300011EE0D8960301A3AFA0
:10038000D886000118E40E6A0D6A340E0C6E870ED2
:100390000B6EA5C312F0A4C311F0A3C310F0A2C347
:1003A0000FF050EC08F00EC031F30DC030F30CC06C
:1003B0002FF30BC02EF312000301B953000120E10B
:1003C00003016F51EAEC09F00EC012F00DC011F0FC
:1003D0000CC010F00BC00FF0A5C30EF0A4C30DF0BD
:1003E000A3C30CF0A2C30BF04EEC08F00EC0A5F3B3
:1003F0000DC0A4F30CC0A3F30BC0A2F3000116D0F0
:1004000003016F51EAEC09F0A5C312F0A4C311F087
:10041000A3C310F0A2C30FF050EC08F00EC0A5F378
:100420000DC0A4F30CC0A3F30BC0A2F30001A5C33D
:10043000EBF3A4C3EAF3A3C3E9F3A2C3E8F3A5C3B0
:100440000EF0A4C30DF0A3C30CF0A2C30BF0E3C3E2
:1004500012F0E2C311F0E1C310F0E0C30FF050EC72
:1004600008F00EC0A5F30DC0A4F30CC0A3F30BC09D
:10047000A2F30301AE530001D8A45DDE1200030114
:100480007931E8320001D8A0120041C312F040C314
:1004900011F03FC310F03EC30FF047C30CF046C34A
:1004A0000BF0ECEC09F0E2EC08F00EC0A5F30DC087
:1004B000A4F30CC0A3F30BC0A2F37EDF1200030170
:1004C0007931E8320001D8A01200410E030146251F
:1004D0002A6E000E47212B6E4A512A24566F000EB9
:1004E0002B20576F5751535D000105E10301565111
:1004F000525D000117E04D0E030146252A6E000EE5
:1005000047212B6E4A512A24566F000E2B20576F1D
:100510005751535D000105E103015651525D000141
:10052000D8A4120003014A51EAEC09F041C312F0C9
:1005300040C311F03FC310F03EC30FF04AEC09F086
:100540000EC03DF30DC03CF30CC03BF30BC03AF3BF
:100550003DC312F03CC311F03BC310F03AC30FF09F
:1005600047C30CF046C30BF0ECEC09F0E2EC08F0EA
:100570000EC0A5F30DC0A4F30CC0A3F30BC0A2F3EF
:1005800000011ADF12000301BA53000120E1030148
:100590006E51EAEC09F00EC012F00DC011F00CC063
:1005A00010F00BC00FF0A5C30EF0A4C30DF0A3C351
:1005B0000CF0A2C30BF04EEC08F00EC0A5F30DC07A
:1005C000A4F30CC0A3F30BC0A2F3000116D00301E7
:1005D0006E51EAEC09F0A5C312F0A4C311F0A3C355
:1005E00010F0A2C30FF050EC08F00EC0A5F30DC040
:1005F000A4F30CC0A3F30BC0A2F30001A5C3EFF357
:10060000A4C3EEF3A3C3EDF3A2C3ECF3A5C30EF0B2
:10061000A4C30DF0A3C30CF0A2C30BF0E7C312F008
:10062000E6C311F0E5C310F0E4C30FF050EC08F09E
:100630000EC0A5F30DC0A4F30CC0A3F30BC0A2F32E
:100640000301AE530001D8A40CEC81F0A5C335F32F
:10065000A4C334F3A3C333F3A2C332F31200D89676
:10066000030179B5D8860001D8A6120045C312F05F
:1006700044C311F043C310F042C30FF049C30CF060
:1006800048C30BF0ECEC09F0E2EC08F00EC0A5F367
:100690000DC0A4F30CC0A3F30BC0A2F374DF1200CF
:1006A00003014B51EAEC09F00EC012F00DC011F03D
:1006B0000CC010F00BC00FF049C30CF048C30BF096
:1006C000ECEC09F0E2EC08F00EC0A5F30DC0A4F3C9
:1006D0000CC0A3F30BC0A2F399C40BF09AC40CF0A6
:1006E000ECEC09F00EC012F00DC011F00CC010F0CF
:1006F0000BC00FF0A5C30EF0A4C30DF0A3C30CF004
:10070000A2C30BF04EEC08F00EC0A5F30DC0A4F38D
:100710000CC0A3F30BC0A2F3126AC00E116E4C0EF4
:10072000106E880E0F6EA5C30EF0A4C30DF0A3C308
:100730000CF0A2C30BF0E2EC08F00EC0A5F30DC064
:10074000A4F30CC0A3F30BC0A2F3A5C30EF0A4C383
:100750000DF0A3C30CF0A2C30BF0FBEC03F00EC032
:10076000A5F30DC0A4F30CC0A3F30BC0A2F3870E36
:100770000E6EF90E0D6E220E0C6E7C0E0B6EA5C366
:1007800012F0A4C311F0A3C310F0A2C30FF04AECFF
:1007900009F00EC0A5F30DC0A4F30CC0A3F30BC069
:1007A000A2F3A5C30EF0A4C30DF0A3C30CF0A2C323
:1007B0000BF063C312F062C311F061C310F060C3A9
:1007C0000FF04AEC09F00EC0A5F30DC0A4F30CC065
:1007D000A3F30BC0A2F300011200D896030179B570
:1007E000D8860001D8A61200410E030148252A6EC2
:1007F000000E49212B6E4B512A24566F000E2B20E0
:10080000576F5751555D000105E103015651545D85
:10081000000117E04D0E030148252A6E000E492104
:100820002B6E4B512A24566F000E2B20576F5751B9
:10083000555D000105E103015651545D0001D8A446
:100840001200010E04019B5D000102E129DF2ED0A0
:1008500003014B51EAEC09F045C312F044C311F017
:1008600043C310F042C30FF04AEC09F00EC03DF351
:100870000DC03CF30CC03BF30BC03AF33DC312F088
:100880003CC311F03BC310F03AC30FF049C30CF066
:1008900048C30BF0ECEC09F0E2EC08F00EC0A5F355
:1008A0000DC0A4F30CC0A3F30BC0A2F300016BDED8
:1008B000120080B812D045A410D017EC74F081B2A9
:1008C00006D003018F6B590E8E6F000104D0030117
:1008D0008F6B5C0E8E6F000145941200050E0301B4
:1008E000746F756B00011200D896010114A5D886AB
:1008F000000107E403016B53000103E08180EEDF98
:100900001200010E0301755D0001D8B48190120040
:100910000301C2BF0AD0000EC45D000EC359360EDB
:10092000C259850EC15900011EE2D89603016BA978
:10093000D886000118E435C30EF034C30DF033C37C
:100940000CF032C30BF0C4C312F0C3C311F0C2C326
:1009500010F0C1C30FF09EEC07F0010803E0010E98
:100960000301C76F00010301C653000120E1030129
:10097000C52900011CE0D89603016BA7D8860001A9
:1009800016E4C5C30BF0C6C30CF0ECEC09F035C39C
:1009900012F034C311F033C310F032C30FF09EECE9
:1009A00007F0010803E0010E0301C76F0001120008
:1009B000010E0301BE5DFE0ED8B4BD5D000128E24C
:1009C000D89603016BA5D886000122E4CFC30EF0B0
:1009D000CEC30DF0CDC30CF0CCC30BF0EEEC09F0A0
:1009E0000EC012F00DC011F00CC010F00BC00FF0D3
:1009F000D3C30EF0D2C30DF0D1C30CF0D0C30BF0B3
:100A0000D6EC07F0010803E0010E0301C76F0001F7
:100A1000010E0301C05DFE0ED8B4BF5D00011FE2F0
:100A200003016B31E83200011AE3CBC30EF0CAC3F5
:100A30000DF0C9C30CF0C8C30BF0EEEC09F0D3C342
:100A400012F0D2C311F0D1C310F0D0C30FF0D6EC26
:100A500007F0010803E0010E0301C76F0001120057
:100A6000010E0301BE5DFE0ED8B4BD5D000124E29F
:100A7000D89603016BA5D88600011EE4BDC30BF018
:100A8000BEC30CF0ECEC09F00EC012F00DC011F07A
:100A90000CC010F00BC00FF031C30EF030C30DF0DE
:100AA0002FC30CF02EC30BF09EEC07F0010803E0FF
:100AB000010E0301C76F0001010E0301C05DFE0EB0
:100AC000D8B4BF5D00011BE203016B31E8320001C5
:100AD00016E3BFC30BF0C0C30CF0ECEC09F031C35C
:100AE00012F030C311F02FC310F02EC30FF09EECA4
:100AF00007F0010803E0010E0301C76F00011200B7
:100B000070C350F3120070C351F312000301C76B9E
:100B1000D896010114B7D886000102E4A1DF71D094
:100B20000301BE53000105E1B40E0301BD5D0001E8
:100B30000EE3980E0301BD25C86FFE0EBE21C96FDE
:100B4000FF0ECA6BCA23CB6BCB23000107D0030176
:100B5000CB6BCA6BBEC3C9F3BDC3C8F30301C0539B
:100B6000000105E1B40E0301BF5D00010EE3980E24
:100B70000301BF25CC6FFE0EC021CD6FFF0ECE6BE3
:100B8000CE23CF6BCF23000107D00301CF6BCE6BF9
:100B9000C0C3CDF3BFC3CCF300010E6A0D6A340E9F
:100BA0000C6E860E0B6E31C312F030C311F02FC3E2
:100BB00010F02EC30FF0D6EC07F0010819E0126A0E
:100BC000116A340E106E870E0F6E31C30EF030C3F3
:100BD0000DF02FC30CF02EC30BF04EEC08F00EC03E
:100BE000D3F30DC0D2F30CC0D1F30BC0D0F308D0B7
:100BF00031C3D3F330C3D2F32FC3D1F32EC3D0F319
:100C0000D7DE86DE010E0301C75D000106E1929684
:100C1000809603016B6B000104D0928680A6FBECEA
:100C20000AF082AA13D0010E0301DA5D00010EE181
:100C3000DBC36BF3430E0301D95D000106E11E0E19
:100C40000301D8156B6F6BC3DBF300010301799FC0
:100C5000E86A66B3010E336E010E6BB3E86A3316B1
:100C6000000104E059EC7BF0030166930001E86A9F
:100C7000030166B5010E336E010E6BB5E86A3316DB
:100C8000000104E037EC7BF0030166950001E86A9F
:100C9000030166B7010E336E010E6BB7E86A3316B7
:100CA000000104E0EBEC7AF0030166970001E86ACA
:100CB000030166B9010E336E010E6BB9E86A331693
:100CC000000104E00EEC7BF0030166990001010EC7
:100CD00003015053D8A4000E336E010E5153D8A413
:100CE000000E33160001D8A45ED004019C999C9B91
:100CF00003016B31E832000109E3D896030185BB9B
:100D0000D886000102E404019C890001D896030101
:100D10006BA5D886000109E4D896030185ABD88677
:100D2000000102E404019C890001D89603016BA72D
:100D3000D886000108E403018535E836000102E2A7
:100D400004019C8B0001D89603016BA9D886000191
:100D500008E403018535E836000102E304019C8BB9
:100D60000001D89604019CA9D88600010BE4030178
:100D70005053000106E080948490180E03016B1715
:100D800066170001D89604019CABD88600010BE4DD
:100D900003015153000106E08392809A060E03017D
:100DA0006B17661700010301D8926BB3D88201015B
:100DB000D8B2148DD8A2149D0301D8926BB5D882F5
:100DC0000101D8B2148BD8A2149B0301D8926BB73F
:100DD000D8820101D8B2148FD8A2149F030179815F
:100DE0006BA97991010114350001D8B0D5EC7AF0E6
:100DF000D896010114ABD8860001D8A622EC7BF06E
:100E000001011435E8360001D8B041EC7BF0030154
:100E10007931000108E3D896030179A1D886000151
:100E2000D8A6F5EC7AF003017935000102E36BC333
:100E300066F3120031C30EF030C30DF02FC30CF077
:100E40002EC30BF003C112F002C111F001C110F06A
:100E500000C10FF09EEC07F0010804E004019C873C
:100E6000000102D004019C85000131C30EF030C3A3
:100E70000DF02FC30CF02EC30BF099C312F098C3E2
:100E800011F097C310F096C30FF09EEC07F0010825
:100E900002E004019C95000195C30EF094C30DF08F
:100EA00093C30CF092C30BF031C312F030C311F0B6
:100EB0002FC310F02EC30FF09EEC07F0010802E0E4
:100EC00004019C970001E86A04019CB7010E336E8F
:100ED000E86A9CB5010E331600012DE031C30EF017
:100EE00030C30DF02FC30CF02EC30BF095C312F0DE
:100EF00094C311F093C310F092C30FF09EEC07F06F
:100F0000010819E099C30EF098C30DF097C30CF0D7
:100F100096C30BF031C312F030C311F02FC310F0A1
:100F20002EC30FF09EEC07F0010805E00101149BB1
:100F3000149D0001120031C30EF030C30DF02FC319
:100F40000CF02EC30BF003C112F002C111F001C16D
:100F500010F000C10FF09EEC07F0010805E0010160
:100F6000148D149B000103D00101149D148B00010A
:100F7000120035C30EF034C30DF033C30CF032C38E
:100F80000BF0FFC012F0FEC011F0FDC010F0FCC06D
:100F90000FF09EEC07F0010804E004019C810001C1
:100FA00002D004019C83000135C30EF034C30DF060
:100FB00033C30CF032C30BF0A1C312F0A0C311F085
:100FC0009FC310F09EC30FF09EEC07F0010802E0F3
:100FD00004019C9300019DC30EF09CC30DF09BC3C4
:100FE0000CF09AC30BF035C312F034C311F033C3C5
:100FF00010F032C30FF09EEC07F0010802E004018C
:101000009C910001E86A04019CB1010E336EE86A0C
:101010009CB3010E331600012EE035C30EF034C32D
:101020000DF033C30CF032C30BF09DC312F09CC320
:1010300011F09BC310F09AC30FF09EEC07F001086B
:101040001AE0A1C30EF0A0C30DF09FC30CF09EC325
:101050000BF035C312F034C311F033C310F032C3B8
:101060000FF09EEC07F0010806E00101149F030158
:1010700079910001120035C30EF034C30DF033C373
:101080000CF032C30BF0FFC012F0FEC011F0FDC037
:1010900010F0FCC00FF09EEC07F0010806E0010123
:1010A000148F03017991000104D00101149F030101
:1010B00079810001120003C10EF002C10DF001C1DF
:1010C0000CF000C10BF07EC312F07DC311F07CC3A5
:1010D00010F07BC30FF050EC08F00EC095F30DC07C
:1010E00094F30CC093F30BC092F303C10EF002C152
:1010F0000DF001C10CF000C10BF07EC312F07DC3F6
:1011000011F07CC310F07BC30FF04EEC08F00EC062
:1011100099F30DC098F30CC097F30BC096F3FFC082
:101120000EF0FEC00DF0FDC00CF0FCC00BF082C351
:1011300012F081C311F080C310F07FC30FF050ECA8
:1011400008F00EC09DF30DC09CF30CC09BF30BC0C8
:101150009AF3FFC00EF0FEC00DF0FDC00CF0FCC015
:101160000BF082C312F081C311F080C310F07FC373
:101170000FF04EEC08F00EC0A1F30DC0A0F30CC0B0
:101180009FF30BC09EF3D896010114B7D8860001D7
:1011900002E450DE40D0010101BF0AD0000E035D21
:1011A000000E0259340E0159860E0059000104E266
:1011B0000301AC6B000103D0010E0301AC6F03010E
:1011C0002FBF0AD0000E315D000E3059340E2F595A
:1011D000860E2E59000104E20301AD6B000103D01D
:1011E000010E0301AD6F0301AC51AD5D000102E1E1
:1011F00021DE11D00301AC51AD5D000103E201011C
:10120000148B149D0301AD51AC5D000103E201019B
:10121000148D149B0001ADDE03016B6B0101D892AC
:1012200014BDD8820301D8B26B83D8A26B9301019D
:10123000D89214BBD8820301D8B26B85D8A26B9523
:101240000101D89214BFD8820301D8B26B87D8A20B
:101250006B976B8979A16B99000112000301DC5334
:10126000000118E1D896030179A9D886000103E4AA
:10127000EDEC83F002D02FEC83F0D896030179A730
:10128000D886000103E45FEC82F002D03FEC82F0EC
:101290007DEC81F06DEC7FF0410E0301695D000192
:1012A00003E183EC7BF007D0410E03016A5D00018E
:1012B000D8B483EC7BF012000EEC7BF0EBEC7AF010
:1012C00059EC7BF037EC7BF058EC11F015D159EC70
:1012D00084F080A811D0010E0301D65D000103E166
:1012E000CEEC7CF008D0020E03018F6FDC0E8E6F07
:1012F0000001E9EC7CF002D0E9EC7CF00301DC5366
:10130000000103E1C9EC7EF002D029EC7EF0A6DFFB
:101310004D0E0301695D0001D8B46CEC7BF0010E49
:101320000301D55D0001D8B482EC7DF00101148F7A
:1013300083AC149F147F0301798183AE7991797115
:10134000D896010114AFD886000102E40301799117
:101350000101148D83A8149D147D148B83AA149B02
:10136000147BD89614ADD886000102E40101149BC9
:1013700003016B6B0101D89214BDD8820301D8B26E
:101380006B83D8A26B930101D89214BBD88203015E
:10139000D8B26B85D8A26B950101D89214BFD882C0
:1013A0000301D8B26B87D8A26B976B8979A16B992F
:1013B000000174EC84F082A47FD786EC85F082AAC9
:1013C00086D759EF8DF00301F353000103E159EC87
:1013D00084F021D0220EDCEC02F00101006FDEEC83
:1013E00002F0016FDEEC02F0026FDEEC02F0036F40
:1013F000260EDCEC02F00001FC6FDEEC02F0FD6F6B
:10140000DEEC02F0FE6FDEEC02F0FF6F010E030176
:101410008F6FB40E8E6F0301DC53000103E1C9EC42
:101420007EF002D029EC7EF019DF010E0301D55DBC
:101430000001D8B482EC7DF080A811D0010E030128
:10144000D65D000103E1CEEC7CF008D0020E030172
:101450008F6FDC0E8E6F0001E9EC7CF002D0E9ECBE
:101460007CF029DE74EC84F082A426D782AA59EF9E
:101470008DF086EC85F082BAA6D759EF8DF0839275
:10148000809A809484900CEEFFF0ED6AE950EA10A7
:10149000FCE1EF6A1E0E3E6E3F6E0C0E406E0F0EAC
:1014A000416E060E446E070E436ED90E426E020E5A
:1014B0000301F06F19EC00F0000185EC0AF0800EDA
:1014C000016E26EC00F0010EAA6ECF0EA96EF5ECAF
:1014D00002F0800E016EC00E26EC00F0020EAA6E25
:1014E000B30EA96EF5EC02F083ACC9EC79F00B0EEB
:1014F0001C6EB80E19EC03F0828884820301DA6B4B
:10150000000EDCEC02F0F26FD892F2B1D882010149
:10151000D8B21485D8A214950301D892F2B3D88218
:101520000101D8B21487D8A21497D89614B5D886DA
:101530000001D8A68190020EDCEC02F00301706F6E
:10154000010EDCEC02F0726F798372A179937985D8
:1015500072A37995798772A57997798972A7799914
:10156000030EDCEC02F05C6FDEEC02F05D6FDEEC93
:1015700002F05E6FDEEC02F05F6F5DBF0AD0000E1E
:101580005F5D000E5E59200E5D59830E5C590001AF
:1015900007E203015F6B5E6B200E5D6F830E5C6F75
:1015A0000001070EDCEC02F00301606FDEEC02F0DC
:1015B000616FDEEC02F0626FDEEC02F0636F61BF20
:1015C0000AD0000E635D000E6259200E6159830E31
:1015D0006059000107E20301636B626B200E616FCB
:1015E000830E606F00010B0EDCEC02F003016F6FE5
:1015F0000C0EDCEC02F06E6F100EDCEC02F0716F82
:101600007151020DF3CFBDF3F4CFBEF30F0EDCEC3E
:1016100002F0716F7151020DF3CFBFF3F4CFC0F33D
:10162000120EDCEC02F0C16FDEEC02F0C26FDEECF9
:1016300002F0C36FDEEC02F0C46F110EDCEC02F0BE
:10164000716FC66B71C3C5F30D0EDCEC02F0716FE8
:10165000126A116A200E106E820E0F6E7151EAEC42
:1016600009F0E2EC08F00EC07EF30DC07DF30CC073
:101670007CF30BC07BF30E0EDCEC02F0716F126A90
:10168000116A200E106E820E0F6E7151EAEC09F095
:10169000E2EC08F00EC082F30DC081F30CC080F3C1
:1016A0000BC07FF32A0EDCEC02F0AF6FD89679B74F
:1016B000D886000102E40301AF6B0301AF530001C0
:1016C00006E10301F76BF66B040EF56FF46B000196
:1016D000010E0301AF5D000106E10301F76BF66B3C
:1016E000100EF56FF46B0001020E0301AF5D0001F7
:1016F00006E10301F76BF66B400EF56FF46B00012A
:10170000030E0301AF5D000106E10301F76B010E5B
:10171000F66FF56BF46B00015FC312F05EC311F05E
:101720005DC310F05CC30FF0F4C30BF0F5C30CF015
:10173000F6C30DF0F7C30EF0EEEC09F0E2EC08F0A2
:101740000EC041F30DC040F30CC03FF30BC03EF39D
:101750002B0EDCEC02F00301B06FD89679B9D88675
:10176000000102E40301B06B0301B053000106E184
:101770000301FB6BFA6B040EF96FF86B0001010EAD
:101780000301B05D000106E10301FB6BFA6B100E73
:10179000F96FF86B0001020E0301B05D000106E174
:1017A0000301FB6BFA6B400EF96FF86B0001030E3F
:1017B0000301B05D000106E10301FB6B010EFA6F4E
:1017C000F96BF86B0001040E0301B05D000106E146
:1017D0000301FB6BFA6B080EF96FF86B0301F8510C
:1017E000FA11FB1100010AE10301F951080A000195
:1017F00005E1010E04019B6F000102D004019B6B07
:1018000000013F0EDCEC02F00301716F840E7125C4
:1018100004019A6B996F030E9A2363C312F062C39B
:1018200011F061C310F060C30FF0F8C30BF0F9C3FF
:101830000CF0FAC30DF0FBC30EF0EEEC09F0E2EC95
:1018400008F00EC045F30DC044F30CC043F30BC0C9
:1018500042F32C0EDCEC02F00301AE6F2D0EDCEC3B
:1018600002F0B96F2E0EDCEC02F0BA6F2F0EDCEC3A
:1018700002F0D56F300EDCEC02F0D66F310EDCECEE
:1018800002F0D76F320EDCEC02F0DC6F330EDCECD2
:1018900002F0DD6F340EDCEC02F0DF6F350EDCECB5
:1018A00002F0E06FDEEC02F0E16FDEEC02F0E26FDE
:1018B000DEEC02F0E36F390EDCEC02F0E46FDEECFC
:1018C00002F0E56FDEEC02F0E66FDEEC02F0E76FAF
:1018D000160EDCEC02F00201146FDEEC02F0156F64
:1018E000DEEC02F0166FDEEC02F0176F380E126EAF
:1018F000A50E116E420E106E950E0F6E17C20EF0F1
:1019000016C20DF015C20CF014C20BF0E2EC08F098
:101910000EC017F20DC016F20CC015F20BC014F277
:101920001A0EDCEC02F00101ED6FDEEC02F0EE6F5E
:10193000DEEC02F0EF6FDEEC02F0F06F1E0EDCEC7E
:1019400002F0B56FDEEC02F0B66FDEEC02F0B76FBE
:10195000DEEC02F0B86F340E0E6EFA0E0D6E0E0E47
:101960000C6E790E0B6EB8C112F0B7C111F0B6C192
:1019700010F0B5C10FF04AEC09F00EC0B8F10DC07F
:10198000B7F10CC0B6F10BC0B5F1B8C10EF0B7C1DC
:101990000DF0B6C10CF0B5C10BF082EC05F00EC035
:1019A0002DF00DC02CF00CC02BF00BC02AF0E60E71
:1019B0000E6E220E0D6E6E0E0C6E7D0E0B6E2DC019
:1019C00012F02CC011F02BC010F02AC00FF04AEC1E
:1019D00009F00EC0FFF30DC0FEF30CC0FDF30BC009
:1019E000FCF33D0EDCEC02F00401086F010E085D13
:1019F000000107E10401116B106B100E0F6F860ED2
:101A00000E6F0001020E0401085D000107E10401F0
:101A1000116B106B580E0F6F870E0E6F0001030EC7
:101A20000401085D000107E10401116B106B220E37
:101A30000F6F890E0E6F0001040E0401085D000196
:101A400008E10401116B300E106F160E0F6F8A0E35
:101A50000E6F0001050E0401085D000108E104019C
:101A6000116B800E106F540E0F6F8A0E0E6F0001F7
:101A7000060E0401085D000107E10401116B106B03
:101A8000340E0F6F8B0E0E6F0001070E0401085D00
:101A9000000107E10401116B106B220E0F6F8C0E19
:101AA0000E6F01011493459C010E0301DE6F19ECCA
:101AB00000F0000182BA03D067EF89F006D004017C
:101AC0009C919C970001E3EF89F0F3D70300FED7C8
:021AD000FFD73E
:020000040030CA
:03000100061E0ECA
:020005008080F9
:060008003FC03FE03F4055
:0200000400F00A
:10000000000F028734000087340000000A0A0AFF4C
:10001000FFFF81A0000082200000860C43338495FE
:10002000E7D57F0000000000000000000100010093
:100030000000000100000000000000000000008738
:100040004D61676E65743D00202020202020202017
:100050002020002A2020202000533D004D3D00415B
:100060003D005554433D0048742041534C3D004CE5
:100070006F6E673D004C61743D005061726B2041B2
:100080005A3D005061726B20454C3D005365633D05
:10009000004D696E3D00486F75723D004461793DC9
:1000A000004D74683D0059723D004D656D207570BE
:1000B0006461746564004465672042656C20486F24
:1000C000723D004E6F42726B2F4E74682073746FD6
:1000D00070004272616B652F4E74682073746F708C
:1000E000004E6F42726B2F5374682073746F7000F0
:1000F0004272616B652F5374682073746F70004493
:10010000656C61793D00496E3D4E6F6E6500496ECC
